:100000000C94800D0C943D0E0C943D0E0C943D0E02
:100010000C943D0E0C943D0E0C94CF5F0C943D0E51
:100020000C943D0E0C943D0E0C943D0E0C943D0E24
:100030000C943D0E0C943D0E0C943D0E0C943D0E14
:100040000C9413590C943D0E0C943D0E0C943D0EE3
:100050000C943D0E0C943D0E0C943D0E0C943D0EF4
:100060000C943D0E0C943D0E0C943D0E0C943D0EE4
:100070000C943D0E0C943D0E0C943D0E0C943D0ED4
:100080000C943D0E0C943D0E0C943D0E0A5072657E
:10009000737320616E79206F662074686520666FC7
:1000A0006C6C6F77696E67206B6579733A002020FE
:1000B000202042202D2053656E642062726F61649F
:1000C0006361737473002020202045202D20457427
:1000D0006865726E657420636F6E74726F6C6C65A8
:1000E0007220726561642F77726974650A2020201E
:1000F000204A202D204A756D7020746F20626F6F2A
:10010000746C6F616465720A2020202053202D20BA
:100110005352414D20726561642F77726974650096
:100120002020202058202D204578697420426173BA
:10013000654D6F6E2C20636F6E6669677572652002
:100140006E6574776F726B20616E64207374617278
:10015000742057656253657276657200FFFFFF3049
:10016000FFFFFFFFFFFFFFFFFFFFFFFFFFFF5072DB
:1001700065737320616E79206B657920746F2073CD
:10018000746F700A00426164204950206164647297
:10019000657373003C48544D4C3E3C484541443ED9
:1001A0003C5449544C453E4E75742F4F532054686F
:1001B00072656164733C2F5449544C453E3C2F4852
:1001C0004541443E3C424F44593E3C68313E4E75A9
:1001D000742F4F5320546872656164733C2F6831EB
:1001E0003E0D0A003C5441424C4520424F5244458A
:1001F000523E3C54523E3C54483E48616E646C65ED
:100200003C2F54483E3C54483E4E616D653C2F5453
:10021000483E3C54483E5072696F726974793C2F75
:1002200054483E3C54483E5374617475733C2F549B
:10023000483E3C54483E4576656E743C42523E51C1
:10024000756575653C2F54483E3C54483E54696D75
:1002500065723C2F54483E3C54483E537461636B76
:100260002D3C42523E706F696E7465723C2F54484B
:100270003E3C54483E467265653C42523E53746172
:10028000636B3C2F54483E3C2F54523E0D0A003CB9
:100290002F5441424C453E3C2F424F44593E3C2F47
:1002A00048544D4C3E003C54523E3C54443E253054
:1002B00034583C2F54443E3C54443E25733C2F5408
:1002C000443E3C54443E25753C2F54443E3C5444EB
:1002D0003E25733C2F54443E3C54443E2530345814
:1002E0003C2F54443E3C54443E253034583C2F541B
:1002F000443E3C54443E253034583C2F54443E3C0C
:1003000054443E25753C2F54443E3C54443E257392
:100310003C2F54443E3C2F54523E0D0A003C48545E
:100320004D4C3E3C484541443E3C5449544C453E6E
:100330004E75742F4F532054696D6572733C2F5462
:1003400049544C453E3C2F484541443E3C424F4475
:10035000593E000D0A4350552072756E6E696E67E6
:100360002061742025752E25303475204D487A3C47
:1003700062723E0D0A003C5441424C4520424F52AD
:100380004445523E3C54523E3C54483E48616E64A3
:100390006C653C2F54483E3C54483E436F756E7428
:1003A000646F776E3C2F54483E3C54483E5469631A
:1003B0006B2052656C6F61643C2F54483E3C54483E
:1003C0003E43616C6C6261636B3C42523E416464CB
:1003D000726573733C2F54483E3C54483E43616CF5
:1003E0006C6261636B3C42523E417267756D656E33
:1003F000743C2F54483E3C2F54523E0D0A003C544E
:10040000523E3C54443E253034583C2F54443E3CEC
:1004100054443E256C753C2F54443E3C54443E2588
:100420006C753C2F54443E3C54443E253034583C7B
:100430002F54443E3C54443E253034583C2F5444C1
:100440003E3C2F54523E0D0A003C2F5441424C4535
:100450003E3C2F424F44593E3C2F48544D4C3E00A9
:100460003C48544D4C3E3C484541443E3C54495424
:100470004C453E53686F7720546872656164733CE5
:100480002F5449544C453E3C2F484541443E3C4244
:100490004F44593E3C5441424C4520424F52444502
:1004A000523E3C54523E3C54483E48616E646C653A
:1004B0003C2F54483E3C54483E547970653C2F5480
:1004C000483E3C54483E4C6F63616C3C2F54483E60
:1004D0003C54483E52656D6F74653C2F54483E3C19
:1004E00054483E5374617475733C2F54483E3C2FFE
:1004F00054523E0D0A003C54523E3C54443E25307A
:1005000034583C2F54443E3C54443E5443503C2FBA
:1005100054443E3C54443E25733A25753C2F544484
:100520003E003C54443E25733A25753C2F54443ECE
:100530003C54443E003C464F4E5420434F4C4F5297
:100540003D234343303030303E45535441424C3CD0
:100550002F464F4E543E003C2F5441424C453E3CAA
:100560002F424F44593E3C2F48544D4C3E0D0A00FB
:100570003C74723E3C74643E25733C2F74643E00B0
:100580003C74643E3C696E70757420747970653D8E
:1005900022636865636B626F7822206E616D653DD2
:1005A000222573222076616C75653D2225752220F7
:1005B0000020636865636B65643D22636865636BF7
:1005C000656422003C48544D4C3E3C484541443E05
:1005D0003C5449544C453E53686F7720506F7274B9
:1005E000733C2F5449544C453E3C2F484541443EB2
:1005F0003C424F44593E3C666F726D2061637469A2
:100600006F6E3D226367692D62696E2F736574702A
:100610006F7274732E6367692220656E63747970DC
:10062000653D22746578742F706C61696E223E207E
:100630003C5441424C4520424F524445523E3C744A
:10064000723E3C74643E4269743C2F74643E3C7458
:10065000643E373C2F74643E3C74643E363C2F74D9
:10066000643E3C74643E353C2F74643E3C74643E8E
:10067000343C2F74643E3C74643E333C2F74643EBF
:100680003C74643E323C2F74643E3C74643E313CA6
:100690002F74643E3C74643E303C2F74643E3C2FA7
:1006A00074723E0D0A003C74723E3C2F74723E0020
:1006B0003C2F7461626C653E3C2F666F726D3E0D1F
:1006C0000A3C2F626F64793E0D0A3C2F68746D6C92
:1006D0003E000A4661696C656420746F20636F6E2A
:1006E000666967757265206E6574776F726B2069D5
:1006F0006E746572666163653A2045746865726EF2
:1007000075742073746F70706564210A07000A465F
:1007100061696C656420746F20636F6E66696775CC
:100720007265206E6574776F726B20766961204404
:100730004843503A2045746865726E75742073742E
:100740006F70706564210A0700474946383961A80F
:10075000003900F7FF00000000C0C0C0FEFEFEFD33
:10076000FDFDFCFCFCFAFAFAF9F9F9F8F8F8F7F7EC
:10077000F7F6F6F6F5F5F5F4F4F4F3F3F3F1F1F139
:10078000F0F0F0EFEFEFEEEEEEEDEDEDECECECEB8C
:10079000EBEBEAEAEAE8E8E8E7E7E7E6E6E6E5E5DC
:1007A000E5E4E4E4E3E3E3E2E2E2E1E1E1E0E0E026
:1007B000DEDEDEDDDDDDDCDCDCDBDBDBDADADAD97C
:1007C000D9D9D8D8D8D7D7D7D6D6D6D5D5D5D3D3C3
:1007D000D3D2D2D2D0D0D0CECECECDCDCDCCCCCC2B
:1007E000CBCBCBC8C8C8C7C7C7C5C5C5C4C4C4C39D
:1007F000C3C3C2C2C2C1C1C1C0C0C0BFBFBFBEBEF1
:10080000BEBDBDBDBCBCBCBABABAB9B9B9B8B8B83E
:10081000B7B7B7B6B6B6B5B5B5B4B4B4B3B3B3B18C
:10082000B1B1B0B0B0AFAFAFAEAEAEADADADACACE0
:10083000ACABABABA9A9A9A8A8A8A6A6A6A5A5A537
:10084000A3A3A3A1A1A19F9F9F9E9E9E9D9D9D9CB2
:100850009C9C9B9B9B9A9A9A999999989898979700
:100860009796969695959594949493939392929245
:100870009191919090908E8E8E8D8D8D8C8C8C8B95
:100880008B8B8A8A8A8989898888888787878686E0
:100890008685858584848483838382828281818125
:1008A0008080807F7F7F7E7E7E7D7D7D7C7C7C7B6B
:1008B0007B7B7A7A7A7878787777777676767575BB
:1008C0007574747473737372727271717170707005
:1008D0006E6E6E6D6D6D6B6B6B6A6A6A6969696865
:1008E00068686666666464646363636161615F5FD0
:1008F0005F5E5E5E5C5C5C5B5B5B5A5A5A58585844
:1009000056565655555554545453535351515150AE
:1009100050504F4F4F4E4E4E4C4C4C4B4B4B4A4A07
:100920004A48484847474746464644444443434369
:100930004141414040403E3E3E3D3D3D3C3C3C3BD4
:100940003B3B3A3A3A383838373737353535323233
:10095000323030302E2E2E2C2C2C2B2B2B2A2A2AC8
:100960002828282727272525252424242222222138
:1009700021211F1F1F1D1D1D1B1B1B1919191818B5
:100980001817171716161614141412121210101026
:100990000F0F0F0D0D0D0A0A0A09090906060604B4
:1009A0000404030303020202000000000000000030
:1009B0000000000000000000000000000000000037
:1009C0000000000000000000000000000000000027
:1009D0000000000000000000000000000000000017
:1009E0000000000000000000000000000000000007
:1009F00000000000000000000000000000000000F7
:100A000000000000000000000000000000000000E6
:100A100000000000000000000000000000000000D6
:100A200000000000000000000000000000000000C6
:100A300000000000000000000000000000000000B6
:100A400000000000000000000000000000000000A6
:100A500000000000000021F90401000001002C004A
:100A6000000000A80039000008FF0003081C48B07F
:100A7000A0C18308076AA93320A1C38710234A9C19
:100A800048B1A2C58B0E49F4F20502A3C78F2043DB
:100A90008A1C39F00F00004048AA5CC9B2A5C511F4
:100AA000C24E527149B3A6CD957C4E024073B3A796
:100AB000CF9F1073C43C6907A8D1A33E2F9CD209D5
:100AC000A00FD2A7504736F050A312530083A26A5A
:100AD0006DD9A0A34A0544FE60C275F5A42C175B2E
:100AE000074E5D4143070F1B2F4C60409036A10914
:100AF000287E30ED52194353D9B2BCC4D0456A00A8
:100B0000C30E359154D9EA258C18B161BF74D13226
:100B100075E80C11130E046C75D0028C255D4C47E2
:100B2000262053ECAFE945148C82808208B469D347
:100B3000C548E931E20169051C67429916D900D020
:100B4000EBD79632DC1420A108A259BF93EB849511
:100B50008785819B05280001942A79480386001423
:100B6000CBF44939D3534008B8FFD43064502DEF4B
:100B7000E84F12CBA464F04A0930D25422EB3DA4D2
:100B80001500AF88CC085125FDC9443FB817520362
:100B90003CF8B18A7F08FE5702490F00514728A54B
:100BA000F907520BC100A0840F41C8A1422F0816BB
:100BB00033CA193770D080661409E0400849F4E15F
:100BC0004A840926C84B18157834400640ECB162B7
:100BD0008B007C044127DA41C1072CBC34C26282FD
:100BE000BB7012481A4EF8F0C2091E5800C1030F1C
:100BF0004060810729C4708418817032148E5C02B1
:100C0000B04A15A94D44C0094D14624B97277994F9
:100C100000213ADDC20A9A7F15F30B2EB3B8920A6F
:100C20002AA8A4E2CA2CB95408E79F5EFAD10408A6
:100C3000091C4440032634710727F4FDE95119804B
:100C4000462A6997C368C287185028B1C414691826
:100C500052DDA4695E64412EA0966AEAA9386284D6
:100C60000187A8B6EAEAAB3A61FF24C01CB0D66A95
:100C7000EBA41E1D30062DB7F6EA6B822081A0C5BD
:100C80002DBF166BEC5F212D41EAB1CC1A1BD203AC
:100C90003108E1C41883803264B3D89ECA52042F4D
:100CA000D4416CB6E0824A131EE1961B694B0FC813
:100CB000418CB9ECA2C9D20EBAB5DBEA242E74F18C
:100CC0000930B0AA740019F2BA5A4C0E0219F00297
:100CD0001B996C692A492530D2AFAB7690A856A2F1
:100CE00086CCB2AEB8213150856B0B9F2AC9030E5A
:100CF0003DF042148178C22BA021E54049C6A816D8
:100D0000934703139D28031361D031C825B0F88998
:100D1000E04729183231CAA6FAC2450B1B2C70D104
:100D2000000840A0810A3510E104166198F1861C84
:100D300071C801071A64709169103460E4C11D061E
:100D4000834A8C2EB0A0224A279548D2C8228CA470
:100D5000AD76249360D20929A8C0824BD7AFE66252
:100D6000091D4BB400415D066DFF60462C7FCA69CA
:100D70004B2A90F491861548E0D0C2081D583001E6
:100D8000040E30A0400208546E39020A28D0C00375
:100D9000114C60C1062254F98312549061471F7DA3
:100DA000F0B1C752A7F2928A2054E8ED305415D41E
:100DB00090072F5CF6520A2483C001850E2858F054
:100DC000DC511C38026B2C813CF182784649C0838F
:100DD0001DA65CEB5D31B6382206102658A000DF58
:100DE0000B8821FDA9C10012414F16B8408521E7AB
:100DF00025C84A2256BCF0C0EC7C0FD4832BB636F3
:100E000032414B02748003168344DFA22769C84134
:100E100007E20711100CC2569508934866B0053FCB
:100E20008442173B430F316671093B402105DB23A8
:100E3000A0440620041EC1AA121A18491D12F48BE0
:100E4000510CA20B3BF800FC34D832370C0356A2ED
:100E5000B8006FBCE00ABA694718BB68C5242C58B3
:100E6000030F4460852CBCC80BF14EF6AA43144016
:100E70002A2E484215C040862E50810940788107AD
:100E80003218449618C0089B78951A8058C52E1AB7
:100E9000A401369843277E811E61104E107100C355
:100EA00014A4C08536108213BB284B31AEE0C53A7E
:100EB00042C4001CF0C11702918953ACE215B0B0D6
:100EC000D3281EB106204C91002B1480012EC004A3
:100ED0000F32050A768C24440800010C74A0031B11
:100EE000A800032AF2802CF88229C1D8812447590E
:100EF0001319004E27ACB0002957C99214B0EE2444
:100F00008C181F2B6729121090822986601E2D775E
:100F100089910E6482296768082F87591109284230
:100F200027C460023197399104D84127B85810334B
:100F3000A7E990015C6128A7E00035B789901E7C85
:100F4000AB127BE3A6380772822C02A011E11CA72A
:100F50003823800540BC41960F0908003BE0822001
:100F60001881085508431F1C31FF8952A8E292C01E
:100F7000F8C52E1A063BAC28081BACA0430F2E2048
:100F8000AF8FC0248905B9D18D0472B05FED4404E0
:100F90006C0806EA94354766A1031CC918C522F2FD
:100FA000208624D0A0030F58C0DC7A4200033C33D3
:100FB000011C30C5513088B9AC7D491DCE18451D86
:100FC0006204948A5649201A980225A8718EB5A900
:100FD000A31BBAA8C41CA4C08208FC665E38A2A6E3
:100FE00054A78AB0D3848B029130074D67C7AC7386
:100FF000A0831A88C8804F20B3269850600767C81E
:101000008433F6E6A5AB304B1DD0584520A6808230
:10101000051072281B321455F7CAD75F09240BD369
:1010200010624183B40E5EDC60290D208112EC1049
:101030008A66980D8E1CED062DF870040D6488A24A
:10104000BEEA2BC23C23B4CE76B65E0F5DD41D87BC
:10105000321E1468E275BB4B473586C0131238E167
:101060000D93E005385285155BFF75541DE2F8C5F8
:1010700023C09082811DD100861A8B67876B5588AB
:10108000FE44402DA5C900B0A08C39EE0E45AB85BD
:1010900092943A228C666D755DE178862B06C18547
:1010A0001734605E6A3A64731072121D852085BE23
:1010B000949D6A59FB979494E182AA241D56BADA4A
:1010C0008D5E78E20F5DC841052EDBAB995475BC8F
:1010D0001B598C669A808BA55D57742892060AD09E
:1010E00033DD8D6C40097490442926898A535CE273
:1010F000107600430F3AC0801A0D8DB30D063046AE
:1011000064D29608740117376BE12C30C0BA94CCC6
:101110000D514F8D5678432CE20047C400137100E7
:101120001444A18D99EA528B6F05136EEB838A5498
:10113000A0E216D628875BB7AA0E509864A51A5964
:10114000CE70A3F21FE3D6B827079BC800448005E2
:1011500044AC82197DBAAE3ABA090C4694E1082D26
:10116000A04002A692800BD0E0DF0A883025931CB5
:10117000C12197D08BC657EEE91D07628009AC806C
:101180000644A08218C0100628E8C004DF35A47801
:10119000AD7986C0A62D1D77906E9E27CD43011593
:1011A0002C21A102566356008BED98432B65A5B404
:1011B000A8592534CE4A8BB8514518C20220814B1C
:1011C000D0661DE2500294464D6BAF0C40010D18E5
:1011D0004C00149089ED3CE303BDAAB5B09B82019D
:1011E00011CC053887D8920B3FB1002B0FFBD9FCEF
:1011F0003B7600E070B3AB30A2CAD0CE764FE63279
:10120000912E1CAB5976809232B54DEE8E84A52D71
:101210004F90C6396CF605888CBBDCF0A6221E65A3
:10122000900B177EA3080140009EE3CD6F84E01170
:10123000039658B7367EC09A7E1B7CC43786D21977
:101240006A310C3FD4AF220101003B656E6C6F67C1
:101250006F2E676966004749463839614700390093
:10126000F7FF00000000C0C0C0FEFEFEFDFDFDFC5B
:10127000FCFCFAFAFAF9F9F9F8F8F8F7F7F7F6F6E4
:10128000F6F5F5F5F4F4F4F3F3F3F1F1F1F0F0F031
:10129000EFEFEFEEEEEEEDEDEDECECECEAEAEAE886
:1012A000E8E8E7E7E7E6E6E6E5E5E5E4E4E4E3E3E6
:1012B000E3E2E2E2E1E1E1E0E0E0DEDEDEDDDDDD31
:1012C000DCDCDCDBDBDBD9D9D9D8D8D8D7D7D7D58C
:1012D000D5D5D3D3D3D2D2D2CDCDCDCACACAC6C624
:1012E000C6C5C5C5C2C2C2BEBEBEBDBDBDBCBCBCFE
:1012F000BABABAB9B9B9B8B8B8B5B5B5B4B4B4B280
:10130000B2B2B1B1B1B0B0B0AEAEAEACACACABABF2
:10131000ABA9A9A9A7A7A7A5A5A5A4A4A4A2A2A271
:10132000A1A1A1A0A0A09F9F9F9C9C9C9B9B9B99DF
:1013300099999494949393939292928C8C8C8B8B96
:101340008B88888887878785858584848482828244
:101350008181818080807F7F7F7D7D7D7C7C7C7BA7
:101360007B7B79797977777774747473737372721E
:10137000727171716F6F6F6E6E6E6D6D6D6C6C6C86
:101380006B6B6B6A6A6A69696964646463636360EE
:1013900060605F5F5F5E5E5E5C5C5C5B5B5B5A5A7D
:1013A0005A5656565555555454545151514F4F4F06
:1013B0004E4E4E4C4C4C4B4B4B484848474747468B
:1013C00046464444444343434141414040403D3DFF
:1013D0003D3737373535353232323030302B2B2BE5
:1013E0002828282525252424242222221E1E1E1DCD
:1013F0001D1D19191918181814141412121210108E
:10140000100F0F0F0D0D0D0909090606060404043F
:1014100003030302020200000000000000000000BD
:1014200000000000000000000000000000000000BC
:1014300000000000000000000000000000000000AC
:10144000000000000000000000000000000000009C
:10145000000000000000000000000000000000008C
:10146000000000000000000000000000000000007C
:10147000000000000000000000000000000000006C
:10148000000000000000000000000000000000005C
:10149000000000000000000000000000000000004C
:1014A000000000000000000000000000000000003C
:1014B000000000000000000000000000000000002C
:1014C000000000000000000000000000000000001C
:1014D000000000000000000000000000000000000C
:1014E00000000000000000000000000000000000FC
:1014F00000000000000000000000000000000000EC
:1015000000000000000000000000000000000000DB
:1015100000000000000000000000000000000000CB
:1015200000000000000000000000000000000000BB
:1015300000000000000000000000000000000000AB
:10154000000000000000000000000000000000009B
:10155000000000000000000000000000000000008B
:1015600000000021F90401000001002C000000002F
:10157000470039000008FF0003081C48B0A0C183E1
:10158000050D2460D0A041020308234A9C48D1E005
:10159000820E2864004962054C9A356FE0BC59837D
:1015A000C6CB93202F4620A8C8B26580010F38B063
:1015B0001852A5CD9F438D00E8DCC9B327A4447D14
:1015C000B4E4F070C0A551811040B438F2C50EA249
:1015D0009E50A34A05A0E80C8E0D472522D000039B
:1015E000CA9B3E83204D1D4B96A7A034310A64153B
:1015F00058C0838B267116959D4B97279A14461BCE
:10160000A850E20650DDBF801D6DF95091071840CB
:101610008F002B565C68875A898B23472E4302B272
:10162000E4CB7F0BD98888B9735D22083D8B260BEC
:10163000A9880083A3534FDDD2A0A0EAD750C52CC0
:101640002008BBF6CE2BA705DAB60DC9C7C0DDB69C
:101650001BD1D00DBCF6A112018ADBAE3341F9DFFC
:10166000447FF2B821B3850A94254CA454D932663C
:10167000CD1C3E429C97C6958304C6090F11204697
:101680001CA0A00206F1511FE96172626556F83C88
:10169000076969317B2D71F18A9871C305FEB9A67E
:1016A0001C1F5CFC20428107016748183358C0208A
:1016B00067B0F9D1850D13E4366168A9E101C50B66
:1016C000186C58516787E011C50D26B426224B913E
:1016D0002D4207163C9840C08A47D5F508216C3842
:1016E0005143080ED0E8DF5885ECA1C6143DA82070
:1016F00081863EFA07092381DC7146164F18A1C383
:101700000A23508064921396900104091470259660
:10171000608629E698649669E69968A6A9E69A6CB7
:10172000B6E9E69B70C629E79C74D669E79D78E622
:10173000A9E79E7CF6E9E79F80065A5140003BF5F9
:1017400061216E30B1C20381DA79677986CAF79870
:101750004E84A07184095766578001438144A8597B
:1017600079CAC7C821735CA103080A045A2748F83C
:10177000817AD2743399AF38C81A489CC068A39C48
:10178000125594AB9122471520694451C307990A19
:10179000E8695A90F2FA6A8F545525C81B5A08F125
:1017A0000207A99689269ECA2A4B59206F6C31845C
:1017B0000C1ECC69D8AA44259B2DA8559578C82025
:1017C0007AA4E1851340CCD0410367397A2797E7A3
:1017D000E61B00113FE41043091B44C0009E59DA88
:1017E000CBAABE08938494A0672AB925BE0923AC6E
:1017F000649249991BF1C51867ACF1C61C77ECF1EE
:10180000C720872CF2C824976CF2C928A7ACF2CA6B
:101810002CB7ECF2CB30C72CF3CC34D76CF3CD38EB
:10182000E7ACF3490101003B656E7461696C2E679A
:101830006966003C68746D6C3E0D0A3C68656164C5
:101840003E0D0A3C7469746C653E45746865726E41
:10185000757420426173654D6F6E3C2F7469746CB2
:10186000653E0D0A3C2F686561643E0D0A3C626F5F
:1018700064793E0D0A0D0A3C63656E7465723E0D17
:101880000A3C696D67207372633D22656E6C6F67F9
:101890006F2E676966223E3C696D67207372633DF7
:1018A00022656E7461696C2E676966223E3C703EEB
:1018B0000D0A3C68313E45746865726E757420424D
:1018C0006173654D6F6E2048545450205365727695
:1018D00065723C2F68313E0D0A0D0A3C612068722A
:1018E00065663D226367692D62696E2F7468726553
:1018F0006164732E636769223E4C69737420746857
:1019000072656164733C2F613E3C703E0D0A3C6120
:1019100020687265663D226367692D62696E2F7467
:10192000696D65722E636769223E4C697374207419
:10193000696D6572733C2F613E3C703E0D0A3C61DF
:1019400020687265663D226367692D62696E2F7338
:101950006F636B6574732E636769223E4C697374A1
:1019600020736F636B6574733C2F613E3C703E0D5A
:101970000A3C6120687265663D226367692D626971
:101980006E2F706F7274732E636769223E492F4FFA
:1019900020706F7274733C2F613E3C703E0D0A3CA8
:1019A0002F63656E7465723E0D0A0D0A3C2F626FDF
:1019B00064793E0D0A696E6465782E68746D6C00FA
:1019C000485454502F25642E256420256420257307
:1019D0000D0A5365727665723A2045746865726EB9
:1019E00075742025730D0A00436F6E74656E742D37
:1019F000547970653A2025730D0A00436F6E746543
:101A00006E742D4C656E6774683A20256C640D0AFF
:101A100000436F6E6E656374696F6E3A20636C6F1E
:101A200073650D0A0D0A003C48544D4C3E3C484538
:101A300041443E3C5449544C453E25642025733C6A
:101A40002F5449544C453E3C2F484541443E3C426E
:101A50004F44593E25642025733C2F424F44593E44
:101A60003C2F48544D4C3E005757572D41757468D4
:101A7000656E7469636174653A20426173696320BD
:101A80007265616C6D3D222573220D0A00FFFFFF18
:101A9000FFFFFFFFFFFFFFFF3EFFFFFF3F34353635
:101AA0003738393A3B3C3DFFFFFFFFFFFFFF0001A6
:101AB00002030405060708090A0B0C0D0E0F10118E
:101AC0001213141516171819FFFFFFFFFFFF1A1B3B
:101AD0001C1D1E1F202122232425262728292A2BCE
:101AE0002C2D2E2F30313233FFFFFFFFFFFFFFFF82
:101AF00030FFFFFFFFFFFFFFFFFFFFFFFFFFFF00C4
:101B000011241FBECFEFD0E1DEBFCDBF1AE0A0E0B1
:101B1000B1E0E2E6F7EE00E00BBF02C007900D92E5
:101B2000A430B107D9F71CE0A4E0BAE001C01D92CF
:101B3000A33BB107E1F7479A8FEF9FE0835B9C409F
:101B4000BC0183EB9CE00E94385240E060E070E012
:101B500088EF98E00E9492580E94FB1C90933C0BE7
:101B600080933B0B4091AD095091AE0964E473E062
:101B700086E493E00E94A66C0E94C958892B49F024
:101B800089E0ACE8BBE0ECE4F3E001900D928A95CB
:101B9000E1F785E593E00E94652B9091670B30910A
:101BA000680B892F83232091690B82238F3F19F0C3
:101BB000932B922B49F486E0A7E6BBE0E8E0F1E046
:101BC00001900D928A95E1F76091790B70917A0BF3
:101BD00080917B0B90917C0B0E945F29BC018AEB6A
:101BE0009AE00E94F5726091710B7091720B809176
:101BF000730B9091740B0E945F29BC018BEF9AE0EC
:101C00000E94F5726091750B7091760B8091770B45
:101C10009091780B0E945F29BC018BED9AE00E94A5
:101C2000F57286E0ABE1BBE0E7E6FBE001900D92E8
:101C30008A95E1F70E941E0F6091040A7091050ACF
:101C40006115710571F080E091E10E94385220E841
:101C500031E040E050E06FE37EE08AE593E00E94EF
:101C60008F5280E80E94D25368EE73E080E090E0EB
:101C70000E948456F9CF0C9400000C9400000E943E
:101C8000CE5528E635E040E050E06AE870E28EE0AC
:101C900091E00E948F528EEF0E94D2530E948E5389
:101CA000FDCFDF92EF92FF920F931F93CF93DF93BD
:101CB00000E0E02EF02ED02E11E0C12FC095CF7E97
:101CC000812F806187BBC8BB64E670E080E090E054
:101CD0000E94F02186B38C1711F0C827EC2A110F4F
:101CE00061F717BBEE2071F08E2D99279F938F938C
:101CF00083E191E09F938F930E94BA6D0F900F90B4
:101D00000F900F9011E015FD24C0C12FC09511BB9D
:101D1000C2BB68EE73E080E090E00E94F02180B3E7
:101D200080628C17B1F099279F938F938C2F9927FE
:101D30009F938F9387E291E09F938F930E94BA6D58
:101D4000012B8DB79EB706960FB6F8949EBF0FBEB7
:101D50008DBF110FC1F611BB002371F0802F9927A1
:101D60009F938F9383E391E09F938F930E94BA6D2B
:101D70000F900F900F900F9014E0103271F0C12F60
:101D8000C09512B9C3B968EE73E080E090E00E949C
:101D9000F02181B183628C13D12A110F71F712B92E
:101DA000DD2071F08D2D99279F938F9387E491E02B
:101DB0009F938F930E94BA6D0F900F900F900F908A
:101DC00011E0C12FC09510936100C093620068EECE
:101DD00073E080E090E00E94F02180B1806F8C136E
:101DE000F12A110FC12FDD27CF70D070209749F74E
:101DF00010926100FF2071F08F2D99279F938F9390
:101E00008BE591E09F938F930E94BA6D0F900F9096
:101E10000F900F90EE2031F4002321F4DD2011F417
:101E2000FF2019F08FEF9FEF01C0CE01DF91CF911E
:101E30001F910F91FF90EF90DF900895AF92BF92A6
:101E4000CF92DF92EF92FF920F931F93CF93DF9386
:101E5000CDB7DEB760970FB6F894DEBF0FBECDBF2B
:101E60000E9410599F938F938091060190910701D2
:101E70009F938F938FE691E09F938F930E94BA6D0B
:101E800087E891E09F938F930E94BA6D84E991E077
:101E90009F938F930E94BA6D8BE991E09F938F93EC
:101EA0000E94BA6D87EA91E00E94EB6D80913B0B36
:101EB00090913C0B2DB73EB7245F3F4F0FB6F8947F
:101EC0003EBF0FBE2DBF97FD0DC09F938F938BEA32
:101ED00091E09F938F930E94BA6D0F900F900F9097
:101EE0000F9004C081EC91E00E94EB6D88ED91E0D1
:101EF0009F938F930E94BA6D0E9407139093050AD7
:101F00008093040A9F938F938EEE91E09F938F931B
:101F10000E94BA6D88EF91E09F938F930E94BA6DF3
:101F20008091040A9091050A9093080A8093070A09
:101F300087E09AE00E94AF138093060AEDB7FEB7E0
:101F400038960FB6F894FEBF0FBEEDBF282F88233A
:101F5000D1F08091070A9091080A9F938F93822F66
:101F600099279F938F938EE092E09F938F930E9487
:101F7000BA6D2DB73EB72A5F3F4F0FB6F8943EBFFC
:101F80000FBE2DBF04C086E292E00E94EB6D8BE293
:101F900092E09F938F930E94BA6D0E94E514DC013A
:101FA000CB018093090A90930A0AA0930B0AB0937D
:101FB0000C0ABF93AF939F938F9381E492E09F931A
:101FC0008F930E94BA6D8CE492E09F938F930E944E
:101FD000BA6D0E94AC19EDB7FEB73A960FB6F894F9
:101FE000FEBF0FBEEDBF892B79F00E94EE15892B45
:101FF00029F01092DA0A82E692E00BC081E0809329
:10200000DA0A88E692E005C082E08093DA0A82E785
:1020100092E00E94EB6D8091DA0A882389F08CE7C8
:1020200092E09F938F930E94BA6D8091DA0A0F908D
:102030000F90813019F40E94261602C00E94E01A07
:1020400082E992E09F938F930E94BA6D0E94510E95
:102050000F900F90892B21F488EA92E00E94EB6D9B
:1020600080913B0B90913C0B99230CF4BFC10E94D3
:10207000841C8823E1F78CE890E00E94006E809138
:10208000040A9091050A892B21F08EEA90E00E94C3
:10209000006E86EC90E00E94006E8091040A9091A0
:1020A000050A8050904240F08091DA0A882321F09E
:1020B00080E291E00E94006E0E94841C8823E1F37C
:1020C0008032D1F32091040A3091050A90E2203049
:1020D000390720F0883799F1883589F1232B71F081
:1020E000823611F0823451F48091DA0A813019F489
:1020F0000E947D16BCCF0E94FD1AB9CF853611F023
:10210000853451F48091DA0A813019F40E94021664
:10211000AECF0E94611CABCF8A3611F08A3439F4FD
:102120008BEA92E00E94EB6D0C9400F8A0CF83370D
:1021300019F0833509F09BCF0E94451498CF809108
:10214000200B99279F938F9380911F0B99279F9323
:102150008F9380911E0B99279F938F9380911D0BD6
:1021600099279F938F9380911C0B99279F938F930F
:1021700080911B0B99279F938F9386EB92E09F93FF
:102180008F930E94BA6D60E270E08DE39BE00E9445
:102190008C1CADE3BBE0FD0101900020E9F7319715
:1021A000EA1BFB0B2DB73EB7225F3F4F0FB6F894EB
:1021B0003EBF0FBE2DBF309709F458C0CC24DD249C
:1021C000CE16DF06A4F49D9190334CF0892F8A53EC
:1021D000873028F08D508A3110F0973614F0EDE0FA
:1021E000F0E00894C11CD11CCE16DF0664F3ED307C
:1021F000F1059CF5CF0181709070E0FD2EC0F59542
:10220000E7958E179F0794F57C01EE1AFF0A81E28D
:102210009BE0E80EF91E9DE3A92E9BE0B92E6F010D
:10222000F50180810E94FC218C0184E0000F111FC8
:102230008A95E1F7F50181810E94FC21800FF70169
:1022400081937F010894C108D10822E030E0A20EFA
:10225000B31EC114D10421F709C080EE92E09F9310
:102260008F930E94BA6D0F900F9069CF8CE89BE01E
:102270009F938F9380EF92E09F938F930E94BA6D0C
:102280006FE070E0CE0101960E948C1C6AEB7AE050
:1022900081E093E00E94BE1C8AEB9AE00E94102924
:1022A000DC01CB010F900F900F900F900097A105CC
:1022B000B105E1F16BEF7AE08CE093E00E94BE1C87
:1022C0006BED7AE085E193E00E94BE1C8BED9AE015
:1022D0000E941029DC01CB010097A105B105E9F1AD
:1022E0008AEB9AE00E9410295B016C018BEF9AE067
:1022F0000E941029DC01CB01A822B922CA22DB22CC
:102300008BED9AE00E9410297B018C018BEF9AE003
:102310000E941029DC01CB01E822F9220A231B23A9
:10232000AE14BF04C006D106C1F0A1CE83E293E093
:102330009F938F930E94BA6D60E270E08DE39BE003
:102340000E948C1C0F900F9080913D0B882329F0E8
:10235000893519F0893709F08ACE82E493E00E942A
:10236000EB6D8AEB9AE00E941029DC01CB0180938F
:10237000790B90937A0BA0937B0BB0937C0B8BEF34
:102380009AE00E941029DC01CB018093710B90939D
:10239000720BA093730BB093740B8BED9AE00E94B9
:1023A0001029DC01CB018093750B9093760BA093E1
:1023B000770BB093780B86E0A7E6BBE0EBE1FBE0A0
:1023C00001900D928A95E1F70E948E2B89818823D6
:1023D00059F04FE050E0BE016F5F7F4F8CE89BE00B
:1023E0000E94227310929B0B0E94E35860960FB6D6
:1023F000F894DEBF0FBECDBFDF91CF911F910F913B
:10240000FF90EF90DF90CF90BF90AF90089585B789
:102410008F7785BF80916500816080936500809192
:102420006400816080936400809165008260809385
:1024300065008091640082608093640080916500F3
:102440008460809365008091640084608093640060
:102450001BBA9FEF9ABB809165008B7F80936500CC
:102460008091650084608093650015BA94BB0895DF
:102470008BBB8FEF8ABB809165008B7F809365005B
:1024800008959C01832F992785BB2BBB8091650004
:102490008B7F8093650065BB809165008E7F809304
:1024A0006500809165008E7F809365008091650056
:1024B00084608093650008959C01832F992785BBD4
:1024C00025BB809165008B7F8093650080916500BE
:1024D0008D7F8093650095B38091650082608093C5
:1024E000650080916500846080936500892F99273D
:1024F00008951F93CF930E940712809164008E7FEE
:10250000809364008091630080FD03C083E090E0CD
:102510005FC080916400816080936400809164005A
:102520008D7F809364008091630080FD03C084E010
:1025300090E04EC08091640082608093640080913E
:1025400064008B7F809364008091630080FD03C0F2
:1025500085E090E03DC01ABA8FEF8BBB60E170E080
:1025600080E090E00E94F02189B38F3F39F089B379
:10257000809580930F0A86E090E02AC0C1E01C2F6E
:1025800010951BBBCABB60E170E080E090E00E9448
:10259000F02189B38117B9F4CC0F89F7CBBB8FEF4A
:1025A0008ABBC4BB85BB60E170E080E090E00E9424
:1025B000F02183B38F3F99F083B3809580930F0A06
:1025C00087E090E005C088E090E002C089E090E0FC
:1025D00090930E0A80930D0A8FEF9FEF15C0C1E014
:1025E0001C2F109515BBC4BB60E170E080E090E04B
:1025F0000E94F02183B3811749F7CC0F89F7C5BB3F
:102600008FEF84BB80E090E0CF911F910895EF920F
:10261000FF920F931F93CF93DF93CDB7DEB724972D
:102620000FB6F894DEBF0FBECDBF19828FEF8A833D
:1026300085E58B838AEA8C832FEFE22EF22E0E94AF
:102640007912892B79F080E090E07CC0F8018081DC
:10265000809580930F0A1093110A0093100A81E06D
:1026600090E063C080E885BF00E011E189819A8134
:10267000AB81BC81F80180839183A283B38344E062
:1026800050E0BE016F5F7F4FC8010E949172892B9D
:1026900029F078010894E108F10806C0F1E1003062
:1026A0001F0711F400E010E100501C4FE016F10686
:1026B000E8F600E011E1E016F10660F040E051E0DC
:1026C0006FEF70E0C8010E94B07200501F4FE0161B
:1026D000F106A0F700E011E1E016F10680F1F80143
:1026E00080818F3F09F0B2CF91E09083F801808123
:1026F000891721F4990F90839923C1F7992321F425
:10270000F80180818823B1F0992329F09095F80190
:102710008081892302C0F801808180930F0A109381
:10272000110A0093100A82E090E090930E0A8093C1
:102730000D0A05C00F5F1F4FE016F10680F6C701B6
:102740008F5F904124960FB6F894DEBF0FBECDBFC9
:10275000DF91CF911F910F91FF90EF9008951F93FC
:10276000CF93DF93DC01C0E0D0E02D913C91119735
:1027700020503F4E81E0809301FFE0E0F1E1E2175D
:10278000F30738F481E08083E050FF4FE217F3074E
:10279000C8F3109200FFE0E0F1E1E217F30730F434
:1027A0001082E050FF4FE217F307D0F381E0E0E042
:1027B000FFEF8183E0E0F1E1E217F30740F480816D
:1027C000813049F0E050FF4FE217F307C0F3209744
:1027D00021F4CE0156C0EF01FACF2C1B3D0B2D93F7
:1027E0003C9311E0E12FFF27E050F1401083E050CF
:1027F000FF4F40E050E4BF01CE010E94B072FE01E5
:1028000080E4C030D80740F48081811729F43196E4
:1028100080E4E030F807C0F3E050F04480F1E0E0FD
:10282000F1E1EC17FD0740F48081882329F4E050A2
:10283000FF4FEC17FD07C0F3EC17FD0700F190E028
:102840009117C0F4E92FFF27E050F1409083FE017B
:1028500080E4C030D80740F48081891729F431968C
:1028600080E4E030F807C0F3E050F04418F09F5FD8
:10287000911740F3911718F01F5F09F0B3CF812F24
:102880009927DF91CF911F910895CF93DF93CFEFD9
:10289000DFEF8FE593E00E94EB6D8EE691E09F9372
:1028A0008F930E94CF6D0F900F9021E030E081E177
:1028B0002030380718F4F901F16101C0F901832FC4
:1028C0009927822B8083220F331F2115310579F739
:1028D00021E030E081E12030380718F4F901F1619E
:1028E00001C0F901832F9927982F922B808189139A
:1028F000EF01220F331F2115310561F768E873E1FD
:1029000080E090E00E94F0210E94841C882369F2FC
:10291000DF93CF938BE793E09F938F930E94BA6DE1
:102920000F900F900F900F90DF91CF9108958FB976
:10293000779BFECF8FB199270895B89BC09AB99A1B
:10294000BA9AC39A81E08EB98CE58DB98EB18EB9F1
:102950008FB10895C49A87E50E94971480E00E9481
:102960009714C498992708950F931F93CF93DF93DB
:10297000EC018B01C498BC9A0E949D140E94AA1479
:10298000282F87FF1BC0269526952F7088E091E0A1
:10299000F80180839183233019F480E092E009C02C
:1029A000253019F480E094E004C0273039F480E049
:1029B00098E08883998380E090E002C08FEF9FEFDA
:1029C000DF91CF911F910F910895EF92FF920F9396
:1029D0001F93CF93DF93CDB7DEB724970FB6F8944C
:1029E000DEBF0FBECDBF80E090E08B839C838983E8
:1029F0009A83BE016F5F7F4FCE0103960E94B4148D
:102A00001DB88B819C817C010027112789819A81C7
:102A10009C0144275527C801B7010E943D73DC0182
:102A2000CB01BC01CD0124960FB6F894DEBF0FBEDA
:102A3000CDBFDF91CF911F910F91FF90EF9008953F
:102A4000EF92FF921F93CF93E12C83E8F82E82E25E
:102A50008093008310E08DE893E09F938F930E9412
:102A6000BA6DC0911F8364EF71E080E090E00E9436
:102A7000F021F701C78FC0E00F900F90809107837E
:102A800087FF0FC080910A83803559F480910B83B2
:102A9000803739F489E993E00E94EB6D80E090E0A3
:102AA00022C0CF5FC43150F38CE993E00E94EB6DFC
:102AB0001A3099F484EA93E00E94EB6D149A1C9A00
:102AC00060EA76E881E090E00E94F0211C9860E9DD
:102AD00070ED83E090E00E94F0211F5F143108F454
:102AE000BACF8FEF9FEFCF911F91FF90EF90089596
:102AF00020E030E0F89480EC85BB84BB81EE8093CD
:102B0000008380E48093018385B78F7785BF9D9B89
:102B100006C02F5F3F4F41F09D99FBCF05C02F5F4F
:102B20003F4F11F09D9BFBCF85B7806885BF15BADD
:102B300014BA809100838132E1F77894232B19F441
:102B40008FEF9FEF089580E090E0089580EC85BBC3
:102B500084BB81EE8093008380E48093018385B7FA
:102B60008F7785BF30E090E09D9BFECF9D99FECF93
:102B70009F5F9B30C8F3E32FFF27E45AFE4F249159
:102B80003F5F90E89D9BFECF822F892309F0AE9A8C
:102B90009D99FECFAE989695A9F7E32FFF27E45AAB
:102BA000FE4F24913F5F90E89D9BFECF822F8923AB
:102BB00009F0AE9A9D99FECFAE989695A9F79D9B88
:102BC000FECF9D99FECF9F5F9530C8F3323158F20A
:102BD00085B7806885BF15BA14BA089580910083BF
:102BE000807C19F081E28093008380910A83909128
:102BF0000B838055904719F08FEF9FEF089580E089
:102C000090E008958EE691E09F938F930E94CF6DA0
:102C10000F900F9081E28093008380910A839091BE
:102C20000B839F938F938DEA93E09F938F930E94E2
:102C3000BA6D0E94841C0F900F900F900F90882304
:102C400049F388EB93E00E94EB6D08950F931F9377
:102C5000CF93C0E000E013E8CC2321F480910783F8
:102C6000882314F180911F83F801878F60E47DE051
:102C700083E090E00E94F02120E030E08091078323
:102C800088232CF02F5F3F4F2F3F3105BCF32F3FA0
:102C9000310554F08CE993E00E94EB6D80913B0B81
:102CA00090913C0B97FDD8CF80910A8390910B8334
:102CB000F0E780359F0729F489E993E00E94EB6DE6
:102CC00016C09F938F9389EB93E09F938F930E94FD
:102CD000BA6D0F900F900F900F90CC2331F0809130
:102CE0003B0B90913C0B992314F4C1E0B5CF80E0ED
:102CF00090E0CF911F910F9108956F927F928F92E4
:102D00009F92AF92BF92CF92DF92EF92FF920F937A
:102D10001F93CF93DF93CDB7DEB726970FB6F89406
:102D2000DEBF0FBECDBF86E03E010894611C711C62
:102D3000D301EFEDF3E001900D928A95E1F7E12CDC
:102D400093E8F92E88249924540185EE93E09F930B
:102D50008F930E94BA6D10920F830FEF0093078339
:102D60000E9420156C010F900F90892B09F08AC1E9
:102D700088EF93E09F938F930E94BA6D60E47DE0AB
:102D800083E090E00E94F0210E9478150F900F9050
:102D9000892B51F486E094E09F938F930E94BA6D43
:102DA0000E94A6150F900F9081EE8093008380EC17
:102DB000809301831092068310E210930583109292
:102DC000018360E573EC80E090E00E94F02181E2F5
:102DD0008093008388E480930E8310920A8310927C
:102DE0000B8310930C8382E080930D8380E48093A7
:102DF00004838FE5809303838CE48093018380E6D2
:102E0000809302830093078381E680930083960179
:102E1000D30120503D478D91F90181832F5F3248C6
:102E200026303105B0F320E030E020503D47F90175
:102E300010862F5F324828303105B8F38CE4F70153
:102E4000878381E28093008384E084878FEF878388
:102E5000178682E280930083158660E472E48FE037
:102E600090E00E94F0218AE194E00E94EB6D82EEF6
:102E70008093008380910383082F1127C801807CF1
:102E80009070009721F0803C910511F12EC08FE1E8
:102E900094E09F938F930E94BA6D0F900F9003FF61
:102EA00008C08AE294E09F938F930E94BA6D0F90BE
:102EB0000F9005FF08C088E394E09F938F930E94D2
:102EC000BA6D0F900F9004FF18C08DE394E00FC00F
:102ED00082E494E09F938F930E94BA6D0F900F90BD
:102EE00003FF0BC08AE294E002C08BE494E09F935E
:102EF0008F930E94BA6D0F900F9002FF08C089E572
:102F000094E09F938F930E94BA6D0F900F9003707F
:102F10001070012B41F08FE594E09F938F930E94F6
:102F2000BA6D0F900F908091048382958F709927CE
:102F3000877090709F938F9388E694E09F938F9310
:102F40000E94BA6D809105830F900F900F900F90A3
:102F50009927807C90708034910581F081349105AF
:102F60001CF4892B41F018C08038910551F0803C49
:102F7000910551F011C08FE694E008C085E794E018
:102F800005C08EE794E002C087E894E09F938F939A
:102F90000E94BA6D0F900F908AE090E00E94E46D5D
:102FA00082E28093008360E271EA87E090E00E9411
:102FB000F021BF92AF929F928F920894811C911C36
:102FC000A11CB11C80E994E09F938F930E94BA6D7D
:102FD0004CED55E0F701428785E090E0838710864D
:102FE00080E4818782E18093008320E030E08DB728
:102FF0009EB706960FB6F8949EBF0FBE8DBF8FEF9B
:10300000F701808B2F5F3F4F26303105C0F3D3018E
:1030100093012B5F3F4F8D91F701808B2A173B0760
:10302000D0F788E0808B108A20E030E0F701108A2A
:103030002F5F3F4FF5E02C3D3F07C0F382E28093C6
:10304000008320E030E08091078386FD05C02F5F7C
:103050003F4F25313105B8F320E4F701278345833D
:1030600085E090E08683248386E2809300830E943B
:10307000841C882339F460E177E280E090E00E94CC
:10308000F02191CF26960FB6F894DEBF0FBECDBFCC
:10309000DF91CF911F910F91FF90EF90DF90CF9034
:1030A000BF90AF909F908F907F906F900895782FF2
:1030B00083E080930EC0909108C09A7F986080E072
:1030C000592F5160509308C0492F4560409308C064
:1030D0008F5F8132A8F3909308C0392F346030930A
:1030E00008C0509308C0409308C0662349F09093ED
:1030F00008C0309308C0509308C0409308C008C06F
:10310000509308C0409308C0909308C0309308C003
:1031100080E0909308C0309308C08F5F8530C8F37B
:1031200020E1872F822329F0509308C0409308C0E4
:1031300004C0909308C0309308C0269591F79093EF
:1031400008C0892F99270895CF93DF93C0E0D0E07E
:1031500060E00E945718282F277F209308C0422F35
:103160004460409308C030E0209308C0409308C0FA
:10317000CC0FDD1F809108C09927969587958170A7
:103180009070C82BD92B3F5F303170F3209308C06B
:10319000CE01DF91CF910895CF93DF93EB0161E0F2
:1031A0000E945718282F782F7160709308C0682FDD
:1031B0006560609308C0809308C0382F34603093F6
:1031C00008C040E050E8CE0184239523892B29F0E4
:1031D000709308C0609308C004C0209308C0309367
:1031E00008C0569547954115510569F7277F2093EB
:1031F00008C0DF91CF910895CF93DF9360E070E82E
:1032000080E00E94CC18C0E0D0E060EA76E881E07F
:1032100090E00E94F02180E00E94A41899232CF4F1
:10322000C430D10520F52196F0CF60E47DE083E045
:1032300090E00E94F02182E10E94A41860EC7FE3FC
:1032400083E10E94CC1810920EC080E198E0809338
:103250000AC088E090E080930BC061EE71E084E0EA
:103260000E94CC18C0E0D0E0C032D10518F08FEF3A
:103270009FEF1FC0CE018F779070892B59F460E0CB
:1032800072E180E00E94CC1860E47DE083E090E091
:103290000E94F02181E00E94A41885FD08C060EE24
:1032A00073E984E090E00E94F0212196DDCF80E078
:1032B00090E0DF91CF9108951F93CF93DF93109209
:1032C0000DC010920EC0109204C080E8809305C01B
:1032D00011E010930EC0109200C0809301C060E214
:1032E0007EE480E090E00E94F02110920EC01092E7
:1032F00004C0109205C0109200C0109201C010933B
:103300000EC010920CC088E080930DC082E08093C4
:103310000EC080E4809300C0C7EED3E0809100C06F
:1033200080FF0BC060ED77E080E090E00E94F0212C
:1033300021978FEFCF3FD80789F7CD2B19F48FEF67
:103340009FEF02C080E090E0009711F08FEF9FEFB9
:10335000DF91CF911F91089580910FC0833359F46D
:1033600083E080930EC080910AC09927807F90707F
:103370008039910519F08FEF9FEF089580E090E07C
:103380000895CF93DF9315980E945C19892B19F04B
:1033900085E994E059C00D9B03C082EA94E054C0D3
:1033A00083E080930EC087E080930CC010920EC023
:1033B000109204C081E0809305C081E8809300C032
:1033C000109201C00E94FC18892B19F08CEA94E03D
:1033D0003BC082E080930EC080E2809300C0C3E6D1
:1033E000D0E0809100C080FF0BC060ED77E080E00E
:1033F00090E00E94F02121978FEFCF3FD80789F707
:10340000CD2B19F48FEF9FEF02C080E090E0892B65
:10341000E9F488E080930DC0CFEF80910CC083FD6C
:103420000CC0C15079F060ED77E080E090E00E9440
:10343000F02180910CC083FFF4CF0D990AC088EB76
:1034400094E002C08FEB94E00E94EB6D8FEF9FEF52
:1034500002C080E090E0DF91CF9108951F93CF9359
:10346000DF930E945C19892B19F185E994E005C06E
:103470008AEC94E002C08FEB94E00E94EB6D8FEF3A
:103480009FEF9AC05F934F939F938F9387ED94E044
:103490009F938F930E94BA6D8FEF9FEF2DB73EB72A
:1034A0002A5F3F4F0FB6F8943EBF0FBE2DBF84C0BA
:1034B00010E082E080930EC080E2809300C0C3E6FB
:1034C000D0E0809100C080FF0BC060ED77E080E02D
:1034D00090E00E94F02121973FEFCF3FD30789F77B
:1034E000CD2B19F48FEF9FEF02C080E090E0892B85
:1034F00009F0BECFCFEF80910CC083FD0DC0C1504D
:1035000009F4B9CF60ED77E080E090E00E94F0210F
:1035100080910CC083FFF3CF809103C0809302C0E1
:10352000109206C0109207C040E050E09A016FEF81
:103530007FEF209306C0832F9927809307C0609365
:1035400008C0822F8F5F809306C02F5F3F4F832F6D
:103550009927809307C0872F9927809308C04F5FD2
:103560005F4F615070402F5F3F4F84E040305807FD
:1035700000F340E050E09A01209306C0C901906238
:10358000892F9927809307C0809108C0909109C026
:10359000809590958417950709F074CF4F5F5F4F22
:1035A0002E5F3F4F84E04030580730F31F5F1330E9
:1035B00008F47FCF80E090E0DF91CF911F910895D4
:1035C000CF93DF930E94C119892B19F08FEB94E000
:1035D00007C00E942E1AEC01892B39F08DEE94E081
:1035E0000E94EB6D8FEF9FEF05C088EF94E00E9483
:1035F000EB6DCE01DF91CF9108958F929F92AF92A4
:10360000BF92CF92DF92EF92FF920F931F93CF93CF
:10361000DF93CDB7DEB726970FB6F894DEBF0FBEA7
:10362000CDBF86E04E010894811C911CD401EBEFC4
:10363000F4E001900D928A95E1F781E095E09F9387
:103640008F930E94BA6D0E945C190F900F90892B86
:1036500019F085E994E01AC083E080930EC087E0FA
:1036600080930CC010920EC081E8809300C010922D
:1036700001C00E94FC189C01892B59F08CEA94E04F
:1036800005C085E195E002C08BE195E00E94EB6DFD
:1036900005C181E080930EC090E0D401F901EC5F98
:1036A000FF438D9180839F5FE350F04C9630B8F3D9
:1036B00088EF94E00E94EB6DAA24BB24650160E2D0
:1036C00071EA87E090E00E94F021DF92CF92BF92F2
:1036D000AF9283E295E09F938F930E94BA6D0CEDB9
:1036E000E02E05E0F02E82E080930EC080E2809311
:1036F00000C08DB79EB706960FB6F8949EBF0FBE5A
:103700008DBF03E610E0809100C080FF0CC060ED2B
:1037100077E080E090E00E94F021015010409FEFA0
:103720000F3F190781F7012B19F48FEF9FEF02C0AC
:1037300080E090E0892B09F0A4CF88E080930DC051
:1037400080910CC083FD46C088E295E00E94EB6D3D
:1037500060E271EA87E090E00E94F02180910CC065
:1037600083FD38C080E4809300C007EE13E08091B1
:1037700000C080FF0CC060ED77E080E090E00E9428
:10378000F021015010408FEF0F3F180781F780E2C2
:10379000809300C003E610E0809100C080FF0CC061
:1037A00060ED77E080E090E00E94F0210150104051
:1037B0009FEF0F3F190781F7012B19F48FEF9FEF50
:1037C00002C080E090E0892B09F068C080910CC0B5
:1037D00083FF64C010920DC0809103C0809302C02B
:1037E000109206C080E4809307C0109208C0109227
:1037F00008C0E09208C085E090E0809309C090E0A6
:103800008FEF809308C09F5F9630D0F390E0F40173
:103810008191809308C09F5F9630D0F388E08093B9
:1038200008C0109208C01BEDE12E15E0F12E109299
:1038300008C00894E108F1088FEFE8168FEFF8064A
:10384000B1F7109208C0109208C003E610E0809112
:1038500000C080FF0CC060ED77E080E090E00E9447
:10386000F021015010409FEF0F3F190781F7012B06
:1038700019F48FEF9FEF02C080E090E0892B09F0F0
:1038800003CF80EC809300C00E94841C882331F415
:103890000894A11CB11CC11CD11C11CF26960FB6D7
:1038A000F894DEBF0FBECDBFDF91CF911F910F9176
:1038B000FF90EF90DF90CF90BF90AF909F908F9050
:1038C00008958EE691E09F938F930E94CF6D0F90A5
:1038D0000F9083E080930EC080910AC099279F9338
:1038E0008F938FE295E09F938F930E94BA6D0E9411
:1038F000841C0F900F900F900F90882351F383E456
:1039000095E00E94EB6D08955F9903C080E090E020
:1039100008958CB199270895CF92DF92EF92FF928C
:103920000F931F93CF938C016B01EE24FF240E9411
:10393000841CC60101978E159F058CF00E94841C83
:10394000C82F8823D9F3803250F099270E94E46D64
:10395000F801C1938F010894E11CF11CEACFF80132
:1039600010828AE090E00E94E46DC701CF911F9120
:103970000F91FF90EF90DF90CF9008950F931F93DA
:10398000CF93DF938C01EB01DF93CF931F930F93C2
:1039900084E495E09F938F930E94BA6D60E270E09B
:1039A0008DE39BE00E948C1C2DB73EB72A5F3F4FF2
:1039B0000FB6F8943EBF0FBE2DBF892BB1F08DE33B
:1039C0009BE00E941029DC01CB018F5F9F4FAF4F1E
:1039D000BF4F31F06DE37BE0CE010E94F57205C070
:1039E00085E891E00E94006ECFCFCE01DF91CF91AC
:1039F0001F910F9108956F927F929F92AF92BF9205
:103A0000CF92DF92EF92FF920F931F93CF93DF93AA
:103A1000CDB7DEB764970FB6F894DEBF0FBECDBF4B
:103A200084E13E010894611C711CD301EEE4F5E0D1
:103A300001900D928A95E1F788E18AB981E0982E8C
:103A4000EE246301F60181916F01A82EBB2468EE7C
:103A500073E080E090E00E94F0215F998CB1A9B8FA
:103A600068EE73E080E090E00E94F0215F998CB1F5
:103A700000E010E05F990BC068EE73E080E090E03A
:103A80000E94F0210F5F1F4F0832110598F3FF24A9
:103A900001E010E05F9B0CC08CB18032A1F4F39484
:103AA000F1E0FF1611F0C5011CC001E010E008C0F4
:103AB000FF2031F064E670E080E090E00E94F021A9
:103AC0000F5F1F4F39F7E39483E18E1508F0BACFEB
:103AD0009394EFE0E91508F0B3CF87E189B98FEF50
:103AE0009FEF64960FB6F894DEBF0FBECDBFDF9197
:103AF000CF911F910F91FF90EF90DF90CF90BF90EB
:103B0000AF909F907F906F9008950F931F93CF93E6
:103B1000DF938C01C091810BD091820B20EB35E0BB
:103B200048EC50E00E94DF492FEF3FEF4FEF5FEF8F
:103B300063EB75E0C8010E941D4AB80184E991E079
:103B40000E94816DB80184EE91E00E94816D209702
:103B500009F451C0E989FA8980819181A281B381F8
:103B60008F5E9E4BAD4ABE4D19F08DEB95E002C0C5
:103B700082EC95E09F938F938E859F8529893A8962
:103B8000821B930B9F938F938E859F859F938F931B
:103B90008B899C899F938F938D899E899F938F9307
:103BA0008D85E82FFF27EE0FFF1FE855FA4F808124
:103BB00091819F938F93888999279F938F932496C0
:103BC000DF93CF932497DF93CF9386EA92E09F937E
:103BD0008F931F930F930E945E6D0990D881C02D23
:103BE0008DB79EB746960FB6F8949EBF0FBE8DBF99
:103BF000209709F0AFCFB8018FE892E00E94816D65
:103C0000C8010E94B66B80E090E0DF91CF911F91D8
:103C10000F9108958F929F92AF92BF92CF92DF92B1
:103C2000EF92FF920F931F93CF93DF934C0120EB02
:103C300035E048EC50E00E94DF492FEF3FEF4FEFB7
:103C40005FEF63EB75E0C4010E941D4AB4018DE192
:103C500093E00E94816D0E941B577B018C0120E440
:103C600032E44FE050E00E948F7359016A01CA01AB
:103C7000B90120E432E44FE050E00E943D73DC01E2
:103C8000CB01E81AF90A0A0B1B0BC801B70124E69D
:103C900030E040E050E00E948F733F932F93BF923B
:103CA000AF9283E593E09F938F939F928F920E94B0
:103CB0005E6DC0914F0AD091500A8DB79EB708969D
:103CC0000FB6F8949EBF0FBE8DBF2097D9F1B401F7
:103CD00086E793E00E94816DEE24FF2487018E81A8
:103CE0009F81A885B985E80EF91E0A1F1B1F8C85C8
:103CF0009D859F938F938A859B859F938F938A81C0
:103D00009B81AC81BD81BF93AF939F938F931F9392
:103D10000F93FF92EF92DF93CF938EEF93E09F93F9
:103D20008F939F928F920E945E6D0990D881C02DD3
:103D30008DB79EB742960FB6F8949EBF0FBE8DBF4B
:103D4000209769F6B40189E494E00E94816DC40172
:103D50000E94B66B80E090E0DF91CF911F910F91B0
:103D6000FF90EF90DF90CF90BF90AF909F908F909B
:103D700008950F931F93CF93DF93EC0120EB35E071
:103D800048EC50E00E94DF492FEF3FEF4FEF5FEF2D
:103D900063EB75E0CE010E941D4ABE0180E694E00F
:103DA0000E94816D0FB60F92F8940091120A109143
:103DB000130A0115110509F4AFC0F801808D918D2A
:103DC000082E892F902D9F938F93648975898689FA
:103DD00097890E945F299F938F931F930F9386EF7C
:103DE00094E09F938F93DF93CF930E945E6D8DB786
:103DF0009EB70A960FB6F8949EBF0FBE8DBFF8010E
:103E0000868D978D082E892F902D9F938F93628D8D
:103E1000738D848D958D0E945F299F938F9382E28D
:103E200095E09F938F93DF93CF930E945E6D8DB744
:103E30009EB708960FB6F8949EBF0FBE8DBFF801CF
:103E4000838999278530910509F441C08630910511
:103E500094F48230910529F18330910534F4009770
:103E600009F445C00197C9F046C083309105E9F0D7
:103E70000497F9F040C08830910589F189309105A7
:103E800034F486309105D9F0079729F134C0893090
:103E90009105C9F00A9739F12EC0BE0185EC95E075
:103EA0002DC0BE018CEC95E029C0BE0184ED95E0EB
:103EB00025C0BE0185E395E00E94816D21C0BE0151
:103EC0008CED95E01BC0BE0185EE95E017C0BE01EC
:103ED0008EEE95E013C0BE0188EF95E00FC0BE01E5
:103EE00080E096E00BC0BE0188E096E007C0BE010E
:103EF00081E196E003C0BE0188E196E00E94706D0A
:103F0000BE018EE196E00E94706DF8010081118182
:103F10000115110509F051CF0F900FBEBE0187E5C5
:103F200095E00E94816DCE010E94B66B80E090E02A
:103F3000DF91CF911F910F910895CF92DF92EF9271
:103F4000FF920F931F93CF93DF93EC016B01E42E4D
:103F50007F936F9380E795E09F938F93DF93CF9349
:103F60000E945E6D2DB73EB72A5F3F4F0FB6F894A3
:103F70003EBF0FBE2DBF87E0F82E0F2D11271F93D8
:103F80000F93DF92CF9280E895E09F938F93DF931A
:103F9000CF930E945E6D8E2D992702C095958795CF
:103FA0000A95E2F72DB73EB7285F3F4F0FB6F8945A
:103FB0003EBF0FBE2DBF80FF05C0BE0181EB95E067
:103FC0000E94816DBE018BE296E00E94706D8F2D84
:103FD000FA94882391F6BE0184E396E00E94706D06
:103FE000DF91CF911F910F91FF90EF90DF90CF90D5
:103FF00008950F931F938C0120EB35E048EC50E0BF
:104000000E94DF492FEF3FEF4FEF5FEF63EB75E06B
:10401000C8010E941D4AB80184EC95E00E94816DA0
:104020004AB36CE376E0C8010E949D1F49B361E486
:1040300076E0C8010E949D1F4BB366E476E0C8019C
:104040000E949D1FB80186EA96E00E94816D47B3E9
:104050006CE476E0C8010E949D1F46B361E576E0FE
:10406000C8010E949D1F48B366E576E0C8010E9422
:104070009D1FB80186EA96E00E94816D45B36CE50C
:1040800076E0C8010E949D1FB80186EA96E00E9472
:10409000816D41B362E676E0C8010E949D1F40B386
:1040A00067E676E0C8010E949D1F42B36CE676E0A9
:1040B000C8010E949D1FB80186EA96E00E94816DAA
:1040C00042B162E776E0C8010E949D1F41B167E7F7
:1040D00076E0C8010E949D1F43B16CE776E0C801FD
:1040E0000E949D1FB80186EA96E00E94816D40B152
:1040F00062E876E0C8010E949D1FB80180EB96E05F
:104100000E94816DC8010E94B66B80E090E01F9113
:104110000F9108958091DA0A813031F445E060E032
:1041200073E881E899E005C040E060E070E08FE36B
:1041300099E00E9492588AEB9AE00E9410295B0154
:104140006C01611571058105910539F18BEF9AE0DC
:104150000E941029DC01CB017C018D01A601950193
:104160006BE17BE087E896E00E94A72A892BC9F1E2
:1041700082ED96E09F938F930E94CF6D80913B0BD1
:1041800090913C0B0F900F9097FD28C068EE73E064
:1041900080E090E00E948456F9CF20E63AEE40E0BD
:1041A00050E06BE17BE087E896E00E940844892BB1
:1041B000C1F08EE097E09F938F930E94CF6D809126
:1041C0003B0B90913C0B0F900F9097FD07C068EE52
:1041D00073E080E090E00E948456F9CFF8940E944A
:1041E000000060916D0B70916E0B80916F0B909140
:1041F000700B0E945F299F938F9380916C0B99277E
:104200009F938F9380916B0B99279F938F938091AE
:104210006A0B99279F938F938091690B99279F939E
:104220008F938091680B99279F938F938091670B51
:1042300099279F938F938CE896E09F938F930E948A
:10424000BA6D6091710B7091720B8091730B9091AC
:10425000740B0E945F299F938F9387EB96E09F9347
:104260008F930E94BA6D8AEB9AE00E941029DC01BC
:10427000CB012DB73EB72C5E3F4F0FB6F8943EBF33
:104280000FBE2DBF0097A105B10599F18BED9AE006
:104290000E941029DC01CB010097A105B10549F16D
:1042A00080913B0B90913C0B97FD0EC08BED9AE0FB
:1042B0009F938F9380EC96E09F938F930E94BA6DAB
:1042C0000F900F900F900F908BED9AE00E941029A5
:1042D000DC01CB0121E8C22E29E0D22E7C018D0128
:1042E00020E030E040E050E0CA01B9010E94C6275A
:1042F00023C02091750B3091760B4091770B509134
:10430000780B2115310541055105B1F080913B0B2A
:1043100090913C0B97FD10C0CA01B9010E945F2922
:104320009F938F9380ED96E09F938F930E94BA6D39
:104330000F900F900F900F908091DA0A813029F43E
:10434000E0919009F091910904C0E0914E09F0913B
:104350004F0967817085818592850E945F299F93AF
:104360008F9389ED96E09F938F930E94BA6D40E002
:1043700060E070E08BEC98E00E94925865E87DE187
:104380008FEF96E00E947A496AE07EE18BE097E049
:104390000E947A4969EB7EE185E197E00E947A49C3
:1043A00069EF7FE181E297E00E947A490F900F90D8
:1043B0000F900F900E94DA227C0160E570E00E946D
:1043C000A9246BE277E0C7010E94596B8C010E941F
:1043D0001C4DC8010E94086BC7010E944F26EACFFE
:1043E000161617061806190634F4000061507040BE
:1043F00080409040D1F70895982F80538A3030F450
:10440000892F992787FD9095C0970895892F815608
:10441000863038F4892F992787FD909587559040ED
:104420000895892F8154863030F4892F992787FD8C
:104430009095C797089580E090E008950F931F939B
:10444000CF93DF938C01EC01C45BDF4FE881F981EE
:10445000309759F08081918188839983CF010E94A0
:10446000B85FE881F9813097A9F7E801E8ADF9ADC7
:10447000309761F080819181E80188AF99AFCF01D9
:104480000E94B85FE8ADF9AD3097A1F7E801C05BD5
:10449000DF4FE881F981309759F0808191818883DD
:1044A0009983CF010E94B85FE881F9813097A9F71D
:1044B000DF91CF911F910F910895CF93DF93EC017E
:1044C000E091120AF091130AA2E1BAE0309771F07C
:1044D000EC17FD0729F4888199818D939C9306C080
:1044E000DF010190F081E02D309791F7EF2BA9F0DB
:1044F000CE010E941E228D859E85892B31F08F85ED
:1045000098890E94BF511D861E8682E7FE01119286
:104510008A95E9F7CE010E94BF51DF91CF910895AE
:10452000EF92FF920F931F93CF93DF937C01EB01E8
:1045300060E070E0E091120AF091130A8F01309769
:10454000E9F0808D918D8E159F0599F4828D938D64
:10455000A48DB58D82179307A407B50751F4868DF6
:10456000978D8C179D0729F48389882311F0BF014B
:1045700005C00190F081E02D309719F761157105A4
:1045800089F4F801012B71F08389813031F4808D39
:10459000918D8E159F0509F4BF010190F081E02DEA
:1045A000309791F7CB01DF91CF911F910F91FF9041
:1045B000EF9008951F93CF93DF93C0E0D0E08091F8
:1045C000140A882359F4182F0E94FE36892B09F407
:1045D00011E01093140A112309F44EC082E790E011
:1045E0000E94AA51EC01892B09F446C01B8A84E081
:1045F0008C8388E696E28D839E838BE996E28F8397
:10460000988787E697E289879A8787E997E28B8779
:104610009C8780E492E4AFE0B0E089A39AA3ABA3C7
:10462000BCA38DA39EA3AFA3B8A789A79AA7ABA746
:10463000BCA7FE01E85BFF4FCC5BDF4F80E99CE04D
:1046400088839983808391832E9628E132E02883A2
:104650003983269688EE93E088839983C855D040A5
:104660008091120A9091130A88839983298B3A8B3F
:10467000D093130AC093120ACE01DF91CF911F91FC
:1046800008950F931F93CF93DF93EC018A014FEFAF
:104690005FEF892B09F46FC080E16230780701F188
:1046A000E0E163307E0744F46230710569F06150E7
:1046B000704109F441C059C080E16530780709F1C3
:1046C0006650704139F151C001151105D9F1223000
:1046D0003105C1F5CE5ADF4FF801808191810EC0BE
:1046E0000115110579F12230310561F5C85BDF4F05
:1046F000F8018081918188839983249788839983A5
:1047000031C001151105F1F024303105D9F4C65935
:10471000DF4F08C001151105A9F02430310591F4CF
:10472000CA59DF4FF80180819181A281B3818883CA
:104730009983AA83BB8316C00115110519F0223095
:10474000310529F0C05ADF4F86E190E012C040E009
:1047500050E0BA01CE010E949B26F8018081918130
:10476000898B9A8B40E050E006C0C05ADF4F8AE345
:1047700097E288839983CA01DF91CF911F910F91AE
:104780000895CF93DF93FC01EA014FEF5FEF892B90
:1047900009F458C080E162307807D9F080E16330D5
:1047A00078073CF46230710561F06150704199F115
:1047B00043C080E165307807B1F066507041D9F0B0
:1047C0003BC0209769F12230310551F5EE5AFF4F79
:1047D00007C0209729F12230310511F5E85BFF4F22
:1047E0008081918124C02097D9F024303105C1F413
:1047F000E659FF4F07C0209799F02430310581F426
:10480000EA59FF4F80819181A281B3818883998386
:10481000AA83BB830EC0209719F02230310529F0FE
:10482000E05AFF4F86E190E00BC08189928988832E
:10483000998340E050E006C0E05AFF4F8AE397E2D8
:1048400080839183CA01DF91CF910895EF92FF9207
:104850000F931F93CF93DF93EC017A018B01A90192
:10486000892B09F45EC08B89813029F4C05ADF4F4F
:104870008DE397E254C08B89882329F0C05ADF4F1B
:1048800088E497E24CC08091490790914A070196CD
:1048900090934A07809349078091490790914A076E
:1048A000892B31F480E090E190934A078093490787
:1048B000E091120AF091130A309789F0809149072C
:1048C00090914A07082E892F902D208D318D281721
:1048D000390729F00190F081E02D309779F7309772
:1048E00091F68091490790914A07082E892F902DC3
:1048F000888F998F042E452F502D4E8F5F8FEA8E13
:10490000FB8E0C8F1D8FAF01C801B7010E94C1281B
:10491000FC01892B49F4C05ADF4F81E597E2888377
:1049200099838FEF9FEF0EC00784F089E02D878178
:104930009085A185B2858C8B9D8BAE8BBF8BCE0174
:104940000E94CC30DF91CF911F910F91FF90EF909B
:104950000895FC01CB01082E892F902D808F918F17
:10496000CF010E94AD300895CF92DF92EF92FF9277
:104970000F931F93CF93DF93EC016B018A010E9489
:104980008E53209709F450C08B898430E1F5C1140F
:10499000D10409F44CC00115110509F448C092E591
:1049A000E92EF12CEC0EFD1EF7018081918180171C
:1049B000910708F48C0149A55AA58DA19EA1481B19
:1049C000590B9A013695279536952795F7018081E1
:1049D00091818217930738F08DA99EA9841B950BAE
:1049E00080179107B8F4FE01E659FF4F40815181CD
:1049F00062817381CE01CA960E947857892BB9F4DF
:104A00008B898430C1F2C05ADF4F89E497E28883F2
:104A100099830AC088A1806188A3A801B601CE014C
:104A20000E94BB2B892B31F04FEF5FEF04C040E0B9
:104A300050E001C0A801CA01DF91CF911F910F91F1
:104A4000FF90EF90DF90CF9008952F923F924F927A
:104A50005F926F927F928F929F92AF92BF92CF920E
:104A6000DF92EF92FF920F931F93CF93DF93CDB717
:104A7000DEB726970FB6F894DEBF0FBECDBF8C0110
:104A800069837A834A010E948E530115110509F446
:104A9000E3C0F8018389843059F08389853041F07F
:104AA000005A1F4F89E497E2D8018D939C93D4C09C
:104AB000E981FA81EF2B09F4D2C08114910409F441
:104AC000CEC056E4E52EF12CE00EF11E4AE4C42ED1
:104AD000D12CC00ED11ED7012D913C91F6018081C1
:104AE000918128173907E1F4F8018389843009F0AE
:104AF000ACC0EA59FF4F4081518162817381C80186
:104B0000825B9F4F0E947857892B09F0A8C0D7017C
:104B10002D913C91F601808191812817390721F36D
:104B200036E4432E512C400E511EC801865B9F4F28
:104B30008B839C83D2018D919C91EB81FC812081A0
:104B40003181821B930B8815990508F44C0181145F
:104B5000910409F489C079016624772468147904E2
:104B600008F046C02CE4222E312C200E311ED1013B
:104B7000AD90BC90F501C188D288CE18DF08C40181
:104B8000861997098D839E83C816D90610F4CD82A5
:104B9000DE8229813A81260D371DF50187859089AE
:104BA0008E0D9F1D4D815E81BC01C9010E949E72C8
:104BB0008D819E81680E791EE80EF91E8C159D056B
:104BC00098F0D5018D919C91F10180839183D20160
:104BD0008D919C9111978E199F098D939C93C5017E
:104BE0000E94B85FEE24FF246814790408F4BACF59
:104BF000EB81FC81E082F182F80183898430A1F5A8
:104C0000EC5BFF4F80819181AC01880D991D085BA1
:104C10001F4FD8012D913C91085410402817390797
:104C200008F4C9010E5A1F4FD8012D913C9102552D
:104C3000104024173507B0F02817390798F48083FF
:104C40009183C8010E941A310FC0005A1F4F89E496
:104C500097E2F801808391834FEF5FEF06C040E059
:104C600050E003C080839183A401CA0126960FB649
:104C7000F894DEBF0FBECDBFDF91CF911F910F9192
:104C8000FF90EF90DF90CF90BF90AF909F908F906C
:104C90007F906F905F904F903F902F9008950F936B
:104CA0001F938C0140E050E0BA010E949B26C8018E
:104CB0000E94E7301F910F910895FC01892B19F490
:104CC00086E397E20895E05AFF4F8081918108952D
:104CD0000E9425250895CF92DF92EF92FF920F93C5
:104CE0001F93CF93DF936C017B018A01C0E0D0E07A
:104CF000C417D507B4F4C8018C1B9D0B97012C0F6A
:104D00003D1FAC01B901C6010E94B4241816190652
:104D10001CF08FEF9FEF06C0C80FD91FC017D10737
:104D200054F3CE01DF91CF911F910F91FF90EF903F
:104D3000DF90CF900895AF92BF92CF92DF92EF9223
:104D4000FF920F931F93CF93DF93EC015A016B01F6
:104D5000209709F498C08B89843039F0C05ADF4F0E
:104D600089E497E2888399838EC04D855E85A1147E
:104D7000B104D1F441155105A1F06F857889CE01B8
:104D80000E946B2697FF07C08F8598890E94BF51AC
:104D9000AD86BE8678C08F8598890E94BF51AD864A
:104DA000BE8640E050E087C069897A894115510587
:104DB00021F5A616B70690F0C5010E9468737C0124
:104DC0008501081B190BA801B601CE010E946B26B4
:104DD00099230CF458C0C00ED11E01C07501E11416
:104DE000F10409F467C089899A890E9433518F8739
:104DF000988B009709F447C052C0CA018A0D9B1DC9
:104E00002F8538898617970770F4240F351FA50161
:104E1000B601C9010E949E728D859E858A0D9B1DDB
:104E20008D879E8747C08B01041B150B240F351FF0
:104E3000A801B601C9010E949E72C00ED11E498907
:104E40005A896F857889CE010E946B269923ACF030
:104E5000C501801B910B8C0169897A898617970798
:104E6000C0F00E9468737C01081B190BA801B601F1
:104E7000CE010E946B2697FF09C08F8598890E94FA
:104E8000BF511D861E864FEF5FEF15C0C00ED11EAD
:104E900001C07C01E114F10439F08F859889A701E4
:104EA000B6010E949E7204C08F8598890E94BF51EE
:104EB000ED86FE86A501CA01DF91CF911F910F916A
:104EC000FF90EF90DF90CF90BF90AF900895CF927A
:104ED000DF92EF92FF920F931F93CF93DF936C01BA
:104EE0007B01EA0100E010E04115510551F0CA01D3
:104EF0000E9433518C01009721F0AE01B7010E944E
:104F0000A772AE01B801C6010E949B26EC010115F3
:104F1000110519F0C8010E94BF51CE01DF91CF9158
:104F20001F910F91FF90EF90DF90CF900895CF9356
:104F3000DF93DC01EA0140E050E06A30710549F09E
:104F40006A307105ECF06B30710579F06C307105E9
:104F5000B9F4FD01E65BFF4FAA5BBF4F8D919C91B9
:104F600020813181821B930B04C01D968D919C91F1
:104F70001E97AA27BB2788839983AA83BB8302C075
:104F80004FEF5FEFCA01DF91CF9108952F923F92CB
:104F90004F925F926F927F928F929F92AF92BF9249
:104FA000CF92DF92EF92FF920F931F93CF93DF93F5
:104FB000CDB7DEB726970FB6F894DEBF0FBECDBFD4
:104FC0002B013C0149015A01E982FA820B831C83BF
:104FD0009FEF292E392E87E1E82E8AE0F82EF7017F
:104FE0000FB6F89480818F5F80830FBE0FB60F924B
:104FF000F8948091170A813009F050C08091150A09
:105000009091160A8D839E8305E11AE00097F9F0CE
:10501000FC0186819781A085B185281739074A0749
:105020005B07A8F40D811E81D8010D90BC91A02DC5
:10503000AD83BE83109759F016968D919D910D907A
:10504000BC91A02D88169906AA06BB0658F380E1EC
:1050500090E00E9433519C01009701F148205920B3
:105060006A207B20FC0142825382648275828682A0
:105070009782A086B18689819A81AB81BC81828723
:105080009387A487B587C686D7868D819E818083C6
:105090009183D8012D933C93222433240F900FBE8B
:1050A000F7010FB6F8948081815080830FBEC10153
:1050B00026960FB6F894DEBF0FBECDBFDF91CF911D
:1050C0001F910F91FF90EF90DF90CF90BF90AF9026
:1050D0009F908F907F906F905F904F903F902F9018
:1050E0000895EF92FF920F931F93CF93DF937B016D
:1050F0008C01EA01622FE0E0F0E02430D0F5E0918D
:10510000150AF091160A3097B1F086819781A08533
:10511000B1858E219F21A023B12322813381448137
:10512000558182179307A407B50729F00190F081F4
:10513000E02D309751F73097E1F0209761F08285AC
:105140009385A485B5850097A105B10521F08883D5
:105150009983AA83BB8386859785892B51F46F5FDA
:10516000262FAE0162857385848595850E947128FE
:10517000FC01CF01DF91CF911F910F91FF90EF9034
:105180000895CF92DF92EF92FF920F931F93CF93E8
:10519000DF937B018C01EA01452B21F018821982F3
:1051A0001A821B8227E1C22E2AE0D22EF6010FB608
:1051B000F89480818F5F80830FBE20E0AE01C8012C
:1051C000B7010E947128FFEFEF16FFEFFF06FFEF18
:1051D0000F07FFEF1F0729F4A091150AB091160AD7
:1051E00007C020E0AE01C801B7010E947128DC01B0
:1051F000F6010FB6F8948081815080830FBE10971E
:1052000029F01E968D919C911F9701C0CD01DF91D1
:10521000CF911F910F91FF90EF90DF90CF90089565
:10522000CF93DF93CDB7DEB724970FB6F894DEBFE8
:105230000FBECDBFFC0119821A821B821C8240E086
:10524000DE011196808180538A3060F520E030E0E5
:10525000C90153E0880F991F5A95E1F7820F931FF8
:10526000280F391F8191280F311D20533040808134
:10527000803330F08A3320F42F3F310549F340F377
:105280002F3F310509F070F44F5F2D938E3239F0C6
:10529000443041F469817A818B819C8107C03196C9
:1052A000443080F26FEF7FEF8FEF9FEF24960FB6C1
:1052B000F894DEBF0FBECDBFDF91CF9108950F935D
:1052C0001F93CF93DF93CDB7DEB727970FB6F89430
:1052D000DEBF0FBECDBF6C837D838E839F83A8E12D
:1052E000BAE08E010C5F1F4F50E040E0F8013081C2
:1052F000832F6AE00E945C73292F832F0E945C73C6
:105300008083BE016F5F7F4FFB01E40FF11D205DC5
:1053100020834F5FF8018081882341F741504F3F40
:1053200039F0FB01E40FF11D80818D934150C8F7E6
:105330008EE28D930F5F1F4F5F5F5430B0F2119775
:105340001C9288E19AE027960FB6F894DEBF0FBE54
:10535000CDBFDF91CF911F910F9108952F923F9272
:105360004F925F926F927F928F929F92AF92BF9275
:10537000CF92DF92EF92FF920F931F93CF93DF9321
:10538000CDB7DEB72A970FB6F894DEBF0FBECDBFFC
:105390001C012A013B0148015901C982DA82EB82D2
:1053A000FC82FC010784F089E02DE987FA8741152A
:1053B00051056105710581F440906D0B50906E0BA5
:1053C00060906F0B7090700B411451046104710474
:1053D00019F48FEF9FEFA2C0E985FA8547825086C6
:1053E0006186728681149104A104B10431F48BE4C6
:1053F00097E00E9410294B015C01E985FA858786B8
:10540000908AA18AB28AA3019201282139214A21D6
:105410005B212D833E834F8358876101EE24FF2457
:105420008701A50194016D817E818F8198850E94FD
:10543000C62789819A81AB81BC810097A105B105FE
:1054400051F07C018D0120E030E040E050E0CA01E5
:10545000B9010E94C62789E0AEE5BBE0F1013296B2
:1054600001900D928A95E1F7E985FA85818188237B
:1054700079F48281882361F48381882349F48481CB
:10548000882331F48581882319F48681882351F09B
:1054900086E0A7E6BBE0E985FA85319601900D929A
:1054A0008A95E1F740926D0B50926E0B60926F0BF4
:1054B0007092700B8092710B9092720BA092730B92
:1054C000B092740B29813A814B815C8121153105A1
:1054D00041055105A9F48091750B9091760BA0912F
:1054E000770BB091780B88219921AA21BB212D81BE
:1054F0003E814F81588582179307A407B50761F055
:1055000089819A81AB81BC818093750B9093760BD6
:10551000A093770BB093780B0E948E2B2A960FB630
:10552000F894DEBF0FBECDBFDF91CF911F910F91D9
:10553000FF90EF90DF90CF90BF90AF909F908F90B3
:105540007F906F905F904F903F902F900895AF9213
:10555000BF92CF92DF92EF92FF920F931F93AA24F4
:10556000BB2465010E94BD2A1F910F91FF90EF900F
:10557000DF90CF90BF90AF9008952F923F924F92BF
:105580005F926F927F928F929F92AF92BF92CF92D3
:10559000DF92EF92FF920F931F93CF93DF93CDB7DC
:1055A000DEB724970FB6F894DEBF0FBECDBF6B8376
:1055B0007C8319012A01370148010E9475589C011A
:1055C00089839A83DC01892B09F464C01B968C9132
:1055D0001B97833009F05EC01F960D90BC91A02DE3
:1055E0008C91863071F41196EB81FC8101900D92C3
:1055F0008A95E1F77601650194018301B201A10169
:1056000044C0873109F046C0F901A188B288F5018C
:1056100021A232A243A254A2E114F1040105110512
:1056200041F48FEFE82E8FEFF82E8FEF082F8FEFDA
:10563000182FF501E1A6F2A603A714A7C5010E9441
:105640005458F501FF96AE014F5F5F4F67E171E07F
:10565000808191810E947F6A40E65AEE60E070E0AE
:10566000C5010E947857892BA9F4F50184AD8930D2
:1056700089F4C5A0D6A0E7A0F0A401A512A523A592
:1056800034A541A152A163A174A189819A810E948C
:10569000AE2902C08FEF9FEF24960FB6F894DEBFBD
:1056A0000FBECDBFDF91CF911F910F91FF90EF9073
:1056B000DF90CF90BF90AF909F908F907F906F9032
:1056C0005F904F903F902F900895CF93DF93EC0120
:1056D00040E250E060E470E08DE59BE00E9467727C
:1056E00080915D0B803239F4BE018EE59BE00E9413
:1056F000E172009781F080E2EDE5FBE011928A957E
:10570000E9F746E050E06FEF70E087E69BE00E942B
:10571000B0728FEF9FEFDF91CF910895EF92FF92DC
:105720000F931F93CF93DF9380E280935D0B8DE502
:10573000E82E8BE0F82E00E010E0C0E4D0E0CE01CF
:105740000E945F72F7016081861719F0CE010E94F6
:1057500078720894E11CF11C0F5F1F4F21960032F4
:10576000110568F380E090E0DF91CF911F910F91D8
:10577000FF90EF9008958F929F92AF92BF92CF9239
:10578000DF92EF92FF920F931F93CF93DF93EC0181
:105790007B014A0100E010E0452B41F488A19927E4
:1057A0008B709070892B11F498015BC114E188A172
:1057B00081FD18E1812F9927AC0160E480E090E041
:1057C0000E944E5E5C01009709F472C0FC01C38424
:1057D000D484888D998DF601808391838E8D9F8DE1
:1057E00082839383110F110F148788A1877F88A369
:1057F00089A59AA5ABA5BCA5082E8B2FB02D092E87
:105800009A2FA02D84839583A683B78388A184FFD4
:1058100018C080E1858788A18F7E88A3C05CDF4F98
:1058200088819981AA81BB81C054D040082E8B2FDA
:10583000B02D092E9A2FA02D80879187A287B3873C
:1058400006C0F6011586108611861286138688A179
:10585000992781FF22C0F60185858260858788A10E
:105860008D7F88A389A59AA5ABA5BCA50196A11D8E
:10587000B11D89A79AA7ABA7BCA782E0848B84E05F
:10588000858BCE5ADF4F88819981C255D040082E32
:10589000892F902D868B978B41C08114910451F1F3
:1058A000A40160E8C5010E944E5E5C01009739F4D6
:1058B000C05ADF4F87E497E288839983CBC0FC010D
:1058C00087859089A401B7010E949E7294014427A4
:1058D000552789A59AA5ABA5BCA5820F931FA41F28
:1058E000B51F89A79AA7ABA7BCA7F60185858860D5
:1058F000858714C080FF12C0F60185858160858789
:1059000088A18E7F88A389A59AA5ABA5BCA5019681
:10591000A11DB11D89A79AA7ABA7BCA7FE01EC5B8F
:10592000FF4FCE5ADF4F2081318188819981C25546
:10593000D0402817390720F4F6011686178606C0CE
:10594000022E232F302DF60126873787F601108A85
:10595000118A128A138AF5018585968521893289F3
:10596000820F931F082E892F902D7C0106E02A8D2F
:105970003B8D4C8D5D8D6C897D898E899F890E94C0
:10598000E737DC01CB01F50145855685B6010E945C
:10599000A737F50141895289678570890E94E237EE
:1059A000F601808B918B892839F48585992783703E
:1059B0009070892B09F442C0F50110821182E8AD84
:1059C000F9AD309769F4A8AEB9AEC25ADF4F0E9464
:1059D0004657DC01CB0188839983CE55D0400DC05A
:1059E00080819181892B39F00190F081E02D8081B7
:1059F0009181892BC9F7A082B1829E012C5A3F4F19
:105A0000F90180819181A281B3810097A105B1053F
:105A100081F4F60184819581A681B781082E8B2FB0
:105A2000B02D092E9A2FA02DF90180839183A28396
:105A3000B383C5010E94335F8C0101C085019801C9
:105A40004A8D5B8D6C8D7D8D86E00E943038EC0137
:105A5000892B19F02FEF3FEF04C0C8010E94B85FF7
:105A60009E01C901DF91CF911F910F91FF90EF909F
:105A7000DF90CF90BF90AF909F908F900895AF929E
:105A8000BF92CF92DF92EF92FF920F93CF93DF936B
:105A90006C01FC01A780B084C385D4858D859927CE
:105AA0009C012470307082FD78C0F601218B328B0E
:105AB00084E190E085879687288139818A819B815E
:105AC000888399832A833B838D85992784FF0FC020
:105AD00084E08D8788859985AA85BB858C839D8385
:105AE000AE83BF83188619861A861B8626C02C8132
:105AF0003D814E815F8181FF16C0DA01C901082E08
:105B00008B2FB02D092E9A2FA02D0196A11DB11D0E
:105B1000082E8B2FB02D092E9A2FA02D88879987BC
:105B2000AA87BB8704C0288739874A875B871C827E
:105B30001D821E821F8284E18D8780E58C871E86F0
:105B40001F861A8A1B8A188A198AF6018585968506
:105B5000082E892F902D7C0106E0F50124853585DE
:105B60004685578560897189828993890E94E737C4
:105B7000DC01CB01F60145855685BE010E94E23766
:105B8000888B998B9601F5014485558566857785C7
:105B9000802F0E943038892B19F4C6010E94B85F0B
:105BA00080E090E0DF91CF910F91FF90EF90DF9038
:105BB000CF90BF90AF9008950895EF92FF920F930A
:105BC0001F93CF93DF93EC018B01FC01E45BFF4F4C
:105BD00080819181009761F0FC0180819181892B06
:105BE00039F00190F081E02D80819181892BC9F7F6
:105BF00000831183DE01AA5BBF4F8D919C911197A9
:105C0000F80121893289820F931F8D939C9380E440
:105C1000E82EF12CEC0EFD1E618972899B01442750
:105C20005527F70180819181A281B381820F931F53
:105C3000A41FB51F80839183A283B383FE01EC5B15
:105C4000FF4F808191816817790718F010821182C7
:105C500004C0861B970B8083918328A1822F8061CB
:105C600088A3F80180819181892B19F0108211821B
:105C700002C0286128A3CE01825B9F4F0E94FD577E
:105C800040E050E0BA01CE010E94BB2BDF91CF91E2
:105C90001F910F91FF90EF900895CF93DF93EC0148
:105CA000FB0180899189A289B3898C8B9D8BAE8BF6
:105CB000BF8BFA01808191818E8F9F8FFB0184853C
:105CC0009585A685B7858A8F9B8FAC8FBD8FFA018E
:105CD00084819581A681B781082E8B2FB02D092E46
:105CE0009A2FA02D8CAF9DAFAEAFBFAF8DA79EA753
:105CF000AFA7B8AB0196A11DB11DC05CDF4F888373
:105D00009983AA83BB83C054D04086859785082E8B
:105D1000892F902D8DAB9EAB40E050E0FB01648558
:105D20007585868597850E94C128FC01892BE1F045
:105D30000784F089E02D838994898897FE01EE5AC3
:105D4000FF4F208131812115310519F0821793070A
:105D500010F48083918389899A8920813181281761
:105D6000390710F4298B3A8BDF91CF910895AF92C8
:105D7000BF92CF92DF92EF92FF920F931F93CF9338
:105D8000DF93EC01FB01BA01E084F1840285138505
:105D90000E2CE12E102D0F2CF02E002D89A59AA58A
:105DA000ABA5BCA58E159F05A007B10720F488A15F
:105DB000886188A3DAC0ADA0BEA0CFA0D8A4EA14A1
:105DC000FB040C051D0581F5248135814681578131
:105DD000022E252F502D032E342F402D8DA59EA54C
:105DE000AFA5B8A982179307A407B50770F02817C5
:105DF00039074A075B07C1F489A99AA9ABA9BCA9CD
:105E0000E816F9060A071B0778F086859785082E9D
:105E1000892F902D8DAB9EAB2DA73EA74FA758ABDA
:105E2000E9AAFAAA0BAB1CABEA14FB040C051D058E
:105E3000F8F0EA14FB040C051D05E9F488AD99ADF2
:105E4000892BB1F0672BA1F4858599278370907019
:105E5000892B71F48FA98F5F8FAB833048F01FAA15
:105E6000CE010E942C31892B19F08FEF9FEF7FC05C
:105E7000EA96CE0178C01FAAEDA2FEA20FA318A732
:105E800086859785082E892F902D8DAB9EAB34E5A6
:105E9000C32ED12CCC0EDD1EF60180819181A28112
:105EA000B3810097A105B10541F08E159F05A007AC
:105EB000B10718F4CE010E946E37F60110821182EC
:105EC0001282138268AD79AD61157105A1F1FB01F4
:105ED000C384D484F6012481358146815781022E02
:105EE000252F502D032E342F402DFB0181899289BF
:105EF000AA27BB27280F391F4A1F5B1FF60185857C
:105F0000992783709070892B21F02F5F3F4F4F4F5F
:105F10005F4FE216F3060407150768F0FB01808166
:105F2000918188AF99AFCB010E94B85F68AD79AD20
:105F30006115710561F688AD99AD2AE3E22EF12C69
:105F4000EC0EFD1E8E01025A1F4FC65ADF4F0097FE
:105F500021F00E944657DC01CB01F8018083918338
:105F600018821982C7010E94FD5780E090E0DF91FE
:105F7000CF911F910F91FF90EF90DF90CF90BF9046
:105F8000AF900895EF92FF920F931F93CF93DF93FB
:105F9000EC01F62E00E010E0EE248B899927853085
:105FA000910509F486C0863091059CF482309105F4
:105FB000A9F18330910534F4009709F484C0019766
:105FC00041F190C08330910509F43EC00497C1F0BF
:105FD00089C08830910509F483C08930910544F463
:105FE0008630910509F450C0079709F468C07AC05B
:105FF0008930910509F457C00A9709F471C072C03D
:10600000862F992785309105E1F0069709F068C041
:1060100053C083E0681709F063C00BC0862F99272F
:106020008330910531F084309105B4F0049721F06C
:1060300057C088A1826150C0CE018C599F4F0E94E9
:10604000FD5788A1886148C0862F99278430910523
:1060500069F08530910524F4019709F443C040C0EC
:106060008530910549F1069761F03AC0CE018E590D
:106070009F4F0E94FD57CE018C599F4F0E94FD57A4
:1060800031C088A1816028C0862F9927873091056B
:10609000C1F2883091051CF4069721F121C00997BF
:1060A0000297F0F41FC08AE0681759F20FEF1FEF54
:1060B000C8CF88E06817A1F488A181610DC08AE08B
:1060C000681781F00DC0862F99278130910551F016
:1060D000029731F488A1826088A341E0E42E02C0D7
:1060E0000FEF1FEF0115110581F5FB8AEE20C9F0B6
:1060F000A801B801CE010E94BB2B892B91F082E050
:10610000F81679F40FEF1FEFC05ADF4F80E597E2E2
:1061100088839983C056D040CE018C599F4F0E94EE
:10612000FD5785E0F81689F4C25BDF4FCE010E946F
:1061300054586497CE010E945458A896CE010E94EC
:1061400054582296CE010E945458C801DF91CF9135
:106150001F910F91FF90EF900895CF93DF93EC0183
:106160008B89882339F0C05ADF4F88E497E288830F
:1061700099830FC061E0CE010E94C22FCE59DF4F3C
:1061800040E050E060E070E0CE010E94785780E08F
:1061900090E0DF91CF9108950F931F938C0162E0FF
:1061A0000E94C22FC8018C599F4F40E050E060E030
:1061B00070E00E947857F8018389843019F08FEFDE
:1061C0009FEF02C080E090E01F910F910895CF9360
:1061D000DF93EC01892B31F10E948E538B89992733
:1061E000853091051CF403975CF406C08530910559
:1061F00049F00B978CF40BC0CE010E945D2215C0B4
:1062000066E001C068E0CE010E94C22F0EC0C05AF5
:10621000DF4F85E397E204C0C05ADF4F89E497E27D
:10622000888399838FEF9FEF02C080E090E0DF9139
:10623000CF910895FC01892B19F48FEF9FEF0895FA
:1062400080A1886180A340E050E0BA01CF010E94A4
:10625000BB2B80E090E00895EF92FF920F931F9385
:10626000CF93DF93EC01FC01E65AFF4F80819181CF
:106270009C010196808391832830310518F06CE4ED
:1062800077E213C0E8ADF9ADE080F1809F014A8D5F
:106290005B8D6C8D7D8D86E00E9430388C01892B62
:1062A00051F0E8AEF9AE62E477E2CE010E94193710
:1062B0008FEF9FEF09C0C25ADF4F0E944657DC01A3
:1062C000CB0188839983C801DF91CF911F910F91F2
:1062D000FF90EF9008950F931F93CF93DF938C015E
:1062E000862FE901992786719070029769F46F8172
:1062F0007885C8010E944D2E63E0C8010E94C22F1C
:10630000CE010E94B85F03C0C9010E943F2DDF91FA
:10631000CF911F910F9108958F929F92AF92BF924C
:10632000CF92DF92EF92FF920F931F93CF93DF9361
:10633000EC015A014901C62EDD24C4FE21C0FA0138
:1063400080859185A285B385082E8B2FB02D092ECF
:106350009A2FA02D29A13AA14BA15CA12F5F3F4FFD
:106360004F4F5F4FE9A4FAA40BA51CA5BC01CD01BA
:106370000E944637892B21F4C4010E943F2D25C07D
:10638000C2FE08C0C4FE1EC06DE477E2CE010E94CA
:10639000193718C0C1FE16C0A501F40167817085C8
:1063A000CE010E944D2EC4FE09C0F40141895289DC
:1063B000B501CE010E94B72E64E001C063E0CE01BA
:1063C0000E94C22FC4010E94B85FDF91CF911F913C
:1063D0000F91FF90EF90DF90CF90BF90AF909F9084
:1063E0008F9008958F929F92AF92BF92CF92DF923B
:1063F000EF92FF920F931F93CF93DF93EC014A012B
:106400006901A62EBB24A2FE1FC0CE59DF4F888192
:106410009981C256D040892B29F061E0CE010E94BB
:10642000C22F05C06DE477E2CE010E941937C60184
:106430000E94B85FC25ADF4F18821982CE55D040F1
:10644000CE010E941E2253C0A1FC23C0A4FC04C0A4
:10645000C9010E94B85F4BC0FA0180859185A28571
:10646000B385082E8B2FB02D092E9A2FA02D2DA18C
:106470003EA14FA158A52F5F3F4F4F4F5F4FE9A45B
:10648000FAA40BA51CA5BC01CD010E944637892B9F
:1064900021F4C6010E943F2D2AC0F601418952898C
:1064A000B401CE010E94B72EF60181899289892B11
:1064B00029F0B601CE010E94DD2D03C0C6010E9465
:1064C000B85FA0FE10C0FE01E05CFF4F80819181AB
:1064D000A281B3810196A11DB11D80839183A28306
:1064E000B38365E001C064E0CE010E94C22FDF915A
:1064F000CF911F910F91FF90EF90DF90CF90BF90C1
:10650000AF909F908F9008952F923F925F926F92DD
:106510007F928F929F92AF92BF92CF92DF92EF9233
:10652000FF920F931F93CF93DF93CDB7DEB72C97D6
:106530000FB6F894DEBF0FBECDBF7C01562E6A01A8
:106540008901862F992782FF09C0C9010E94B85F7F
:1065500066E477E2C7010E94193746C1F2E08F2E48
:10656000912C8822992281FF19C0FA01848195819A
:10657000A681B781082E8B2FB02D092E9A2FA02D22
:10658000F70124AD35AD46AD57AD82179307A4078B
:10659000B50731F0C8010E943F2D26C184FD0BC014
:1065A000C8010E94B85F20C1DB010D931C93F80164
:1065B0008082918268C0F90141895289B601C70180
:1065C0000E94B72EF6014481558166817781498703
:1065D0005A876B877C875A016B010A2CAD2CD02C13
:1065E0000B2CBC2CC02CE0E42E2E312C2E0C3F1C8E
:1065F000D1018D919D910D90BC91A02D8D839E8395
:10660000AF83B8878A159B05AC05BD0508F046C069
:10661000F80181899289892B09F4C1C0F701E05BF7
:10662000FF4F80809180BF018114910461F1F401DA
:10663000A385B48529853A854B855C85022E252F57
:10664000502D032E342F402D14968D919D910D9039
:10665000BC91A02D082E8B2FB02D092E9A2FA02D86
:10666000281739074A075B0708F49ECF2817390710
:106670004A075B0709F493C0B401D4018D909C9044
:1066800081149104A1F68114910409F08BC0FB01DF
:1066900000831183D8018D929C9284C0042E472FD1
:1066A000702D052E562F602DAD80BE80CF80D884F2
:1066B0004A155B056C057D05D1F0F70180A1886165
:1066C00080A3E259FF4F80819181A281B38101961D
:1066D000A11DB11D80839183A283B383C8010E9451
:1066E000B85FA401B401C7010E94BB2B69C0F801C7
:1066F00081899289892B09F460C0B801C7010E9481
:10670000DD2D50E5A52EB12CAE0CBF1CD5010D9191
:106710001C910115110509F453C0F801C384D484F8
:10672000F60184819581A681B7819C01AD01082E77
:106730008B2FB02D092E9A2FA02DF1016080718032
:10674000828093806D827E828F8298866816790619
:106750008A069B06A8F1D8018D919C91F501808352
:106760009183022E252F502D032E342F402D2615D8
:1067700037054805590541F4B801C7010E94DD2DD0
:10678000F6018585582A03C0C8010E94B85FD5016B
:106790000D911C910115110509F0BFCF11C0C80161
:1067A0000E94B85FF70180A1886180A340E050E0BB
:1067B000BA01C7010E94BB2B17C0C8010E94B85F75
:1067C00050FE12C0F701E05CFF4F80819181A281F1
:1067D000B3810196A11DB11D80839183A283B383F0
:1067E00065E0C7010E94C22F2C960FB6F894DEBF59
:1067F0000FBECDBFDF91CF911F910F91FF90EF9012
:10680000DF90CF90BF90AF909F908F907F906F90D0
:106810005F903F902F900895EF92FF920F931F93F8
:10682000CF93DF93EC01862FBA018901E82EFF2474
:10683000E2FE07C0C9010E94B85FCE010E945D223E
:106840004FC0E1FE04C0C9010E943F2D49C0E4FCD5
:1068500004C0C9010E94B85F43C0F901418952894F
:10686000CE010E94B72E29A53AA54BA55CA58DA106
:106870009EA1AFA1B8A5281739074A075B0721F4E5
:1068800069E0CE010E94C22FF80181899289892B8B
:1068900029F0B801CE010E94DD2D03C0C8010E947D
:1068A000B85FE0FE1DC0FE01E05CFF4F808191817A
:1068B000A281B3810196A11DB11D80839183A28322
:1068C000B383C45ADF4F18821982CC55D0408B89CC
:1068D000893011F46AE001C067E0CE010E94C22F46
:1068E000DF91CF911F910F91FF90EF900895EF925C
:1068F000FF920F931F93CF93DF938C01862FBA01E2
:10690000E901E82EFF24E2FE07C0C9010E94B85F3A
:10691000C8010E945D2238C0E1FE04C0C9010E9486
:106920003F2D32C0E4FC04C0C9010E94B85F2CC0F6
:1069300049895A89C8010E94B72E89899A89892B69
:1069400029F0BE01C8010E94DD2D03C0CE010E94C6
:10695000B85FE0FE19C0F801E05CFF4F80819181D3
:10696000A281B3810196A11DB11D80839183A28371
:10697000B383045A1F4FF801108211820C55104046
:106980006AE0C8010E94C22FDF91CF911F910F9141
:10699000FF90EF9008950F931F93CF93DF938C0197
:1069A000862FBA01E901992782FF09C0C9010E9417
:1069B000B85F66E477E2C8010E94193710C081FF12
:1069C00004C0C9010E943F2D0AC084FF05C0498947
:1069D0005A89C8010E94B72ECE010E94B85FDF918C
:1069E000CF911F910F910895EF92FF920F931F93F4
:1069F000CF93DF93EC01862FBA018901992782FF9B
:106A000007C0C9010E94B85FCE010E945D222DC05F
:106A1000A2E0EA2EF12CE822F92281FF04C0C9018C
:106A20000E943F2D22C084FF1DC0F9014189528977
:106A3000CE010E94B72E29A53AA54BA55CA58DA134
:106A40009EA1AFA1B8A5281739074A075B0751F4E3
:106A5000C45ADF4FE882F982CC55D0406AE0CE01BB
:106A60000E94C22FC8010E94B85FDF91CF911F9191
:106A70000F91FF90EF9008950F931F93CF93DF93A3
:106A80008C01862FBA01E901992782FF04C0C90150
:106A90000E94B85F22C081FF04C0C9010E943F2D3F
:106AA0001FC084FD04C0C9010E94B85F19C0498994
:106AB0005A89C8010E94B72ECE010E94B85FF80122
:106AC00021A532A543A554A585A196A1A7A1B0A54E
:106AD000281739074A075B0719F4C8010E945D228D
:106AE000DF91CF911F910F9108950F931F93CF9333
:106AF000DF938C01FB01A385B4851D966C911D97D6
:106B0000EC018B8999278530910509F448C08630BE
:106B1000910594F48230910551F18330910534F45C
:106B2000009709F44EC00197E1F04FC08330910502
:106B300021F1049781F049C088309105E1F1893055
:106B4000910534F486309105F1F0079771F13DC05D
:106B50000997F9F03AC09F01AD01C8010E94843243
:106B600037C09F01AD01C8010E946B3131C09F0148
:106B7000AD01C8010E948C312BC09F01AD01C8013D
:106B80000E94F23125C09F01AD01C8010E940C3462
:106B90001FC09F01AD01C8010E94773419C09F0139
:106BA000AD01C8010E94CB3413C09F01AD01C801E3
:106BB0000E94F4340DC09F01AD01C8010E943C3514
:106BC00007C0CF010E943F2D03C0CF010E94B85FD4
:106BD000DF91CF911F910F910895DD2480E20E94F3
:106BE000D253D39483E08D1558F048EC50E060E028
:106BF00070E08FE79BE00E947857009709F464C02B
:106C0000DD24C091120AD091130A209751F388A174
:106C100084FF08C0886088A340E050E0BA01CE013C
:106C20000E94BB2B88AD99AD892BF1F08E01025AE1
:106C30001F4FF80180819181892BB1F00E94465746
:106C4000DC01CB01F80120813181821B930B9C0177
:106C5000C85ADF4F88819981C855D0408217930761
:106C600018F4CE010E942C318B898A3019F08B895F
:106C7000893081F4FE01E45AFF4F808191819C01AB
:106C800001968083918329303105B8F0CE010E94AE
:106C90005D22A7CF8B89833081F4FE01E45AFF4F38
:106CA000808191819C010196808391832D323105F1
:106CB00020F081E08B8B108211820990D881C02D49
:106CC000209709F0A4CF8DCF00917D0B10917E0B02
:106CD00090937E0B80937D0B90932B0A80932A0ACE
:106CE0000115110509F47DCFE801EF81F885AB8529
:106CF000BC8524853585468557856D917C91119796
:106D000012968D919C9113970E949022EC01F801AC
:106D1000E080F180009741F0B8010E94DC2DB801BD
:106D2000CE010E94753503C0C8010E943F2D870126
:106D3000EF28D1F656CFCF92DF92EF92FF920F93CA
:106D40001F93CF93DF93EC01188219828091280A58
:106D50009091290A892B21F4CE010E943F2D45C034
:106D6000C0907D0BD0907E0BC114D10429F4D09338
:106D70007E0BC0937D0B31C0E984FA848D859E859E
:106D8000E80EF91E89899A89E80EF91E00912A0AEF
:106D900010912B0A0E0D1F1D0050184F0E943F52DC
:106DA00008171907F8F480912A0A90912B0A8E0D82
:106DB0009F1D90932B0A80932A0AF601808191816E
:106DC000892B41F0F601C080D180F601808191814C
:106DD000892BC1F7F601C083D1838FE79BE00E9426
:106DE000235803C0CE010E94B85FDF91CF911F915D
:106DF0000F91FF90EF90DF90CF9008954091280A77
:106E00005091290A4115510589F420E032E06DEED8
:106E100075E389E597E00E948F529093290A809349
:106E2000280A892B19F48FEF9FEF089580E090E0F6
:106E30000895CF93DF93EC01C05ADF4F68837983C5
:106E40001A921A921A921A92CC55D0408B89863097
:106E500018F08AE08B8B01C01B8ACE010E941E2293
:106E6000C25BDF4FCE010E9454586497CE010E944E
:106E70005458A896CE010E9454582296CE010E94E2
:106E8000545880E090E0DF91CF910895EF92FF9207
:106E90000F931F93E216F3060407150758F06217C5
:106EA00073078407950798F0E616F7060807190791
:106EB00070F00AC0261737074807590740F06E15CB
:106EC0007F058007910718F081E090E002C080E024
:106ED00090E01F910F91FF90EF9008950F931F93F3
:106EE000CF93DF938C01EC01C25ADF4F88819981E7
:106EF000892B41F10E944657DC01CB012881398161
:106F0000821B930B9C01F801E85AFF4F808191810D
:106F1000880F991F820F931F880F991F880F991F41
:106F20006AE070E00E9468738EE46032780730F4A3
:106F3000683C710528F468EC70E002C060E27EE411
:106F400060837183DF91CF911F910F910895CF934B
:106F5000DF939B01FA01AC0166277727E901E23054
:106F6000F10560F089919991AA27BB27480F591F15
:106F70006A1F7B1F3297E230F105A0F7EF2B29F053
:106F80008881480F511D611D711DCB01AA27BB27A8
:106F90000097A105B10591F0DB01CA01A070B070A6
:106FA000AB0166277727480F591F6A1F7B1FCB014C
:106FB000AA27BB270097A105B10571F7CA01DF9188
:106FC000CF9108950E94A737809590950895EF92EC
:106FD000FF920F93CF93DF93CDB7DEB72C970FB609
:106FE000F894DEBF0FBECDBFDC01CB0189839A834D
:106FF000AB83BC832D833E834F83588719860A87D2
:10700000EB86FC864CE050E0BE016F5F7F4F80E076
:1070100090E00E94A737AA27BB27BC01CD012C9680
:107020000FB6F894DEBF0FBECDBFDF91CF910F91A9
:10703000FF90EF900895AF92BF92CF92DF92EF92C0
:10704000FF920F930E94E737DC01CB01809590956A
:107050000F91FF90EF90DF90CF90BF90AF90089589
:107060006F927F928F929F92AF92BF92CF92DF9258
:10707000EF92FF920F931F93CF93DF93CDB7DEB7BD
:107080002A970FB6F894DEBF0FBECDBF182F3A0176
:107090004B0144E150E060E2C9010E944E5E6C0188
:1070A000009709F4F0C0FC01E780F08485E4F70163
:1070B00080831182F6018185928525853685820F30
:1070C000931F21893289820F931F082E892F902DBB
:1070D000F701828393831682178280E48087118769
:1070E000608A718A828A938AFFEF6F16FFEF7F06AC
:1070F000FFEF8F06FFEF9F0609F060C046E050E00B
:107100006FEF70E0CE0101960E94B072A090660A07
:10711000B090670A20E030E0A114B10409F44CC03B
:10712000F5018385833009F03DC007851089F8019A
:10713000858996899C010196858B968B022E232F3B
:10714000302DF70124833583F80187819085A1854F
:10715000B285F70184879587A687B787128613863D
:10716000F601418552856781708580E090E00E943C
:10717000E237F70182879387F8018081A58DB68D6C
:10718000863039F49601AE014F5F5F4F60E078E0E2
:1071900005C0960140E050E061E270E0C501FD01EC
:1071A00009959C01F501A080B180A114B10421F0E2
:1071B0002115310509F4B4CFC90167C0AE01495F9B
:1071C0005F4FC401B3010E94C1285C01009709F41C
:1071D00057C0FC0107851089F801858996899C01B3
:1071E0000196858B968B022E232F302DF701248359
:1071F0003583F80187819085A185B285F701848761
:107200009587A687B78712861386F6014185528532
:107210006781708580E090E00E94E237F701828705
:107220009387F80180818630E9F44F81588569851C
:107230007A85411551056105710511F4B401A30169
:107240009E012F5F3F4FC5010E94853A892BC1F4F3
:10725000F801A58DB68D9601AE014F5F5F4F60E0DE
:1072600078E00AC0873161F4F801A58DB68D9601EA
:1072700040E050E061E270E0C501FD01099505C004
:10728000C6010E94B85F8FEF9FEF2A960FB6F89461
:10729000DEBF0FBECDBFDF91CF911F910F91FF9049
:1072A000EF90DF90CF90BF90AF909F908F907F90A6
:1072B0006F900895CF93DF93CDB7DEB726970FB6C3
:1072C000F894DEBF0FBECDBF1B821C8260E67AEE53
:1072D00080E090E00E9484560091660A1091670A4F
:1072E0000115110599F3F8018385833009F044C035
:1072F000A785B08957968D919C91589789839A83D9
:107300005796AD83BE8389819A81892BA9F1E98142
:10731000FA81848582FD14C0E981FA818585982FE0
:107320008F5F8587993060F0AD81BE81E981FA81F8
:10733000808191818D939C9389819A818B839C8399
:107340008B819C81892B21F489819A818D839E83F5
:10735000E981FA818081918189839A838B819C81E3
:10736000892B31F08B819C810E94BF511B821C8232
:1073700089819A81892B59F6F801008111810115C3
:10738000110509F0B0CFA2CFCF93DF93CDB7DEB711
:1073900022970FB6F894DEBF0FBECDBFFC018789E0
:1073A000908D89839A8389819A81892BA9F0E981BB
:1073B000FA8182819381A481B58184179507A607FC
:1073C000B70751F0E981FA818081918189839A839D
:1073D00089819A81892B59F789819A8122960FB6E2
:1073E000F894DEBF0FBECDBFDF91CF9108958F928D
:1073F0009F92AF92BF92CF92DF92EF92FF920F9344
:10740000CF93DF934C016A017B01590180E190E049
:107410000E94AA51FC01892BE1F0C282D382E4824E
:10742000F582A114B10441F086E0EF012696D50162
:107430000D9009928A95E1F704870FB60F92F894A0
:10744000E4018F89988D80839183EF8BF88F0F9063
:107450000FBECF01DF91CF910F91FF90EF90DF90A2
:10746000CF90BF90AF909F908F900895AF92BF92B2
:10747000CF92DF92EF92FF920F93CF93DF93EC01C5
:107480006A017B01590140912C0A50912D0A411546
:10749000510561F420E831E06AE579E38FE597E092
:1074A0000E948F5290932D0A80932C0AB701A60157
:1074B0008F8598890E94C439FC01892BA1F08485AD
:1074C00082FD0CC0158686E0EF012696D5010D9051
:1074D00009928A95E1F78485826084873E96CF0180
:1074E0000E94545808C002E09501B701A6018F859B
:1074F00098890E94F739DF91CF910F91FF90EF901B
:10750000DF90CF90BF90AF9008954F925F926F92AF
:107510007F928F929F92AF92BF92CF92DF92EF9223
:10752000FF920F93CF93DF935C016A017B012901E6
:10753000882499248FEF682E782EF501878590890D
:107540000E94C439EC01892B69F08C8581FF16C03B
:1075500086E0D201FE01369601900D928A95E1F700
:1075600094013DC000E09401B701A601F5018785B3
:1075700090890E94F739EC01892B81F120E030E0FD
:10758000B701A60181E090E00E94003B4C01892BED
:1075900069F42FEF3FEF23C086E0D201FE0136965B
:1075A00001900D928A95E1F7390115C003E0B4010D
:1075B000C5010E94593B9C01892B69F48C8581FD92
:1075C000EBCF44EF51E060E070E0CE010E960E94F8
:1075D0007857015060F7C4010E94B85F9301C90158
:1075E000DF91CF910F91FF90EF90DF90CF90BF9000
:1075F000AF909F908F907F906F905F904F90089585
:107600008F929F92AF92BF92CF92DF92EF92FF92B2
:107610000F931F93CF93DF938C015A016B014901A4
:107620004CE150E060E280E090E00E944E5E7C0120
:10763000009709F431C0FC01C781D08581E090E05A
:10764000082E892F902D8883998380E098E0082E5A
:10765000892F902D8A839B8326E02C8384E08D8361
:10766000002E012F102D0E831F83CE014296811410
:10767000910439F0DC01F40101900D922A95E1F7B3
:1076800006C046E050E06FEF70E00E94B072A88E36
:10769000B98ECA8EDB8EC701DF91CF911F910F91FA
:1076A000FF90EF90DF90CF90BF90AF909F908F9022
:1076B00008950F931F93CF93DF938C019B01EB01F0
:1076C0004F815885EC01EF85F88986E0EA0128961C
:1076D000DF0111960D9009928A95E1F787819085D7
:1076E000A185B285EA018E879F87A88BB98B4E5EF4
:1076F0005F4F058CF68DE02D66E078E0C8010995B6
:10770000DF91CF911F910F910895EF92FF920F9308
:107710001F93CF93DF938C017B01EA01DC018D91F4
:107720009C91009711F00E945A6ECE0101960E9422
:10773000576EF80180839183209721F0AE01B70145
:107740000E949E72D801ED91FC91EC0FFD1F1082FA
:10775000DF91CF911F910F91FF90EF9008956F925D
:107760007F928F929F92AF92BF92CF92DF92EF92D1
:10777000FF920F931F93CF93DF935C01E901980170
:10778000EFEF6E2E7E2E89E2F50111928A95E9F7D0
:107790008881823029F0E4C02FEF622E722EE0C083
:1077A000F50145A356A367A370A788899989AA897B
:1077B000BB8981839283A383B4838E0100511F4FC1
:1077C00090E1892E9FEF992E820E931E18141904B2
:1077D0000CF0C6C0F80190819F3F09F4C1C0992305
:1077E00031F40F5F1F4F089481089108B5C0F8016C
:1077F0008181C82FDD278C169D0674F2C430D10517
:1078000021F4C280D380E480F580892F99278F30BE
:10781000910509F455C0803191058CF483309105B0
:1078200009F43DC0843091051CF4019721F187C013
:107830008630910509F44DC00C97D9F180C083338F
:10784000910509F468C0843391051CF44C97E9F064
:1078500076C08533910521F0C69709F453C06FC0F7
:10786000C130D10509F068C0F8018281F50180833B
:107870006624772464C0C430D10509F05DC0F501E9
:10788000C582D682E782F0865AC0C430D1050CF496
:1078900053C0F501C186D286E386F48650C0C43059
:1078A000D1050CF449C0F501C586D686E786F08A75
:1078B00046C0C8010296AE01BC01C501819606C052
:1078C000C8010296AE01BC01C50183960E94853BAA
:1078D00036C0C430D1052CF0F501C18AD28AE38AC2
:1078E000F48AC830D10554F0F80186819781A085CB
:1078F000B185F501858B968BA78BB08FC430D105F0
:10790000F4F41AC0C430D105BCF0F501C18ED28E9A
:10791000E38EF48E14C0C430D10571F4D701C601D2
:10792000082E8B2FB02D092E9A2FA02DF501858FB3
:10793000968FA78FB0A303C08FEF682E782E0C0F01
:107940001D1F0E5F1F4F8C1A9D0A8EEF9FEF880E32
:10795000991E6114710421F4181419040CF43ACF1F
:10796000C301DF91CF911F910F91FF90EF90DF90B6
:10797000CF90BF90AF909F908F907F906F90089521
:10798000BF92CF92DF92EF92FF920F931F93CF930C
:10799000DF93FC01B62EBA01A901960184E292E0C0
:1079A000DF011D920197E9F7A1E0DA2ED082D182A2
:1079B00086E08283DF015C96C7E6DBE009900D92EA
:1079C0008A95E1F74483558366837783022E232FBC
:1079D000302D20873187E486F58606871787E451A6
:1079E000FF4F8091650790916607A0916707B0915E
:1079F000680780839183A283B38385E38483D582E0
:107A0000B68287E090E0DF91CF911F910F91FF90B8
:107A1000EF90DF90CF90BF900895EF92FF920F9379
:107A20001F93DC01F801E20FF31FE451FF4F8FEFCA
:107A3000808303511F4F81E00C32180710F40CE2D1
:107A400011E07801890123E430E0CD010E94AE64A9
:107A500097FF09C068E873E180E090E00E948456D7
:107A60008FEF9FEF02C080E090E01F910F91FF9099
:107A7000EF9008952F923F924F925F926F927F9274
:107A80008F929F92AF92BF92CF92DF92EF92FF922E
:107A90000F931F93CF93DF93CDB7DEB722970FB627
:107AA000F894DEBF0FBECDBF1C014A015B01290166
:107AB0003801B8E8CB2EB3E1DB2EE12CF12C04E247
:107AC00012E09301AE014F5F5F4FB201C1010E940E
:107AD000EF648C01181619065CF4F301848195811A
:107AE000A681B78188159905AA05BB0511F708C0BD
:107AF00097FF06C068E873E180E090E00E9484563A
:107B0000C80122960FB6F894DEBF0FBECDBFDF913D
:107B1000CF911F910F91FF90EF90DF90CF90BF908A
:107B2000AF909F908F907F906F905F904F903F901D
:107B30002F9008956F927F928F929F92AF92BF92F3
:107B4000CF92DF92EF92FF920F931F93CF93DF9329
:107B5000CDB7DEB723970FB6F894DEBF0FBECDBF0B
:107B60003C014B01C8011CEEA12EB12CA60EB71E84
:107B70006C01EE24FF24870161E0C4010E94C03C37
:107B80007C0120916D0B30916E0B40916F0B5091E9
:107B9000700B8091710B9091720BA091730BB0914F
:107BA000740B82239323A423B5230097A105B10569
:107BB00079F0F501EE0DFF1D82E3819384E081935E
:107BC000208331834283538386E090E0E80EF91EE0
:107BD00081E0898393E09A8386E08B83F501EE0D43
:107BE000FF1D87E38193919343E050E0BE016F5FF7
:107BF0007F4FCF010E949E7285E090E0E80EF91E53
:107C00002CE83BE0D9010D900020E9F71197A21B69
:107C1000B30B1A161B068CF4F501EE0DFF1D8CE05C
:107C20008193A1930A2F1127A801B901CF010E94C6
:107C30009E720E5F1F4FE00EF11EF501EE0DFF1D4F
:107C400080E492E0082E892F902D29E3219322E0F1
:107C500021938083918384E090E0E80EF91E8701F0
:107C600094014FEF5FEF6FEF7FEFC3010E940D3D77
:107C700023960FB6F894DEBF0FBECDBFDF91CF9134
:107C80001F910F91FF90EF90DF90CF90BF90AF903A
:107C90009F908F907F906F9008952F923F924F9278
:107CA0005F926F927F928F929F92AF92BF92CF928C
:107CB000DF92EF92FF920F931F93CF93DF93CDB795
:107CC000DEB72B970FB6F894DEBF0FBECDBF8C8307
:107CD0009D834E835F83688779872A873B87370137
:107CE0004801A601950128A039A04AA05BA088A55B
:107CF00099A5AA84BB846CEE70E0A60EB71E6C0139
:107D000079018A01A401930163E08A859B850E9421
:107D1000C03C7C01211431044104510479F0F50187
:107D2000E80FF91F82E3819384E0819320823182FE
:107D30004282538286E090E0E80EF91E6CA17DA19C
:107D40008EA19FA1611571058105910599F0F5013D
:107D5000EE0DFF1D86E3819384E081938CA19DA1AC
:107D6000AEA1BFA180839183A283B383A6E0B0E0DC
:107D7000EA0EFB1E81E0898393E09A8386E08B8381
:107D8000F501EE0DFF1D87E38193919343E050E0F1
:107D9000BE016F5F7F4FCF010E949E7265E070E071
:107DA000E60EF71E2CE83BE0D9010D900020E9F724
:107DB0001197A21BB30B1A161B068CF4F501EE0DDE
:107DC000FF1D8CE08193A1930A2F1127A801B9010F
:107DD000CF010E949E720E5F1F4FE00EF11E8701C1
:107DE0002A853B854E815F81688579858C819D815F
:107DF0000E940D3D2B960FB6F894DEBF0FBECDBF8F
:107E0000DF91CF911F910F91FF90EF90DF90CF9076
:107E1000BF90AF909F908F907F906F905F904F90AA
:107E20003F902F9008952F923F924F925F926F92C2
:107E30007F928F929F92AF92BF92CF92DF92EF92FA
:107E4000FF920F931F93CF93DF93CDB7DEB72497A5
:107E50000FB6F894DEBF0FBECDBF1C0149835A8315
:107E60006B837C833901A8019701D601C501898CF8
:107E70009A8CAB8CBC8C0CEE402E512C460C571CB3
:107E8000CC24DD247C018D0167E0C3010E94C03C4D
:107E90008C0181149104A104B10469F0F201E80F8E
:107EA000F91F86E3819384E0819380829182A2828C
:107EB000B3820A5F1F4FF201E00FF11F80E492E0EE
:107EC000082E892F902D29E3219322E0219380838E
:107ED00091830C5F1F4F930149815A816B817C8193
:107EE000C1010E940D3D24960FB6F894DEBF0FBE6F
:107EF000CDBFDF91CF911F910F91FF90EF90DF9059
:107F0000CF90BF90AF909F908F907F906F905F9039
:107F10004F903F902F900895CF93DF93EC01892BE2
:107F200079F089A19AA1009711F00E945A6E8BA155
:107F30009CA1009711F00E945A6ECE010E945A6EC9
:107F4000DF91CF9108954F925F926F927F928F92BF
:107F50009F92AF92BF92DF92EF92FF920F931F9387
:107F6000CF93DF933C01D62E49015A01280184E0CA
:107F70008617B8F120E02617A8F4E22FFF27EE0FAE
:107F8000FF1FE60DF71D0190F081E02D85A196A160
:107F9000A7A1B0A588159905AA05BB0511F12F5F0A
:107FA0002D1558F3CD2DDD27CC0FDD1FC60DD71DA8
:107FB00089E290E00E94576E88839983870192013D
:107FC000B501A4010E94AF3B892B29F4E881F98116
:107FD0008081823029F0888199810E948C3F01C084
:107FE000D3948D2D9927DF91CF911F910F91FF9001
:107FF000EF90DF90BF90AF909F908F907F906F90A9
:108000005F904F900895EF92FF920F931F93CF933D
:10801000DF93EC01EE24FF2410E020916D0B3091F2
:108020006E0B40916F0B5091700B8091710B909182
:10803000720BA091730BB091740B82239323A42332
:10804000B5230097A105B105B9F0162F1150A1F085
:10805000E12FFF27EE0FFF1FEC0FFD1F0190F081B6
:10806000E02D81819281A381B48182179307A407B7
:10807000B50711F0115061F761506F3FC1F0062F45
:108080000150E62FFF27611739F4EE0FFF1FEC0FA9
:10809000FD1FE080F18008C0EE0FFF1FEC0FFD1FF9
:1080A000808191810E948C3F602F0F3F41F7C70173
:1080B000DF91CF911F910F91FF90EF900895CF9393
:1080C000DF93CDB7DEB76E970FB6F894DEBF0FBE65
:1080D000CDBF898B9A8B1B8A1C8AFC010784F0898F
:1080E000E02DEF8BF88F198E1A8E1B8E1C8E442478
:1080F0004D8E4E8E80E492E08B879C8706C060E1B7
:1081000077E280E090E00E94845684E490E00E9450
:1081100062641C01009799F322E030E0AE01455FF4
:108120005F4F62E070E10E94A06584E292E00E94ED
:10813000576E8D8B9E8B80916D0B90916E0BA091E5
:108140006F0BB091700B2091710B3091720B4091BD
:10815000730B5091740B82239323A423B5230097B0
:10816000A105B10521F082E08093300A02C010928F
:10817000300AEF89F88D63807480858096800E9434
:108180002657DC01CB01680E791E8A1E9B1E50907B
:10819000300AF3E05F1609F07DC02114310429F0A4
:1081A000C1010E94586522243324EB89FC89458D46
:1081B000568D678D70A1411551056105710509F452
:1081C00047C0DB01CA0122E0B695A7959795879530
:1081D0002A95D1F77A018B01E81AF90A0A0B1B0BD1
:1081E0000E943657298D3A8D4B8D5C8D621B730B27
:1081F000840B950B6E157F058007910708F5E61A2D
:10820000F70A080B190B31E8E31634E8F3063EE1F0
:10821000030730E0130738F080E8E82E84E8F82EF2
:108220008EE1082F112DC801B70128EE33E040E0A0
:1082300050E00E943D73DC01CB01AC01BD0108C0E0
:108240008091300A833041F484E08093300A04C086
:1082500083E39AE00E9478578091300A833009F4D2
:1082600096CF06C068EE73E080E090E00E948456EE
:1082700084E490E00E9462641C01009799F322E07C
:1082800030E0AE01455F5F4F62E070E10E94A065A3
:108290001D8E75CF44E0541609F069C08D8D582F9E
:1082A0005F5F5D8F833008F057C0898D9A8D9F93F3
:1082B0008F931F921F921F921F9280916D0B90912E
:1082C0006E0BA0916F0BB091700BBF93AF939F9308
:1082D0008F935C016D01840173012D893E89EB89C7
:1082E000FC8945A156A167A170A5C1010E944D3E20
:1082F0002DB73EB7265F3F4F0FB6F8943EBF0FBE77
:108300002DBF99230CF4C3C10D891E899E01235FE3
:108310003F4FB401A301C1010E943A3D99230CF4DF
:10832000B6C1181619060CF032CF8C012D893E8982
:108330004D855E856F8578898B899C890E94AF3BCE
:10834000892B09F024CFEB89FC898081853009F4E1
:1083500069C0863009F01BCF1D8E0E942657DC01B4
:10836000CB01680E791E8A1E9B1E85E0B1C1F5E027
:108370005F1609F068C08D8D282F2F5F2D8F8330F9
:1083800008F0D8C1498D5A8D5F934F931F921F9269
:108390001F921F9280916D0B90916E0BA0916F0BAD
:1083A000B091700BBF93AF939F938F935C016D015E
:1083B000840173012D893E894FEF5FEF6FEF7FEFEF
:1083C000C1010E944D3EEDB7FEB73A960FB6F89444
:1083D000FEBF0FBEEDBF99230CF459C10D891E8954
:1083E0009E01235F3F4FB401A301C1010E943A3DAA
:1083F00099230CF44CC1181619060CF0C8CE8C0148
:108400002D893E894D855E856F8578898B899C890C
:108410000E94AF3B892B09F0BACEEB89FC898081A1
:10842000853039F40E943657698F7A8F8B8F9C8FF5
:108430004EC1863009F0ABCE0E943657698F7A8FD5
:108440008B8F9C8F77C1FE8DFF2379F4EF89F88D98
:1084500087819085A185B2850097A105B10529F096
:1084600060E177E280E090E0D0C1552009F04BC098
:108470008B899C890E948C3F1B8A1C8A098D1A8DCE
:10848000A40193016D897E89C1010E949A3D9923BF
:108490000CF4FDC00D891E899E01235F3F4FB4017E
:1084A000A301C1010E943A3D7C0199230CF4EFC065
:1084B00018161906D4F40D891E892D853E854F8521
:1084C0005889642DCE0101960E94A33F482E8091C9
:1084D000350A9091360AA091370AB091380A885926
:1084E0009A43A040B040B0F603C0442009F44FCEF8
:1084F000642DCE0101960E9403408B8B9C8B4424FB
:108500004D8E81E0E5C021E0521609F07CC08D8DD2
:10851000382F320F3D8F833008F00CC1498D5A8DB2
:108520005F934F93EB89FC89818D928DA38DB48DE0
:10853000BF93AF939F938F9381819281A381B481E5
:10854000BF93AF939F938F93AA24BB2465018401AB
:1085500073012D893E894FEF5FEF6FEF7FEFC10110
:108560000E944D3E2DB73EB7265F3F4F0FB6F894A1
:108570003EBF0FBE2DBF99230CF489C00D891E8903
:108580009E01235F3F4FB401A301C1010E943A3D08
:108590007C0199230CF47BC0181619060CF0F7CD5A
:1085A00089E290E00E94576E8B8B9C8B87012D890E
:1085B0003E894D855E856F8578890E94AF3B892B0A
:1085C00009F0E5CDEB89FC898081853009F0AFC0E9
:1085D000FE8DFF2309F07BC0EB89FC89C584D6841E
:1085E000E784F08805811681278130854181528199
:1085F0006381748189899A890E94AE29009709F064
:10860000C6CD5E8E7FC0F2E05F1609F09EC08D8DF4
:10861000282F2F5F2D8FF81708F48CC0498D5A8DA5
:108620005F934F931F921F921F921F9280916D0B29
:1086300090916E0BA0916F0BB091700BBF93AF93A5
:108640009F938F93AA24BB246501840173012D8914
:108650003E894FEF5FEF6FEF7FEFC1010E944D3E0C
:10866000EDB7FEB73A960FB6F894FEBF0FBEEDBF5A
:1086700099236CF00D891E899E01235F3F4FB40141
:10868000A301C1010E943A3D7C0197FF02C086E030
:108690001FC0181619060CF07ACD89E290E00E94EE
:1086A000576E8B8B9C8B87012D893E894D855E850E
:1086B0006F8578890E94AF3B892B09F068CDEB89E3
:1086C000FC898081853099F5FE8DFF2321F083E0C0
:1086D0008093300A5CCDEB89FC89C584D684E7841D
:1086E000F08805811681278130854181528163811F
:1086F000748189899A890E94AE29009709F047CD33
:10870000F1E0FE8FEB89FC89E588F6880789108DFA
:108710002189328943895489BC010E94AD4783E095
:108720008093300A81E39AE00E94545830CD86301D
:1087300009F02DCD0E942657DC01CB01680E791E71
:108740008A1E9B1E1092300A22CDF7E05F16C9F5F3
:10875000EB89FC89818D928DA38DB48DBF93AF93EE
:108760009F938F93A0906D0BB0906E0BC0906F0B8A
:10877000D090700B840173012D893E8945A156A1CB
:1087800067A170A5C1010E94133F0D891E899E013A
:10879000235F3F4FB401A301C1010E943A3D81E331
:1087A0009AE00E945458EB89FC89158E168E178E1C
:1087B00010A283E08093300A0F900F900F900F90DB
:1087C000E6CCF6E05F1609F0E2CC2114310429F082
:1087D000C1010E94586522243324442061F0E42D15
:1087E000FF27EE0FFF1FEC0FFD1F818192810E947A
:1087F0008C3F4A94A1F78B899C890E948C3F1B8AED
:108800001C8A68EE73E080E090E00E948456BFCC42
:108810008F929F92AF92BF92CF92DF92EF92FF9290
:108820000F931F93CF93DF934C017B0159016A0192
:108830000E947558EC01892B09F47CC08B8583302C
:1088400009F078C00F851889F8018081863009F019
:1088500071C0E114F10441F0A7E6BBE0F70101901B
:108860000D928A95E1F706C0C4010E94652B892B01
:1088700009F060C086E0F8013196A7E6BBE00D90F4
:1088800001928A95E1F764EF71E080E090E00E9448
:1088900084562091790B30917A0B40917B0B50914B
:1088A0007C0B8091710B9091720BA091730BB09126
:1088B000740B82239323A423B5230097A105B1054C
:1088C000E1F5A092350AB092360AC092370AD092EA
:1088D000380A80912E0A90912F0A892B69F420E0A2
:1088E00032E0AE016FE570E489E697E00E948F52B6
:1088F00090932F0A80932E0AB601A50181E39AE096
:108900000E94785780916D0B90916E0BA0916F0B28
:10891000B091700B2091710B3091720B4091730BE1
:108920005091740B82239323A423B5230097A105B0
:10893000B10559F48FEF9FEF25C020936D0B309355
:108940006E0B40936F0B5093700BA090750BB09013
:10895000760BC090770BD090780BE090710BF09075
:10896000720B0091730B1091740B20916D0B309171
:108970006E0B40916F0B5091700B67E67BE0C4016A
:108980000E94BD2ADF91CF911F910F91FF90EF9030
:10899000DF90CF90BF90AF909F908F900895EF920F
:1089A000FF920F931F937A018B01892B21F0809105
:1089B000300A833019F08FEF9FEF0DC087E080936E
:1089C000300A83E39AE00E942358B801A70181E3AB
:1089D0009AE00E9478571F910F91FF90EF900895B1
:1089E000FC01872F99278193608382E090E00895AE
:1089F0000F931F93CF93DF93DC01EB01FB010190F9
:108A00000020E9F79F0121503040261B370B2E5FD5
:108A10003F4FFC01AC011196108288818823C1F080
:108A20008991BD016F5F7F4F8E018E3239F4CD0188
:108A3000AD01DB01EC011882E80106C08C93DB017B
:108A4000FA0180818F5F8083F8018081882341F75C
:108A50001C92C901DF91CF911F910F910895FC01E4
:108A6000DB0181919927382F22272D933C93119771
:108A700080819927282B392B2D933C9382E090E01D
:108A80000895FC0181919927AA27BB272227382F17
:108A9000492F5A2FDB012D933D934D935C931397F0
:108AA00081919927AA27BB27282B392B4A2B5B2B8F
:108AB000542F432F322F2227DB012D933D934D93CB
:108AC0005C93139781919927AA27BB27282B392BD1
:108AD0004A2B5B2B542F432F322F2227DB012D9360
:108AE0003D934D935C93139780819927AA27BB27C9
:108AF000282B392B4A2B5B2BFB01208331834283AC
:108B0000538384E090E00895EF92FF920F931F93B8
:108B1000CF93DF93EC018B01FB0180819181009762
:108B200029F00E94BF51F801108211828881992793
:108B3000807C9070803C910519F482E090E021C027
:108B4000FE0101900020E9F77F01EC1AFD0AC70140
:108B50000E943351F80180839183FC0199919923FC
:108B600071F091509F3F21F0899181939150E0F7EE
:108B70009991992311F08EE28193992391F71082B4
:108B8000C701DF91CF911F910F91FF90EF90089552
:108B9000EF92FF920F931F93CF93DF937C018B0192
:108BA000EA01FB0180819181009711F00E94BF5181
:108BB000CE010E943351F80180839183AE01B70149
:108BC0000E949E72CE01DF91CF911F910F91FF9075
:108BD000EF900895CF93DF93FC01EB01892B29F4EB
:108BE0008CE090E00E94AA51FC01309751F0C083C4
:108BF000D18380E091E08283938381E090E084835D
:108C00009583CF01DF91CF910895009711F00E94D5
:108C1000BF510895CF92DF92EF92FF920F931F936F
:108C20007C016B01FB01608171810E94F0448C0129
:108C3000C701800F911FF601628173810E94F04489
:108C4000080F191FC701800F911FF60164817581FC
:108C50000E94F044080F191FC701800F911FF601F1
:108C6000668177810E94F044080F191FC701800FA9
:108C7000911FF601608571850E94F044080F191F4D
:108C8000E00EF11EF60162857385C7010E94F04473
:108C9000080F191FC8011F910F91FF90EF90DF90EF
:108CA000CF900895CF92DF92EF92FF920F931F9390
:108CB0007C016B01BC01C6010E942F458C0182E042
:108CC00090E0E80EF91EC601800F911FB7010E94C7
:108CD0002F45080F191F82E090E0E80EF91EC6012B
:108CE000800F911FB7010E942F45080F191F82E0C6
:108CF00090E0E80EF91EC601800F911FB7010E9497
:108D00002F45080F191F82E090E0E80EF91EC601FA
:108D1000800F911FB7010E942F45080F191F82E095
:108D200090E0E80EF91EC00ED11EB701C6010E94E8
:108D30002F45080F191FC8011F910F91FF90EF9049
:108D4000DF90CF900895EF92FF920F931F93CF93F0
:108D5000DF93EC018B017A01892B29F486E090E006
:108D60000E94AA51EC012097D1F088819981009747
:108D700011F00E94BF51F80101900020E9F7E01BBB
:108D8000F10BCF010E94335188839983B8010E946F
:108D9000F572EA82FB8281E090E08C839D83CE01B4
:108DA000DF91CF911F910F91FF90EF900895CF9396
:108DB000DF93EC01892B49F088819981009711F0AC
:108DC0000E94BF51CE010E94BF51DF91CF91089503
:108DD000CF92DF92EF92FF920F931F937C016B0172
:108DE000FB01608171810E94F8448C01C701800FF2
:108DF000911FF601628173810E94F044080F191FD0
:108E0000E00EF11EF60164817581C7010E94F044F5
:108E1000080F191FC8011F910F91FF90EF90DF906D
:108E2000CF900895CF92DF92EF92FF920F931F930E
:108E30007C016B01BC01C6010E9484458C0182E06B
:108E400090E0E80EF91EC601800F911FB7010E9445
:108E50002F45080F191F82E090E0E80EF91EC00EA2
:108E6000D11EB701C6010E942F45080F191FC80166
:108E70001F910F91FF90EF90DF90CF900895009792
:108E800021F48EE090E00E94AA510895CF93DF93E1
:108E9000EC01892B79F088819981009711F00E946B
:108EA000BF518C859D85009711F00E94BF51CE0166
:108EB0000E94BF51DF91CF910895CF92DF92EF9240
:108EC000FF920F931F937C016B01BC01C6010E94AE
:108ED00084458C01C70102969601200F311FBC0109
:108EE000C9010E942F45080F191FC701049696015A
:108EF000200F311FBC01C9010E942F45080F191F07
:108F0000C70106969601200F311FBC01C9010E94BE
:108F10004145080F191FC7010A969601200F311FFE
:108F2000BC01C9010E942F45080F191FC00ED11E98
:108F3000F701428553858CE090E0E80EF91EB701F9
:108F4000C6010E94C845080F191FC8011F910F9143
:108F5000FF90EF90DF90CF9008958F929F92AF9205
:108F6000BF92CF92DF92EF92FF920F931F93CF9316
:108F7000DF93EC016B0149015A018091390A90910C
:108F80003A0A009731F00E94BF5110923A0A1092AB
:108F9000390A80913B0A90913C0A009731F00E9477
:108FA000BF5110923C0A10923B0A209781F0FE01BB
:108FB00001900020E9F7EC1BFD0BCF010E9433511B
:108FC00090933A0A8093390ABE010E94F572C11447
:108FD000D10481F0F60101900020E9F7EC19FD09B8
:108FE000CF010E94335190933C0A80933B0AB60113
:108FF0000E94F57280923D0A90923E0AA0923F0A2A
:10900000B092400AE092410AF092420A0093430A69
:109010001093440ADF91CF911F910F91FF90EF9031
:10902000DF90CF90BF90AF909F908F900895EF9278
:10903000FF920F931F93EE24FF2487010E94AD47F8
:109040001F910F91FF90EF90089561E070E00E94F2
:109050003748DC01CB01BC01CD0108956FE070E021
:109060000E943748DC01CB01BC01CD0108952F924D
:109070003F924F925F926F927F928F929F92AF92A8
:10908000BF92CF92DF92EF92FF920F931F93CF93F5
:10909000DF93CDB7DEB764970FB6F894DEBF0FBE8F
:1090A000CDBF8F83988769877A871B861C861D862C
:1090B0001E86662477246F86788A2301698A7A8AD5
:1090C00080913D0A90913E0AA0913F0AB091400ADA
:1090D0000097A105B10561F48091410A9091420A7F
:1090E000A091430AB091440A0097A105B10539F057
:1090F00080E090E00E9462641C01892B99F460E09A
:1091000070E080E090E0DDC0F20124853585D90172
:109110008D919D910D90BC91A02D8B879C87AD87E3
:10912000BE87BBC080E092E00E9433514C011B8A95
:109130001C8AEF85F8893196EF87F88BBF01C30150
:109140000E94EA453C0149855A856F817885898965
:109150009A890E94A346898B9A8BB301C4010E940D
:109160000A465C01C4018A0D9B1D69897A890E94A7
:10917000E846A80EB91EFB89F0FF0DC04091410AD8
:109180005091420A6091430A7091440A4115510579
:109190006105710569F47501840125E330E04091B2
:1091A0003D0A50913E0A60913F0A7091400A04C006
:1091B0007501840125E330E0C1010E94AE6499236A
:1091C0000CF46BC0AA24BB2438EEC32E33E0D32E9C
:1091D000E12CF12C00E012E09401AE014F5F5F4FF3
:1091E000BE016D5F7F4FC1010E94EF641816190622
:1091F0007CF40D973CF3B401C3010E9452465C011C
:10920000D3018D919C91EF85F8898E179F07D1F638
:10921000A114B104C1F1F3010481158101301105DC
:1092200091F5C4018A0D9B1DBC0189899A890E9410
:109230001247A80EB91EF30186819781009769F144
:1092400080179107D0F0C2010E943F472C01C40152
:109250008A0D9B1DBC01C2010E945D47A80EB91E6C
:10926000F20182819381019741F00F5F1F4FF3015B
:10927000868197818017910730F7F2018285938567
:10928000049709F441CF2B893C892F5F3F4F2B8BEB
:109290003C8B263031050CF44CCFC3010E940546AF
:1092A00089899A890E94D746C2010E944647C40113
:1092B0000E94BF51C1010E9458656B857C858D85D8
:1092C0009E8564960FB6F894DEBF0FBECDBFDF91CA
:1092D000CF911F910F91FF90EF90DF90CF90BF90B3
:1092E000AF909F908F907F906F905F904F903F9046
:1092F0002F9008950F931F93CF93DF93EC018B0171
:1093000086E090E00E943351FC01892B19F48FEF25
:109310009FEF10C08091450A9091460A8083918307
:10932000C283D38304831583F093460AE093450AEE
:1093300080E090E0DF91CF911F910F910895EF921F
:10934000FF920F931F93CF93DF937C018B01FB015F
:10935000808191810197029718F045EF51E025C077
:10936000C091450AD091460A209781F0F801868184
:1093700097810896BC018A819B810E94B772892BD4
:1093800029F00990D881C02D209781F7209719F4F2
:1093900044E951E009C0EC81FD81B801C70109959C
:1093A000892B31F044EF51E0B801C7010E945D4ABA
:1093B000DF91CF911F910F91FF90EF900895AF92A1
:1093C000BF92CF92DF92EF92FF920F931F935C01B7
:1093D0006B017A0189010E9410599F938F931F930B
:1093E0000F93FF92EF92F60122813381EAE0F0E0E1
:1093F000C901BF010E947C739F938F93C901BF0174
:109400000E947C737F936F9380EC99E19F938F937D
:10941000BF92AF920E945E6D8DB79EB70E960FB64B
:10942000F8949EBF0FBE8DBF1F910F91FF90EF90DC
:10943000DF90CF90BF90AF900895EF92FF920F937F
:109440001F93CF93DF93EC0179018A0161157105B8
:1094500091F07F936F9388EE99E19F938F93DF93C1
:10946000CF930E945E6D8DB79EB706960FB6F894A7
:109470009EBF0FBE8DBF17FD14C01F930F93FF92A9
:10948000EF928BEF99E19F938F93DF93CF930E949D
:109490005E6D8DB79EB708960FB6F8949EBF0FBE4F
:1094A0008DBFBE0181E19AE10E94816DDF91CF9174
:1094B0001F910F91FF90EF900895AF92BF92CF92BE
:1094C000DF92EF92FF920F931F93CF93DF935C0194
:1094D000EB017A0181E044395807F1F091E0453918
:1094E000590744F4E1E040395E0761F041595140C9
:1094F00071F021C081E0443F580799F0455F514029
:10950000A9F019C051E0C52E58E0D52E18C04DE085
:10951000C42E48E0D42E13C03AE1C32E38E0D32E37
:109520000EC024E2C22E28E0D22E09C093E3C92E39
:1095300098E0D92E04C083E4C82E88E0D82E960186
:10954000A701BE01C5010E94DF49E1E9EE16E1E095
:10955000FE0641F50E80DF81C02D6FE270E0CE0186
:109560000E9431738C01009719F0FC01108202C037
:10957000C9E4D8E0DF93CF9388E69AE19F938F9375
:10958000BF92AF920E945E6D8DB79EB706960FB6E2
:10959000F8949EBF0FBE8DBF0115110519F08FE223
:1095A000F80180832FEF3FEF4FEF5FEF65E877E043
:1095B000C5010E941D4ADF92CF92FF92EF92DF9287
:1095C000CF92FF92EF9287E29AE19F938F93BF929F
:1095D000AF920E945E6D8DB79EB70C960FB6F89451
:1095E0009EBF0FBE8DBFDF91CF911F910F91FF9056
:1095F000EF90DF90CF90BF90AF900895CF92DF9221
:10960000EF92FF920F931F93CF93DF938C010097FC
:1096100041F0EC0109900020E9F72197C81BD90B14
:1096200049F48091EB079091EC072CC0F7018281FF
:10963000938128C075EEE72E77E0F72E68E1C62EFD
:10964000D12CCE0CDF1CF701A081B181FD0101906E
:109650000020E9F73197EA1BFB0BCE018E1B9F0B15
:10966000800F911FBD010E94B772892BF9F284E02F
:1096700090E0E80EF91ECE14DF0428F78091E7078A
:109680009091E807DF91CF911F910F91FF90EF909C
:10969000DF90CF9008956F927F928F929F92AF92BA
:1096A000BF92CF92DF92EF92FF920F931F93CF93CF
:1096B000DF933C016B01CB010E942F4F892B19F0E6
:1096C00041E951E0D4C048E050E06BE478E0E601C5
:1096D0008E819F810E940C73892B29F4B601C301EE
:1096E0000E949F491CC18091470A9091480A0E80B0
:1096F000DF81C02D0097E1F0DC010D900020E9F73B
:109700001197A81BB90BFE0101900020E9F73197D2
:10971000EC1BFD0BAE0FBF1F1196CD010E94335104
:10972000EC016091470A7091480A0E94F57214C0DA
:10973000FE0101900020E9F73197EC1BFD0B3696F6
:10974000CF010E943351EC0186E0FE01A4E5B8E0B0
:109750000D9001928A95E1F7F60166817781CE013D
:109760000E94C97260E070E8CE010E94926A5C01BA
:10977000CE010E94BF51FFEFAF16FFEFBF0609F009
:109780007BC0E601EE81FF81EF0109900020E9F73F
:109790002197CE1BDF0BCE010C960E94AA518C01A3
:1097A000009719F444EF51E062C0209729F0F601C8
:1097B000668177810E94F572209759F0C00FD11F02
:1097C000219788818F3229F06AE578E0C8010E94EC
:1097D000C9726CE578E0C8010E94C972C091470A5D
:1097E000D091480AD8010D900020E9F72097C1F0E8
:1097F000FE0101900020E9F73197EC1BFD0B11975A
:10980000A01BB10BEA0FFB1F3196CF010E94335111
:10981000EC016091470A7091480A0E94F57210C0ED
:109820001197A01BB10B1696CD010E943351EC018C
:1098300086E0FE01A4E5B8E00D9001928A95E1F77B
:10984000B801CE010E94C972C8010E94BF5160E0F8
:1098500070E8CE010E94926A5C01CE010E94BF5165
:10986000FFEFAF16FFEFBF0639F444E951E0B60150
:10987000C3010E945D4A53C0C5010E94C36B7B01B6
:109880008C0127E638E048EC50E0B601C3010E94A5
:10989000DF49E6018E819F810E94FE4AA80197015F
:1098A000BC01C3010E941D4A888199810397A1F1DF
:1098B000812CE2E09E2EC4010E943351EC01892BE1
:1098C00059F1E114F1040105110519F1E0E0EE167A
:1098D000E2E0FE06E0E00E07E0E01E070CF44701C0
:1098E000A401BE01C5010E94F36A6C019301AC01A1
:1098F00061E070E0CE010E94956D892B51F0C601A8
:10990000AA2797FDA095BA2FE81AF90A0A0B1B0B94
:10991000E9F6CE010E94BF51C5010E94696ADF913C
:10992000CF911F910F91FF90EF90DF90CF90BF905C
:10993000AF909F908F907F906F900895FC018081F1
:10994000882361F0803251F0893041F03196808176
:10995000882321F0803211F08930C1F78081811194
:1099600011928081803211F0893031F431968081FA
:109970008032E1F38930D1F3CF01089582E190E0A4
:109980000E94AA510895CF93DF93EC018E819F81AD
:10999000009711F00E94BF5188859985009711F0BA
:1099A0000E94BF518A859B85009711F00E94BF518C
:1099B0008C859D85009711F00E94BF518E859F85F3
:1099C000009711F00E94BF5188899989009711F082
:1099D0000E94BF51CE010E94BF51DF91CF910895E7
:1099E000CF93DF93EC018091470A9091480A00974A
:1099F00011F00E94BF512097B1F0FE0101900020AC
:109A0000E9F73197EC1BFD0B71F03196CF010E9405
:109A100033519093480A8093470A009741F0BE0162
:109A20000E94F57204C01092480A1092470A80E022
:109A300090E0DF91CF910895AF92BF92CF92DF92E5
:109A4000EF92FF920F931F93CF93DF935C010E94DD
:109A5000BE4C7C01892B09F4A3C180E091E00E94F7
:109A600033516C01009709F498C1A50160E071E0E1
:109A70000E942D6D6DE070E0C6010E94D472EC0171
:109A8000892B09F018826AE070E0C6010E94D47246
:109A9000EC01892B09F0188280E091E00E9433519B
:109AA0008C01892B09F45DC1A50160E071E0C8015A
:109AB0000E942D6D892B09F4D1C06DE070E0C801C2
:109AC0000E94D472EC01892B09F018826AE070E0E0
:109AD000C8010E94D472EC01892B09F01882F801A8
:109AE0008081882309F4BAC04EE050E06AE678E04D
:109AF000C8010E940C73892B01F5F70186859785B3
:109B0000892B91F6E8012E96F8018685803211F0B6
:109B1000893031F4219688818032E1F38930D1F3A4
:109B2000FE0101900020E9F7EC1BFD0BCF010E9424
:109B30003351F701868797878BC04FE050E069E784
:109B400078E0C8010E940C73009721F4F701848328
:109B50009583AACF4DE050E069E878E0C8010E9403
:109B60000C73892B09F5F70182859385892B09F000
:109B70009BCFE8012D96F8018585803211F0893060
:109B800031F4219688818032E1F38930D1F3FE01EE
:109B900001900020E9F7EC1BFD0BCF010E9433512F
:109BA000F7018287938754C047E050E067E978E087
:109BB000C8010E940C73892B09F5F70184859585EE
:109BC000892B09F071CFE8012796F801878180324F
:109BD00011F0893031F4219688818032E1F38930A7
:109BE000D1F3FE0101900020E9F7EC1BFD0BCF0142
:109BF0000E943351F701848795872AC04BE050E0DB
:109C00006FE978E0C8010E940C73892B09F04CCFF2
:109C1000F70180899189892B09F046CFE8012B96BD
:109C2000F8018385803211F0893031F421968881E2
:109C30008032E1F38930D1F3FE0101900020E9F791
:109C4000EC1BFD0BCF010E943351F701808B918BF0
:109C5000009721F0BE010E94F57226CFC8010E9434
:109C6000BF51C6010E949E4C8C010E949E4CEC018B
:109C70000E949E4C6BEA78E0C6010E94B772892B65
:109C800019F481E090E01DC06FEA78E0C6010E94FF
:109C9000B772892B19F483E090E013C064EB78E08D
:109CA000C6010E94B772892B19F482E090E009C0C6
:109CB000C6010E94BF51C7010E94C34C45EF51E04D
:109CC00012C0F70180839183F8018081882319F005
:109CD0008881882369F4C6010E94BF51C7010E9490
:109CE000C34C40E951E0B701C5010E945D4A58C02C
:109CF0008AE090E0F7018283938369EB78E0CE01FC
:109D00000E94B772892B29F489E090E0F7018283E1
:109D100093836FE370E0C8010E94D472EC01892B39
:109D200091F01992FE0101900020E9F7EC1BFD0B68
:109D3000CF010E943351F70180879187009789F006
:109D4000BE010E94F572F80101900020E9F7E01BC6
:109D5000F10BCF010E943351F7018683978300975F
:109D600021F4C6010E94BF5118C0B8010E94F572CB
:109D7000C6010E94BF51F701868197810E941A5047
:109D8000892B39F440E951E0B701C5010E945D4AD1
:109D900004C0B701C5010E944B4BC7010E94C34CD0
:109DA000DF91CF911F910F91FF90EF90DF90CF90B7
:109DB000BF90AF900895EF92FF920F931F93CF93B0
:109DC000DF937C018B01C091490AD0914A0A209708
:109DD000C9F0E114F10439F06A817B81C7010E9466
:109DE000E172892B51F40115110561F06C817D81BF
:109DF000C8010E94E172892B29F00990D881C02DF9
:109E0000209739F7CE01DF91CF911F910F91FF90ED
:109E1000EF9008950F931F93CF93DF93EC018B0185
:109E200086E090E00E943351FC01892B19F48FEFFA
:109E30009FEF10C08091490A90914A0A80839183D4
:109E4000C283D38304831583F0934A0AE093490ABB
:109E500080E090E0DF91CF911F910F9108958F9254
:109E60009F92AF92BF92CF92DF92EF92FF920F93A9
:109E70001F93CF93DF937C018FEF882E982EF701ED
:109E8000068117816FE270E0C8010E9431736C0196
:109E9000009719F0FC01108202C002EC18E060E0AB
:109EA00070E0C8010E94DB4E892BE1F0F701C68506
:109EB000D7852097C9F046E050E064EC78E0CE0109
:109EC0000E949172892B81F42696CE010E94884FC0
:109ED000F701868597850696BC01C8010E94DB4E76
:109EE000892B11F088249924C114D10419F08FE230
:109EF000F6018083C401DF91CF911F910F91FF90F4
:109F0000EF90DF90CF90BF90AF909F908F9008958B
:109F1000CF93DF93AC019FEF60E0EA01DA01888123
:109F2000882309F460C0E881E0320CF457C0FF27B1
:109F3000E7FDF095E359F54EE491EF3F09F44EC08B
:109F4000262F332727FD30956F5F22303105F9F03A
:109F50002330310524F42130310529F03EC023306F
:109F6000310569F13AC0892F992787FD9095880FAF
:109F7000991F880F991F2E2F332727FD30952073A7
:109F8000307094E0359527959A95E1F715C0892FA3
:109F9000992787FD90958F709070F4E0880F991F36
:109FA000FA95E1F72E2F332727FD30952C7330706B
:109FB0003595279535952795822B8D930EC0892F42
:109FC000992787FD90958370907026E0880F991FE0
:109FD0002A95E1F78E2B8D9360E09E2F2196888144
:109FE000882309F0A0CF1C92CA01DF91CF91089578
:109FF000982F80538A3030F4892F992787FD9095C8
:10A00000C0970895892F8156863038F4892F992773
:10A0100087FD9095875590400895892F815486300B
:10A0200030F4892F992787FD9095C79708958FEF72
:10A030009FEF0895BF92CF92DF92EF92FF920F931E
:10A040001F93CF93DF937C016C01FC01B080FFE292
:10A05000BF1619F080E090E038C0EC012196FC01B9
:10A060008181882379F188818532B9F489810E94C0
:10A07000F84F8C0197FD11C08A810E94F84F9C0116
:10A0800097FD0BC02296C80134E0880F991F3A95BE
:10A09000E1F7820F88838823A9F088818C3511F439
:10A0A0008FE288838B2D8E52823020F488818E52ED
:10A0B000823020F0B880F601B1926F01219688813C
:10A0C000882389F6F6011082C701DF91CF911F9195
:10A0D0000F91FF90EF90DF90CF90BF900895EF9297
:10A0E000FF920F931F93CF93DF93FC017B01EA0153
:10A0F00004811581D8014D915C911197FA018481F9
:10A10000958112962D913C911397821B930B8C177E
:10A110009D0708F4EC01209789F0FA018681978168
:10A12000820F931FAE01BC01C7010E94A772F80104
:10A13000828193818C0F9D1F82839383CE01DF9157
:10A14000CF911F910F91FF90EF9008958FEF9FEFA8
:10A1500008958FEF9FEF0895AF92BF92CF92DF9255
:10A16000EF92FF920F931F93CF93DF935C016B01EC
:10A1700086E090E00E9433518C01EE24FF24892B6D
:10A1800049F48CE090E09093B20C8093B10C8FEF87
:10A190009FEF39C0C0914707D0914807209761F0E1
:10A1A0006A817B81C6010E94EB72892B29F009909C
:10A1B000D881C02D2097A1F7209771F084E090E01E
:10A1C0000E94AA517C01009721F0FC01C083D18339
:10A1D00009C08CE090E002C082E090E09093B20C65
:10A1E0008093B10CE114F10441F0F8011082118266
:10A1F000A282B382E482F58205C0C8010E94BF51E9
:10A200000FEF1FEFC801DF91CF911F910F91FF90CA
:10A21000EF90DF90CF90BF90AF900895CF93DF93F2
:10A22000EC01892B69F08FEFCF3FD80749F08C8183
:10A230009D81009711F00E94BF51CE010E94BF5135
:10A2400080E090E0DF91CF910895FC010480F581DA
:10A25000E02D0190F081E02D84819581AA27BB2714
:10A26000BC01CD0108950F931F93CF93DF93AC01F1
:10A27000C0E0D0E0DE0180914D0A90914E0A48176F
:10A28000590720F061C0EF01DB0128C04A5F5F4F32
:10A290004430510510F444E050E0E0914B0AF09155
:10A2A0004C0A6BE47AE03097C9F0208131812417A1
:10A2B000350760F02417350731F3209729F088819E
:10A2C00099812817390710F4EF01DB01BF016E5F98
:10A2D0007F4F0280F381E02D309739F72097A1F16D
:10A2E000CA010A96288139816A817B818E010E5FBD
:10A2F0001F4F8217930770F4FE01E40FF51F241B14
:10A30000350B208331836283738348835983ED93B4
:10A31000FC9302C06D937C9380914D0A90914E0AFC
:10A3200028813981821B930B90934E0A80934D0AAA
:10A33000C20FD31F24978FEE9EEBADEABEED88834C
:10A340009983AA83BB83E801CE01DF91CF911F914E
:10A350000F9108950F931F93CF93DF938C010E9469
:10A360003351EC01009729F0A80160E070E00E94F1
:10A37000B072CE01DF91CF911F910F910895CF93CD
:10A38000DF93DC01129780914D0A90914E0A2D9136
:10A390003C911197820F931F90934E0A80934D0A20
:10A3A000E0914B0AF0914C0A6BE47AE0309709F4A3
:10A3B00051C040815181CF01840F951F8A179B079F
:10A3C000D1F42D913C911197240F351F20833183B7
:10A3D000EF01C20FD31F82819381C817D907D1F52E
:10A3E00088819981280F391F208331838A819B813D
:10A3F000828393832FC0AE17BF07E8F4EB01A883D5
:10A40000B9832D913C911197CD01820F931F8E1727
:10A410009F0761F4240F351F2D933C931197828180
:10A42000938112968D939C93139714C01296ED937B
:10A43000FC9313970FC0A817B90718F48FEF9FEF7D
:10A4400014C0BF016E5F7F4F0280F381E02D309713
:10A4500009F0AFCF309739F41296ED93FC93139730
:10A46000FB01A083B18380E090E0DF91CF9108955C
:10A47000FC0161937193CF010E94BF5108958091B7
:10A480004D0A90914E0A08959F918F910F900BBEA7
:10A490000F900FBE1F9018952F923F924F925F9290
:10A4A0006F927F928F929F92AF92BF92CF92DF92E4
:10A4B000EF92FF920F931F93CF93DF938DB79EB7C9
:10A4C000E091850BF091860B868797878091830BAF
:10A4D0009091840B9093860B8093850BE091850B74
:10A4E000F091860B81E08587E091850BF091860BDA
:10A4F000868597858DBF9EBFDF91CF911F910F916C
:10A50000FF90EF90DF90CF90BF90AF909F908F9093
:10A510007F906F905F904F903F902F900895AF92F3
:10A52000BF92CF92DF92EF92FF920F931F93CF9340
:10A53000DF937C016B015A0189012091EE08309173
:10A54000EF08C90180589F4F8017910710F4021B34
:10A55000130B0FB60F92F894C80147960E9433511F
:10A56000EC01009719F40F900FBE7CC0080F191F63
:10A57000B80167507040A8014B51504028E0C80115
:10A580000496DC01F70101900D922A95E1F7F8019C
:10A590001486C8014C9786879787C18BD28B8FEE24
:10A5A0009EEBADEABEED88839983AA83BB838C833F
:10A5B0009D83AE83BF8388879987AA87BB878C8753
:10A5C0009D87AE87BF8780E4808B8D2D9927FB0107
:10A5D0008583C68280E8838312821482A1828B2DB8
:10A5E0009927808324E432E5832F9927FA01828B0F
:10A5F000238B8091810B9091820BD8018D939C933A
:10A6000011971093820B0093810BC2E01D96CC939F
:10A610001D9753961D921C92549755961D921C920D
:10A62000569763E87BE0C8010E943D538091850BFB
:10A630009091860B892B09F449CF2091850B30919D
:10A64000860B8091830B9091840B2817390739F082
:10A65000E091850BF091860BC5870E944C520F90BC
:10A660000FBEC801DF91CF911F910F91FF90EF9026
:10A67000DF90CF90BF90AF900895CF93DF93EC0120
:10A68000DB016D8B7E8BED91FC911197309771F012
:10A6900080899889981750F0DF0112960280F38123
:10A6A000E02D309719F080899817B0F7EA83FB8383
:10A6B000CD93DC93DF91CF910895DB01ED91FC9177
:10A6C0001197309789F022813381E817F90739F41F
:10A6D0002D933C9312821382158A168A0895DF0106
:10A6E0001296F901232B79F70895CF93DF93EC01AC
:10A6F000892B51F08D85833039F463E87BE0CE01FE
:10A700000E943D5382E08D87DF91CF910895FB0138
:10A71000138A148ACB010E94755308950FB60F92C5
:10A72000F8942091850B3091860B8091830B90914A
:10A73000840B2817390701F5E091850BF091860B02
:10A7400082819381892BC1F0E091850BF091860B7A
:10A75000828193819093840B8093830BE091850B8E
:10A76000F091860B1282138263E87BE08091850B67
:10A770009091860B0E943D532091850B3091860B62
:10A780008091830B9091840B2817390741F0E09159
:10A79000850BF091860B82E085870E944C520F90CA
:10A7A0000FBE08951F93CF93182FE091850BF09162
:10A7B000860BC0890FB60F92F89463E87BE0809116
:10A7C000850B9091860B0E945D53E091850BF09173
:10A7D000860B108B1F3F49F063E87BE08091850B6F
:10A7E0009091860B0E943D5302C00E942F542091ED
:10A7F000850B3091860B8091830B9091840B2817E9
:10A80000390739F4E091850BF091860B81E085875B
:10A8100008C0E091850BF091860B82E085870E944D
:10A820004C520F900FBE8C2F9927CF911F910895F6
:10A830008FEF0E94D25308958091870B9091880BDF
:10A84000892B61F0E091870BF091880B81899289C7
:10A850000E94BF511092880B1092870B08950F939E
:10A860001F93CF93DF93C091810BD091820B01E8AE
:10A870001BE00E941C54209799F08091850B9091C9
:10A88000860BC817D90731F488819981F801808334
:10A89000918306C08E010990D881C02D209769F759
:10A8A0008091850B9091860B9093880B8093870BFA
:10A8B000DF91CF911F910F9108950F931F93CF9325
:10A8C000DF938C01C091810BD091820B209771F0A6
:10A8D000CE010496B8010E94E172892B11F4CE01D9
:10A8E00007C00990D881C02D209791F780E090E0B3
:10A8F000DF91CF911F910F9108952091580A3091C7
:10A90000590AE22FF32F3197F1F78A95D1F708957D
:10A91000CF93DF9380915A0A90915B0AA0915C0AD1
:10A92000B0915D0A0196A11DB11D80935A0A9093C2
:10A930005B0AA0935C0AB0935D0A8091570A80FF7E
:10A940000CC080915E0A90915F0AA091600AB0915C
:10A95000610ACE96A11DB11D0BC080915E0A909137
:10A960005F0AA091600AB091610ACF96A11DB11D46
:10A9700080935E0A90935F0AA093600AB093610A85
:10A980008091570A982F8F5F8093570A9F30A8F0C5
:10A990001092570A8091620A9091630AA091640A0A
:10A9A000B091650A0196A11DB11D8093620A909332
:10A9B000630AA093640AB093650A80914F0A90914C
:10A9C000500A892B09F486C0E0914F0AF091500A91
:10A9D00086819781A085B1850097A105B10579F0A1
:10A9E000E0914F0AF091500A86819781A085B18548
:10A9F0000197A109B10986839783A087B1878091C8
:10AA00004F0A9091500A892B09F464C0E0914F0AD3
:10AA1000F091500A86819781A085B1850097A105A4
:10AA2000B10509F057C0E0914F0AF091500A8285B4
:10AA30009385892BA1F0E0914F0AF091500AA091E3
:10AA40004F0AB091500A0284F385E02D1C966D9157
:10AA50007C911D9780914F0A9091500A0995C09161
:10AA60004F0AD091500AE0914F0AF091500A80812C
:10AA700091819093500A80934F0A8A819B81AC8187
:10AA8000BD818E839F83A887B9870097A105B105F3
:10AA900021F0CE010E94D4550AC08091510A9091B4
:10AAA000520A88839983D093520AC093510A8091A5
:10AAB0004F0A9091500A892B69F0E0914F0AF0916A
:10AAC000500A86819781A085B1850097A105B105BF
:10AAD00009F4A9CFDF91CF910895EF92FF920F93E0
:10AAE0001F9387B78E7F87BF87B78D7F87BF80B75C
:10AAF000886080BF12BE82E083BF40E050E068E81B
:10AB000074E58CE99BE00E946F5900B601FCFDCF13
:10AB100087B7816087BF80E19927AA27B091570A3C
:10AB2000B230E0F3000000000196A11DB091570A79
:10AB3000B330C0F38093530A9093540AA093550AFC
:10AB400087B78E7F87BF8091530A9091540AA09156
:10AB5000550AB091560ABC01CD0120EA30E040E030
:10AB600050E00E943D737B018C016093530A709307
:10AB7000540A8093550A9093560A20EA3FE040E039
:10AB800050E00E948F733093590A2093580AC801ED
:10AB9000B7011F910F91FF90EF9008950E946D559E
:10ABA00087B7816087BF0895CF93DF93EC016FE48F
:10ABB0007AE0E0914F0AF091500A309721F12E810E
:10ABC0003F814885598586819781A085B185281761
:10ABD00039074A075B0748F4821B930BA40BB50B9C
:10ABE00086839783A087B1870EC0281B390B4A0B39
:10ABF0005B0B2E833F8348875987BF010190F0810B
:10AC0000E02D3097E1F6E883F983DB01CD93DC9307
:10AC1000DF91CF9108955F926F927F928F929F9272
:10AC2000AF92BF92CF92DF92EF92FF920F931F935A
:10AC3000CF93DF935B016C014A013901502E0FB6AF
:10AC40000F92F894C091510AD091520A209759F06E
:10AC5000E091510AF091520A808191819093520AB9
:10AC60008093510A05C08EE090E00E943351EC01C0
:10AC70002097B9F1C601B5012DE730E040E050E082
:10AC80000E948F7379018A01E20EF31E041F151FC3
:10AC9000C601B5012DE730E040E050E00E948F731F
:10ACA000DC01CB01CF97A105B10528F00894E11C88
:10ACB000F11C011D111DEE82FF820887198750FECD
:10ACC00005C01A821B821C821D8204C0EA82FB829C
:10ACD0000C831D838A869B866C867D86CE010E94AE
:10ACE000D4550F900FBECE01DF91CF911F910F91E0
:10ACF000FF90EF90DF90CF90BF90AF909F908F909C
:10AD00007F906F905F900895EF92FF920F9361157F
:10AD100071058105910541F10FB60F92F894E0900D
:10AD2000850BF090860B01E02091850B3091860B0E
:10AD300047E853E50E940B56F701838B948B892BD0
:10AD400081F063E87BE08091850B9091860B0E94F7
:10AD50005D53E091850BF091860B83E085870E941F
:10AD60004C520F900FBE02C00E948E530F91FF9065
:10AD7000EF900895CF93DF93EFE4FAE0C0914F0A8C
:10AD8000D091500A209769F128813981C817D907D5
:10AD900021F52083318380819181892B99F0019065
:10ADA000F081E02D86819781A085B1852E813F813C
:10ADB00048855985820F931FA41FB51F86839783EB
:10ADC000A087B1878091510A9091520A8883998314
:10ADD000D093520AC093510A04C0FE01E901232B0B
:10ADE00099F6DF91CF9108950FB60F92F8940E94D3
:10ADF000BA562091510A3091520A2091510A30914D
:10AE0000520A21153105A1F0E091510AF091520A40
:10AE1000808191819093520A8093510AC9010E94C6
:10AE2000BF512091510A3091520A2115310561F725
:10AE30000F900FBE08958091530A9091540AA091EB
:10AE4000550AB091560ABC01CD0108950FB60F9274
:10AE5000F89480915A0A90915B0AA0915C0AB09193
:10AE60005D0A0F900FBEBC01CD0108950FB60F9281
:10AE7000F8948091620A9091630AA091640AB0915B
:10AE8000650A0F900FBEBC01CD0108950FB60F9259
:10AE9000F89480915E0A90915F0AA091600AB09147
:10AEA000610A0F900FBEBC01CD010895AC01DB011A
:10AEB000ED91FC9111978FEFEF3FF807C1F03097BC
:10AEC000B1F083899489228133818417950751F4E5
:10AED0002D933C9312821382138A148ACF010E940D
:10AEE00075530895DF011296F901232B51F7089548
:10AEF000AF92BF92CF92DF92EF92FF920F93CF93D8
:10AF0000DF93EC015A016B010FB60F92F894888120
:10AF100099818F5F9F4F39F4188219820F900FBE6D
:10AF20000E948E534DC063E87BE08091850B909129
:10AF3000860B0E945D53E091850BF091860B83E0B8
:10AF40008587BE018091850B9091860B0E943D53B1
:10AF5000A114B104C104D10481F0E090850BF090FC
:10AF6000860B01E09E0146E557E5C601B5010E944A
:10AF70000B56F701838B948B06C0E091850BF09103
:10AF8000860B138A148A0E944C52E091850BF09133
:10AF9000860B83899489892B39F0E091850BF09198
:10AFA000860B138A148A0AC0A114B104C104D10407
:10AFB00029F00F900FBE8FEF9FEF04C00F900FBED0
:10AFC00080E090E0DF91CF910F91FF90EF90DF90C4
:10AFD000CF90BF90AF900895FC010FB60F92F894F8
:10AFE000808191818F5F9F4F11F410821182CF0178
:10AFF0000E9478570F900FBE0895CF93DF93FC0106
:10B0000020E030E0808191818F5F9F4FC1F0C0814F
:10B01000D181209781F0BF01CE010E945D538B89C1
:10B020009C89009711F00E94BA56CE010E94755378
:10B0300021E030E004C08FEF9FEF80839183C9014E
:10B04000DF91CF9108950F931F930FB60F92F8944D
:10B050000E94FD578C010E948E530F900FBEC801B5
:10B060001F910F9108950F931F93CF93DF93EC01DE
:10B0700000E010E0888199812FEF8F3F920719F44B
:10B08000088319830BC0892B49F0CE010E94FD571C
:10B09000080F191F88819981892BB9F7C801DF91A1
:10B0A000CF911F910F9108950F931F93CF93DF932B
:10B0B000EC0100E010E0888199812FEF8F3F92072B
:10B0C00019F4088319830BC0892B49F0CE010E9423
:10B0D0002358080F191F88819981892BB9F7C80156
:10B0E000DF91CF911F910F9108950F931F93CF93ED
:10B0F000DF938C01C091660AD091670A209761F0B6
:10B10000CE010296B8010E94E172892B29F00990C4
:10B11000D881C02D2097A1F7CE01DF91CF911F914B
:10B120000F910895EF92FF920F931F93CF93DF93A8
:10B13000EC018FEFE82EF82ECF3FD10511F108F189
:10B140006115710511F06C877D8741114E87CE0125
:10B1500002960E9475588C01892B99F4EB89FC8921
:10B16000309721F0CE010995892B59F48091660A18
:10B170009091670A88839983D093670AC093660A7F
:10B180007801C701DF91CF911F910F91FF90EF9050
:10B19000089543E150E060E070E089E89BE00E94A0
:10B1A00067728091890B833141F480918A0B8F34CF
:10B1B00021F480918B0B833519F08FEF9FEF089569
:10B1C00080E090E008950F931F93CF93DF9383E186
:10B1D0008093890B8FE480938A0B83E580938B0B9C
:10B1E00009E81BE0C0E0D0E0CE010E945F72F801E8
:10B1F0006081861719F0CE010E9478720F5F1F4F91
:10B200002196C331D10580F380E090E0DF91CF91AA
:10B210001F910F91089560E070E085E093E008953C
:10B2200080EF98E008958F938FB78F938091A60C4D
:10B23000882361F48DB78093A40B8EB78093A50CFF
:10B2400084EA8DBF8CE08EBF8091A60C839580939D
:10B25000A60C0F921F9211242F933F934F935F934D
:10B260006F937F939F93AF93BF93EF93FF938CE97B
:10B270009BE00E945959FF91EF91BF91AF919F912F
:10B280007F916F915F914F913F912F911F900F9000
:10B29000F8948091A60C8A958093A60C31F4809145
:10B2A000A40B8DBF8091A50C8EBF8F918FBF8F9106
:10B2B0001895FC0180819181A281B3810196A11D25
:10B2C000B11D80839183A283B383268137812115A9
:10B2D000310521F084819581F90109950895FC01DA
:10B2E0000FB60F92F89444835583668377830F904B
:10B2F0000FBE80E090E00895CF93DF93EA016150A4
:10B30000714029F50E941B57DC01CB01880F991F62
:10B31000AA1FBB1F288139814A815B8164E0220F0B
:10B32000331F441F551F6A95D1F7BC01CD010E9400
:10B330008F73DA01C9010196A11DB11DB695A795BC
:10B3400097958795815089B980E090E002C08FEF92
:10B350009FEFDF91CF91089587E089B988E18AB99D
:10B3600080E090E008955D9BFECF8CB98A3011F4A7
:10B370008DE0F9CF0895EF92FF920F931F93CF9333
:10B38000DF937A018B01EA0121978FEFCF3FD80736
:10B3900051F0F80181918F010E94B3592197FFEF7D
:10B3A000CF3FDF07B1F7C701DF91CF911F910F9119
:10B3B000FF90EF900895EF92FF920F931F93CF931A
:10B3C000DF937A018B01EA0121978FEFCF3FD807F6
:10B3D00059F0F80184910E94B3590F5F1F4F2197D4
:10B3E000FFEFCF3FDF07A9F7C701DF91CF911F9193
:10B3F0000F91FF90EF9008951092690A1092680AD9
:10B4000090936B0A80936A0A10926D0A10926C0AEC
:10B4100088E69AE0089580E090E00895782F83E030
:10B4200080930EC0909108C09A7F986080E0592F59
:10B430005160509308C0492F4560409308C08F5F0A
:10B440008132A8F3909308C0392F3460309308C03C
:10B45000509308C0409308C0662349F0909308C0F9
:10B46000309308C0509308C0409308C008C0509360
:10B4700008C0409308C0909308C0309308C080E093
:10B48000909308C0309308C08F5F8530C8F320E1E7
:10B49000872F822329F0509308C0409308C004C02E
:10B4A000909308C0309308C0269591F7909308C0F8
:10B4B000892F99270895CF93DF93C0E0D0E060E013
:10B4C0000E940E5A282F277F209308C0422F4460E5
:10B4D000409308C030E0209308C0409308C0CC0FD0
:10B4E000DD1F809108C0992796958795817090708F
:10B4F000C82BD92B3F5F303170F3209308C0CE01A9
:10B50000DF91CF910895CF93DF93EB0161E00E942B
:10B510000E5A282F782F7160709308C0682F6560CD
:10B52000609308C0809308C0382F3460309308C0FF
:10B5300040E050E8CE0184239523892B29F07093B5
:10B5400008C0609308C004C0209308C0309308C0AE
:10B55000569547954115510569F7277F209308C0F7
:10B56000DF91CF910895CF93DF9360E070E880E0A2
:10B570000E94835AC0E0D0E06FE370E080E090E08A
:10B580000E94845680E00E945B5A99232CF4C430B8
:10B59000D10528F52196F0CF82E10E945B5A60EC3C
:10B5A0007FE383E10E94835A10920EC080E198E00D
:10B5B00080930AC088E090E080930BC061EE71E058
:10B5C00084E00E94835A6FE370E080E090E00E9484
:10B5D0008456C0E0D0E084E0C030D80718F08FEF88
:10B5E0009FEF1FC0CE018F779070892B59F460E0D8
:10B5F00072E180E00E94835A6FE370E080E090E0A7
:10B600000E94845681E00E945B5A85FD08C06FE36A
:10B6100070E080E090E00E9484562196DCCF80E0CC
:10B6200090E0DF91CF9108951F93CF93DF93109215
:10B630000DC010920EC0109204C080E8809305C027
:10B6400011E010930EC0109200C0809301C08AE0F8
:10B650000E947D5410920EC0109204C0109205C03A
:10B66000109200C0109201C010930EC010920CC036
:10B6700088E080930DC082E080930EC080E48093C8
:10B6800000C0C7EED3E0809100C080FF08C081E019
:10B690000E947D5421978FEFCF3FD807A1F7CD2B84
:10B6A00019F48FEF9FEF02C080E090E0009711F057
:10B6B0008FEF9FEFDF91CF911F9108951F93CF934D
:10B6C000DF93EC010E94145B892BB1F483E080933B
:10B6D0000EC087E080930CC010920EC0109204C080
:10B6E00011E0109305C081E8809300C0109201C062
:10B6F0000E94B35A009719F08FEF9FEF16C0109376
:10B700000EC020E0DE01FC01EC5FFF438D918083E1
:10B710002F5FE350F04C2630B8F382E080930EC0E8
:10B7200081E580930DC080E090E0DF91CF911F9183
:10B730000895FF920F931F93CF93DF93FC0101892C
:10B740001289F80186859785A089B1890196A11D86
:10B75000B11D86879787A08BB18B92E090930EC026
:10B76000F0900DC010920DC080910CC08F21C82F99
:10B77000DD27C2FF06C084E080930CC0FBEFFF22F0
:10B7800014C0C1FF16C010920EC0809100C081602D
:10B79000809300C0809100C0109201C090930EC0B1
:10B7A00090930CC080EA809300C0C80102960E946A
:10B7B000FD57C4FF03C080E180930CC0C6FF06C0E4
:10B7C00080E480930CC0C8010E94FD57C0FF08C0F0
:10B7D00081E080930CC08EEFF822C8010E94FD57D3
:10B7E000C3FF06C0E7EFFE2280E79AE00E94FD5704
:10B7F000F0920DC0DF91CF911F910F91FF900895AE
:10B80000FC019B0121503040832F9927982F672BF3
:10B8100039F08191809308C02150D8F79150C8F732
:10B820000895FC019B0121503040832F9927982FC8
:10B83000672B39F0809108C081932150D8F791503F
:10B84000C8F708950F931F93CF93DF9300E010E0A4
:10B8500082E080930EC0809104C0909105C099232E
:10B8600084F1109206C080EE809307C000000000B3
:10B8700000000000809108C0909109C0C09108C0EC
:10B88000D09109C080709C7A892B31F4CE0182540A
:10B890009040835B954018F00FEF1FEF0FC0239788
:10B8A000AE0160E1C8010E944E5E8C01009731F04C
:10B8B000BE01FC01838194810E94115C80E8809329
:10B8C00000C0C801DF91CF911F910F910895CF92D1
:10B8D000DF92EF92FF920F931F93CF93DF937C0140
:10B8E000CC24FC010185128585859685080F191FDA
:10B8F00081899289080F191FF5E00D3D1F0708F097
:10B90000D2C0D0900DC0C0920DC082E080930EC016
:10B9100080E2809300C0C3E6D0E0809100C080FF49
:10B9200008C081E00E947D5421978FEFCF3FD80758
:10B93000A1F7CD2B19F48FEF9FEF02C080E090E0CC
:10B94000892B09F0B0C0E8E0DE2AD0920DC0F701E3
:10B9500085819681080F191F0A5F1F4F00FF04C0E1
:10B960000F5F1F4F81E0C82E80910CC083FD48C03F
:10B970004DE750E060E070E080E79AE00E94785781
:10B98000892BD1F180E4809300C0C7EED3E0809191
:10B9900000C080FF08C081E00E947D542197FFEF26
:10B9A000CF3FDF07A1F780E2809300C0C3E6D0E07D
:10B9B000809100C080FF08C081E00E947D542197E3
:10B9C0008FEFCF3FD807A1F7CD2B19F48FEF9FEF63
:10B9D00002C080E090E0892B21F480910CC083FDAF
:10B9E0000BC04DE750E060E070E080E79AE00E9415
:10B9F0007857892B09F057C080910CC083FFB8CFCE
:10BA0000D0900DC010920DC0809103C0809302C0F1
:10BA1000109206C080E4809307C0109208C0109274
:10BA200008C0009308C0812F9927809309C0F701AF
:10BA300065817681838194810E94005CF701618534
:10BA40007285878190850E94005CF7016585768507
:10BA5000838594850E94005CF701618972898785DE
:10BA600090890E94005CCC2011F0109208C01092C6
:10BA700008C0109209C0C3E6D0E0809100C080FFEA
:10BA800008C081E00E947D542197FFEFCF3FDF0780
:10BA9000A1F7CD2B19F42FEF3FEF02C020E030E0EB
:10BAA0002115310519F08FEF9FEF08C080EC8093CE
:10BAB00000C086E0D82AD0920DC0C901DF91CF9195
:10BAC0001F910F91FF90EF90DF90CF9008957C0130
:10BAD000FC0107851089C189D289F8018181928191
:10BAE000A381B4810097A105B10529F08F5F9F4F15
:10BAF000AF4FBF4F39F46FE370E080E090E00E94F9
:10BB00008456EBCFC80101960E945E5B8AB78460C1
:10BB10008ABF8AB788608ABF89B7806289BF8EE68C
:10BB20009AE00E94235889E00E94D25340ED57E0EA
:10BB300060E070E0CE010E947857D0900DC0109266
:10BB40000DC015C02FEF6F3F720789F08E819F8166
:10BB5000A885B9850196A11DB11D8E839F83A887F5
:10BB6000B987F801218D328DC701F90109950E942D
:10BB7000225CBC01892B31F7F1E4DF2AD0920DC0A1
:10BB8000D5CFCF92DF92EF92FF920F931F93CF9377
:10BB9000DF938C017B019FEFC92ED92E48E95AE330
:10BBA00060E070E08EE69AE00E947857F801C18963
:10BBB000D289C7010E94675C9C01892B61F48A8548
:10BBC0009B85AC85BD850196A11DB11D8A879B878C
:10BBD000AC87BD8769018EE69AE00E942358C601B2
:10BBE000DF91CF911F910F91FF90EF90DF90CF9059
:10BBF00008950F931F93CF93DF93EC0189B78F7D47
:10BC000089BF82E2E989FA8911928A95E9F7AE0142
:10BC100069E97BE587EA9CE00E946F598C01892BDA
:10BC200019F08FEF9FEF0AC020E832E0AE0167E61F
:10BC30007DE58BE199E00E948F52C801DF91CF91A1
:10BC40001F910F9108950F931F93CF93DF93EC01F2
:10BC50008B01CB010E94335188839983009729F48B
:10BC60008A839B838FEF9FEF04C00A831B8380E04E
:10BC700090E0DF91CF911F910F9108950F931F9343
:10BC80008C01FC01808191810E94BF51F8011082DA
:10BC90001182128213821F910F910895BF92CF9249
:10BCA000DF92EF92FF920F931F93CF93DF93EC01FC
:10BCB000B62E7A01892B29F483E190E00E94AA51E3
:10BCC000EC01209709F4C4C0BB2009F4C1C0E11401
:10BCD000F10409F49DC0CB2CDD24C4FE24C08A816C
:10BCE00099278C010071107084FF15C08D819E8191
:10BCF0008E159F0568F48E010D5F1F4FC8010E94CD
:10BD00003E5EB701C8010E94235E892B61F077C0B7
:10BD1000ED82FE8208C0CE010396B7010E94235E29
:10BD2000892B09F04AC0C5FE23C08A8199278C015E
:10BD30000072107085FF15C089859A858E159F0544
:10BD400068F48E01095F1F4FC8010E943E5EB70173
:10BD5000C8010E94235E892B59F051C0E986FA86FA
:10BD600007C0CE010796B7010E94235E892B29F5F3
:10BD7000C6FE28C08A8199278C010074107086FF46
:10BD800015C08D859E858E159F0568F48E01055F13
:10BD90001F4FC8010E943E5EB701C8010E94235E8A
:10BDA000892B81F02CC0ED86FE860CC0CE010B964F
:10BDB000B7010E94235E892B29F0CE010E94B85F53
:10BDC000C80147C0B7FE21C08A8187FF11C0898999
:10BDD0009A898E159F0548F48E01015F1F4FC80197
:10BDE0000E943E5EB701C80106C0E98AFA8A0DC00A
:10BDF000CE010F96B7010E94235E892B31F0CE0150
:10BE00000E94B85F80E090E024C08A818B291FC027
:10BE10008A81B8220B2D112704FF04C0CE0103969E
:10BE20000E943E5E05FF04C0CE0107960E943E5E62
:10BE300006FF04C0CE010B960E943E5EB7FE04C012
:10BE4000CE010F960E943E5EB0948A818B218A8338
:10BE5000CE01DF91CF911F910F91FF90EF90DF9076
:10BE6000CF90BF9008950F931F93CF93DF938C01D2
:10BE700083E190E00E94AA51EC01009709F473C09D
:10BE8000F8016581768161157105A9F003960E941C
:10BE9000235E892B09F051C0AB81BC81F80123815D
:10BEA000348185819681AC01B901CD010E949E72D9
:10BEB0008A8180618A83F8016185728561157105C7
:10BEC000A9F0CE0107960E94235E892BB1F5AF81C0
:10BED000B885F8012781308581859285AC01B9014B
:10BEE000CD010E949E728A8180628A83F8016585F5
:10BEF000768561157105A9F0CE010B960E94235E2F
:10BF0000892BD9F4AB85BC85F801238534858585DB
:10BF10009685AC01B901CD010E949E728A81806430
:10BF20008A83F8016189728961157105D9F0CE01A2
:10BF30000F960E94235E892B31F0CE010E94B85FDC
:10BF400080E090E010C0AF85B889F801278530897E
:10BF500081899289AC01B901CD010E949E728A81CA
:10BF600080688A83CE01DF91CF911F910F91089550
:10BF7000CF93DF93EC01009769F040E050E06A81D5
:10BF80000E944E5ECE010E94BF51892B19F08FEFA7
:10BF90009FEF02C080E090E0DF91CF9108958F93F2
:10BFA0008FB78F938091A60C882361F48DB780930F
:10BFB000A40B8EB78093A50C84EA8DBF8CE08EBF56
:10BFC0008091A60C83958093A60C0F921F9211244A
:10BFD0002F933F934F935F936F937F939F93AF9371
:10BFE000BF93EF93FF9387EA9CE00E945959FF911A
:10BFF000EF91BF91AF919F917F916F915F914F9121
:10C000003F912F911F900F90F8948091A60C8A95E4
:10C010008093A60C31F48091A40B8DBF8091A50C68
:10C020008EBF8F918FBF8F9118951F93CF9310E084
:10C03000C0911F8385E00E947D54C0931F83C0E0A0
:10C0400082E30E947D548091078387FF0BC080911B
:10C050000A83803539F480910B83803719F480E0AE
:10C0600090E008C0CF5FC43158F31F5F143100F374
:10C070008FEF9FEFCF911F910895CF93DF93C0E093
:10C08000D0E00FB60F92F894AE9AA69AAF9AA79AFC
:10C0900084E10E947D5481EE8093008380E480934C
:10C0A000018380916C00836080936C009D9B05C030
:10C0B000219639F09D99FCCF04C0219611F09D9BEB
:10C0C000FCCF80916C008C7F80936C00AE98A6981A
:10C0D000AF98A7980F900FBE809100838132E1F74F
:10C0E000CD2B19F48FEF9FEF02C080E090E0DF913D
:10C0F000CF9108950FB60F92F894AE98A69AAF9A82
:10C10000A79A84E10E947D5481EE8093008380E4AD
:10C110008093018380916C00836080936C0030E099
:10C1200090E09D9BFECF9D99FECF9F5F9B30C8F313
:10C13000E32FFF27E351F54E24913F5F90E89D9B4D
:10C14000FECF822F892309F0AE9A9D99FECFAE983B
:10C150009695A9F7E32FFF27E351F54E24913F5F12
:10C1600090E89D9BFECF822F892309F0AE9A9D997E
:10C17000FECFAE989695A9F79D9BFECF9D99FECFD9
:10C180009F5F9530C8F3323158F280916C008C7FFC
:10C1900080936C00A698AF98A7980F900FBE089553
:10C1A000CF92DF92FF920F931F93CF93DF936C0197
:10C1B0000E941560EC01892B19F08FEF9FEF68C08A
:10C1C0000E943D60892B11F40E947A6010920F83C7
:10C1D0001FEF1093078381EE8093008380EC8093A0
:10C1E000018300E20093058380E4F82EF092068339
:10C1F00010920183812F0E947D5481E280930083FD
:10C2000088E480930E8310920A8310920B8300932C
:10C210000C8382E080930D83F09204838FE58093FA
:10C22000038386E48093018380E6809302831093E6
:10C23000078381E68093008390E0D601FE01EF5FE3
:10C24000FC478D9180839F5FE050F3489630B8F3B0
:10C2500090E0E8E0F3E811929F5F9830E0F386E425
:10C260008093078381E28093008384E080930C8332
:10C270009FEF909307838DE180930F8382E28093F9
:10C28000008310920D83892F0E947D5480E090E0FE
:10C29000DF91CF911F910F91FF90DF90CF90089584
:10C2A00082E28093008390E08091078386FD03C043
:10C2B0009F5F9531C8F380E4809307830895FC0164
:10C2C0009B0121503040832F9927982F672B39F0FD
:10C2D0008191809310832150D8F79150C8F7089529
:10C2E000FC01AB019B0121503040832F9927982FEF
:10C2F000452B39F08091108381932150D8F79150CC
:10C30000C8F70895DF92EF92FF920F931F93CF9398
:10C31000DF93EC01DD240D811E8189859A85080F4C
:10C32000191F8D859E85080F191F89899A89080F05
:10C33000191F85E00B3E180718F08FEF9FEF59C0CB
:10C340000C33110528F4ECE3DE2ED01A0CE310E0D8
:10C350008091008382FF06C00E948E5380910083EB
:10C3600082FDFACF89B78F7D89BF00930A83E12EC2
:10C37000FF24E0920B831092088380E4809309836A
:10C3800082E1809300836D817E818B819C810E94FC
:10C390005F6169857A858F8198850E945F616D856F
:10C3A0007E858B859C850E945F6169897A898F85EE
:10C3B00098890E945F6180E090E02D2D33278217DD
:10C3C000930730F410921083019682179307D0F3ED
:10C3D0000E94506100930583E092068380E480937D
:10C3E000048386E28093008389B7806289BF80E0FE
:10C3F00090E0DF91CF911F910F91FF90EF90DF9030
:10C400000895BF92CF92DF92EF92FF920F931F9306
:10C41000CF93DF93CDB7DEB724970FB6F894DEBF86
:10C420000FBECDBFCC24DD24BB2489B78F7D89BF4F
:10C4300082E68093008300000000000000000000FE
:10C4400000000000000000000000000000000000EC
:10C450000000000000009091078382E28093008337
:10C46000E0900383E3944FE54E1510F426E4E22EAA
:10C47000E91609F49CC084E080930A83B0920B8390
:10C48000B0920883E09209838E010F5F1F4FF8017D
:10C490008AE080930083000000000000000000009C
:10C4A000000000000000000000000000000000008C
:10C4B00000000000000096018091108381932F5F9F
:10C4C0003F4F24303105C0F30E945061F8012281B2
:10C4D0003381C901805490408F5A954010F081E01B
:10C4E000B82E232F33272E0D311DF801828188238A
:10C4F00011F02F5F3F4FF22EFFE5F21710F446EEDA
:10C50000F40EF8019181F91671F08F2D8F5F80364E
:10C5100008F08A51891731F089B7806289BF8FEF9F
:10C520009FEF49C0F82EBB2009F039C089819927B7
:10C530008E709070009709F032C0F801028113816B
:10C5400004501040A80160E10E944E5E6C01892BEE
:10C5500031F100930A83812F992780930B8384E024
:10C5600080930883E09209838AE08093008300002F
:10C5700000000000000000000000000000000000BB
:10C580000000000000000000000000000000B801F2
:10C59000F601838194810E9470610E945061FA9437
:10C5A000F5E4FF1510F0FFE5FF2EF092038389B745
:10C5B000806289BFC60124960FB6F894DEBF0FBE15
:10C5C000CDBFDF91CF911F910F91FF90EF90DF9042
:10C5D000CF90BF90089530E08091008382FDFCCF22
:10C5E0008091008391E6909300832091078391E2EC
:10C5F0009093008310920A8310920B8382FF08C0ED
:10C600008091078399278A709070892B09F431E013
:10C6100082E080930D8382E2809300832150263450
:10C6200008F42FE52093038310920D83332319F030
:10C6300086E28093008380E180930783832F99278C
:10C6400008950F931F93CF93DF93FC01C189D28983
:10C650008A859B85AC85BD850196A11DB11D8A8704
:10C660009B87AC87BD878091078380930783082FC2
:10C67000112704FF0EC00E94EB628E859F85A8895A
:10C68000B9890196A11DB11D8E879F87A88BB98B93
:10C690003EC003FF0BC08AA19BA1ACA1BDA1019626
:10C6A000A11DB11D8AA39BA3ACA3BDA300FF03C022
:10C6B000CE010E94FD5702FF2AC020910D838A8976
:10C6C0009B89AC89BD89820F911DA11DB11D8A8BEB
:10C6D0009B8BAC8BBD8B20910E838E899F89A88DFF
:10C6E000B98D820F911DA11DB11D8E8B9F8BA88FBF
:10C6F000B98F20910F838A8D9B8DAC8DBD8D820F5C
:10C70000911DA11DB11D8A8F9B8FAC8FBD8FDF91B5
:10C71000CF911F910F9108956C01FC01C785D089BD
:10C72000E188F28889E00E94D25389819A81892325
:10C730009B8189238F3FB9F46DE770E080E090E042
:10C740000E94845689819A8189239B8189238F3F06
:10C7500099F389B78F7D89BFCE0101960E94D06081
:10C7600089B7806289BF40E050E060E070E0C701B7
:10C770000E9478570E9401628C01FFEF8F3F9F0754
:10C7800089F4CE0101960E94D060F701868D978DC5
:10C79000A0A1B1A10196A11DB11D868F978FA0A365
:10C7A000B1A313C0892B89F0F70182819381A48101
:10C7B000B5810196A11DB11D82839383A483B583A6
:10C7C000E98DFA8DB801C6010995012B99F6CBCFF9
:10C7D0000F931F93CF93DF93FC01CB010FEF1FEF5C
:10C7E000C189D2890E9482619C01892B61F48E816A
:10C7F0009F81A885B9850196A11DB11D8E839F8358
:10C80000A887B9878901C801DF91CF911F910F9146
:10C810000895EF92FF920F931F93CF93DF93EC0154
:10C8200080915D0B882321F4CE0102960E94652B36
:10C830000F85188986E078010894E11CF11CF70146
:10C84000A7E6BBE00D9001928A95E1F786E2E989BF
:10C85000FA8911928A95E9F720E832E0AE016CE896
:10C8600073E684EA99E00E948F5264EF71E080E001
:10C8700090E00E948456AE0161E273E687EA9CE094
:10C880000E946F59892B79F489B78F7D89BFF80190
:10C8900091818281982B8381982B41F0C7010E945E
:10C8A000D060892B19F08FEF9FEF05C089B78062A8
:10C8B00089BF80E090E0DF91CF911F910F91FF90B1
:10C8C000EF900895CF93DF93EC01892B69F5809168
:10C8D000A9099091AA0901969093AA098093A909A0
:10C8E000892B31F480E090E19093AA098093A90903
:10C8F0002091A9093091AA09E9010C2ECD2FD02D44
:10C90000AE01E091AF0CF091B00C309751F0828104
:10C9100093818417950729F00190F081E02D3097DD
:10C92000B1F7EF2BA1F6E9018CE090E00E94AA514B
:10C93000FC01892B79F00C2ECD2FD02DC283D3830F
:10C940008091AF0C9091B00C80839183F093B00CE8
:10C95000E093AF0CCF01DF91CF9108956F927F925A
:10C960008F929F92AF92BF92CF92DF92EF92FF92FF
:10C970000F931F93CF93DF933C015A016B01490141
:10C98000A70160E880E090E00E944E5EEC01892BF8
:10C9900019F48FEF9FEF14C08F859889A701B80114
:10C9A0000E949E728E019401B601A501C3010E94EE
:10C9B00062668C01892B19F4CE010E94B85FC80110
:10C9C000DF91CF911F910F91FF90EF90DF90CF906B
:10C9D000BF90AF909F908F907F906F9008954F92EF
:10C9E0005F926F927F928F929F92AF92BF92CF92FF
:10C9F000DF92EF92FF920F931F93CF93DF935C012F
:10CA00004B013A012901FC0184819581892B31F484
:10CA1000C5010696B701A6010E947857F501C481A9
:10CA2000D581209711F48E0131C088819981F5015B
:10CA300084839583EF81F88584859585A685B78560
:10CA4000F40180839183A283B383EB85FC8580818D
:10CA50009181082E892F902DF3018083918329895C
:10CA60003A892017310708F48901F50180859185FD
:10CA7000821B930B808791878F859889A801BC01C1
:10CA8000C2010E949E72CE010E94B85FC801DF9170
:10CA9000CF911F910F91FF90EF90DF90CF90BF90BB
:10CAA000AF909F908F907F906F905F904F90089580
:10CAB000CF93DF93EC018FEF9FEFAFEABCE0E09103
:10CAC000AF0CF091B00C309709F120813181EC1757
:10CAD000FD07C1F42D933C930480F581E02D309740
:10CAE00059F0808191818C839D83CF010E94B85F32
:10CAF000EC81FD813097A9F7CE010E94BF5180E003
:10CB000090E004C0DF01F901232BF9F6DF91CF910A
:10CB100008959C0140E050E0E091AF0CF091B00C22
:10CB2000309761F0828193818217930711F4AF01EE
:10CB300005C00190F081E02D3097A1F7CA0108955A
:10CB4000DC01FA018FEF9FEF109781F06250704186
:10CB500069F4309759F02230310541F48081918198
:10CB60001A968D939C931B9780E090E00895CF9345
:10CB7000DF93DC01FA018FEF9FEF109781F0625095
:10CB8000704169F4309759F02230310541F41A961A
:10CB90008D919C911B978083918380E090E0DF9141
:10CBA000CF910895CF93DF939C01DB011396ED9114
:10CBB000FC9114973E961796ED93FC9318973E9729
:10CBC00015968D919C9116970E9719968D939C931F
:10CBD0001A978EE090E015968D939C931697848516
:10CBE0009585082E892F902D48E08030940721F0FC
:10CBF0008650984029F008C0C9010E94FD6607C010
:10CC0000C9010E945A6903C0CB010E94B85FDF913D
:10CC1000CF9108958F929F92AF92BF92CF92DF9261
:10CC2000EF92FF920F931F93CF93DF934C017B0101
:10CC30005A0189014EE050E060E1C9010E944E5E58
:10CC4000892B89F1F801C381D481F401C784D0888C
:10CC500086E0DE011696F601319601900D928A95D6
:10CC6000E1F7A114B10441F086E0DE01F501019085
:10CC70000D928A95E1F707C046E050E06FEF70E053
:10CC8000CE010E94B0720E2CEF2CF02CEC86FD86AB
:10CC9000E601EB8DFC8DB801C4010995009729F0E0
:10CCA000C8010E94B85F8FEF9FEFDF91CF911F9176
:10CCB0000F91FF90EF90DF90CF90BF90AF909F903B
:10CCC0008F9008954F925F926F927F928F929F9272
:10CCD000AF92BF92CF92DF92EF92FF920F931F938A
:10CCE000CF93DF93CDB7DEB724970FB6F894DEBFAE
:10CCF0000FBECDBF2C013A014B01790148E050E055
:10CD000060E4C8010E944E5E6C01009719F48FEF39
:10CD10009FEF5CC0FC01A384B484F2018281938103
:10CD2000F501808391830E2CEF2CF02CE282F382AC
:10CD3000F6018585968521893289820F931F082EF9
:10CD4000892F902DF50184839583AE014F5F5F4F4E
:10CD5000C401B3010E94C128FC01892B61F0078442
:10CD6000F089E02D87819085A185B28589839A839A
:10CD7000AB83BC8304C019821A821B821C82F5011A
:10CD800016821782E480F58001E1A4019301698194
:10CD90007A818B819C810E94E737DC01CB0148E0DE
:10CDA00050E0B5010E94A737AA27BB27F6014189A9
:10CDB0005289678570890E94E237F50186839783DF
:10CDC0009601B401A301802F0E94303824960FB63B
:10CDD000F894DEBF0FBECDBFDF91CF911F910F91B1
:10CDE000FF90EF90DF90CF90BF90AF909F908F908B
:10CDF0007F906F905F904F9008952F923F924F9247
:10CE00005F926F927F928F929F92AF92BF92CF92DA
:10CE1000DF92EF92FF920F931F93CF93DF93CDB7E3
:10CE2000DEB725970FB6F894DEBF0FBECDBF89835E
:10CE30009A836C837D83FB0167807084F30120817A
:10CE4000822F807F803409F0C0C086819781082EB0
:10CE5000892F902D9F73892B09F0B7C02F70222E38
:10CE60003324220C331C220C331CF301808891885C
:10CE7000A288B388E981FA8147845088FFEF8F1632
:10CE8000FFEF9F06FFEFAF06FFEFBF06F9F0F201DD
:10CE90000781108521853285011511052105310590
:10CEA000C1F087859089A189B2898F3FFFEF9F07E5
:10CEB000FFEFAF07FFEFBF0761F088299929AA2983
:10CEC000BB298F5F9F4FAF4FBF4F19F481E08B831A
:10CED00038C01B820115110521053105E9F4F30164
:10CEE00081858130C9F4D501C40180709070A07033
:10CEF0008030F0E09F07F0E0AF07FFEFBF0761F081
:10CF00000097A105B10541F068017901B501A401BF
:10CF100089819A810E94AE29F20187819085A1853D
:10CF2000B2850097A105B10561F081149104A104B7
:10CF3000B10409F44AC088169906AA06BB0609F08E
:10CF400044C0EC81FD8121863286C301820D931D90
:10CF500083879487F30182819381082E892F902DF6
:10CF600082199309EC81FD8185879687F30181857C
:10CF7000992786309105A9F0873091051CF4019717
:10CF800021F017C0419741F014C06C817D818981E7
:10CF90009A810E9460681DC08C819D810E94FC69FD
:10CFA00018C0FB81FF2389F48C819D810E94C56993
:10CFB00010C00C811D8120E030E040E050E062E0D4
:10CFC00083E00E940069892B21F48C819D810E945D
:10CFD000B85F25960FB6F894DEBF0FBECDBFDF91C8
:10CFE000CF911F910F91FF90EF90DF90CF90BF9066
:10CFF000AF909F908F907F906F905F904F903F90F9
:10D000002F900895FF920F931F93CF93DF93FC010E
:10D01000F62E8A01EA012F813885E9014C855D856C
:10D020006E857F850784F089E02D87819085A185B5
:10D03000B2858C879D87AE87BF878FEF88879801E1
:10D040008F2D0E949068DF91CF911F910F91FF90DB
:10D050000895CF93DF93EC0189899A894D9700F168
:10D06000AF85B88919968C9119978630C9F4CD018E
:10D0700080579E4F1C962D913D914D915C911F972D
:10D08000FC0160817181828193810E949022FC0168
:10D09000892B31F08389823031F08389843019F013
:10D0A0008FEF9FEF0AC061E577E2CF010E94193749
:10D0B000CE010E94B85F80E090E0DF91CF910895AB
:10D0C000CF93DF939C01EB018D859E85893091057F
:10D0D00008F1EB85FC850897898B9A8B3896EF874A
:10D0E000F88B389788E090E08D879E87808199271C
:10D0F0008330910551F0089769F4AB0160E0C901F4
:10D100000E940268892B49F405C0CB010E9429685E
:10D11000892B19F0CE010E94B85FDF91CF9108955D
:10D12000AF92BF92CF92DF92EF92FF920F931F9335
:10D130005A016B018901F901E384F484F7018083CA
:10D1400012821382F901458556856385748580E0D6
:10D1500090E00E94A737F80141895289678570895C
:10D160000E94E237F701828393839801B601A501FB
:10D1700081E00E9430381F910F91FF90EF90DF9077
:10D18000CF90BF90AF9008956F927F928F929F92B1
:10D19000AF92BF92CF92DF92EF92FF920F931F93C5
:10D1A000CF93DF93782E662E49015A0148E050E074
:10D1B00060E4C6010E944E5EDC01009719F48FEF17
:10D1C0009FEF0FC01B96ED91FC911C9761828482AA
:10D1D0009582A682B7829C01B801A701872D0E9483
:10D1E0009068DF91CF911F910F91FF90EF90DF90AA
:10D1F000CF90BF90AF909F908F907F906F90089549
:10D200006F927F928F929F92AF92BF92CF92DF9256
:10D21000EF92FF920F931F93CF93DF93682E762E9A
:10D2200049015A01D8011796ED91FC911897E484B1
:10D23000F584068517854CE150E060E8CD010E9439
:10D240004E5EDC01892B19F48FEF9FEF24C084E13F
:10D250001F96CD91DC91509717962D913C91189780
:10D26000F901019009928A95E1F71F96ED91FC91E1
:10D27000509788E074961B962D913C911C97E9017C
:10D28000099001928A95E1F76D01A5019401672D3E
:10D29000862D0E94C468DF91CF911F910F91FF905E
:10D2A000EF90DF90CF90BF90AF909F908F907F9046
:10D2B0006F900895CF92DF92EF92FF920F931F939A
:10D2C000CF93DF936C017B01FB01C781D0858881FF
:10D2D0009981082E892F902D019709F04AC08A81E3
:10D2E0009B81082E892F902D8050984009F041C0D5
:10D2F0008C81863009F03DC08D81843009F039C0C1
:10D30000F601A785B089288D398D4A8D5B8D1796DA
:10D310008D919D910D90BC91A02D281739074A073A
:10D320005B0739F58E01085F1F4F98014E855F85B9
:10D3300068897989C6010E94363A8E819F81082EBC
:10D34000892F902D0197A9F498014E855F856889F2
:10D35000798982E090E00E94003BEC01009749F05F
:10D36000BC01C6010E94593B892B19F4CE010E94D1
:10D37000B85FC7010E94B85FDF91CF911F910F91F5
:10D38000FF90EF90DF90CF900895CF93DF93FC0153
:10D39000A385B4851C968C911C9782958F70282F3D
:10D3A0003327220F331F220F331F85859685821B5B
:10D3B000930B818B928B892B71F01C968C911C970F
:10D3C00082958F709927880F991F880F991F8A0F50
:10D3D0009B1F8787908B1C968C9182958F709927C5
:10D3E000880F991F880F991F85879687CF010E9404
:10D3F0009B36DF91CF9108950F931F93CF93DF93C7
:10D40000EC01EB85FC853896EF87F88B38978D8596
:10D410009E850897898B9A8B88E090E08D879E8700
:10D42000828193810E9489658C01009721F4CE014D
:10D430000E94B85F49C0FC01228533852115310562
:10D4400059F14085518569897A89CA01860F971FEC
:10D450002817390720F4CE010E94B85F2BC0F801CD
:10D4600084819581009779F0FC0180819181892BDD
:10D4700039F00190F081E02D80819181892BC9F7ED
:10D48000C083D18303C0F801C483D583460F571FDF
:10D49000F801408751870EC0FC0184819581009777
:10D4A00011F00E94B85FF801C483D58389899A89F5
:10D4B00080879187F80186819781892B29F00A5FFF
:10D4C0001F4FC8010E942358DF91CF911F910F91E8
:10D4D0000895CF93DF93EC01AA81BB81109731F4BB
:10D4E000EF81F885AD01BD01099506C05F962D91CC
:10D4F0003C919097F9010995DF91CF910895CF93D1
:10D50000DF93EC01AA81BB81109719F4EB85FC85B0
:10D5100005C05596ED91FC915697CD010995DF9187
:10D52000CF910895CF92DF92EF92FF920F931F93C6
:10D53000CF93DF93CDB7DEB729970FB6F894DEBF50
:10D540000FBECDBF7B018C0140E0FC0180818823B0
:10D55000A9F08A3399F020E030E0FE01E20FF31FDA
:10D5600081830F5F1F4F4F5F2F5F3F4FF801808117
:10D57000882321F08A3311F0483078F3CE010196E8
:10D58000FC01E40FF11D10820E947558DC01892B0B
:10D5900049F482E090E09093B20C8093B10C8FEF4D
:10D5A0009FEF12C0F80181918F018A3311F000E0E2
:10D5B00010E05D96CD90DC905E9720E030E0A70112
:10D5C000B801CD01F601099529960FB6F894DEBF92
:10D5D0000FBECDBFDF91CF911F910F91FF90EF90C4
:10D5E000DF90CF900895CF93DF93DC011296ED91F9
:10D5F000FC911397309729F41596ED91FC911697AD
:10D6000003C00788F08DE02D0995DF91CF91089533
:10D61000EF92FF921F93CF93DF93EC018FEFE82EF1
:10D62000F82E209739F489E090E09093B20C809323
:10D63000B10C38C010E08091AB099091AC098C1707
:10D640009D0771F01F5F183090F4E12FFF27EE0F58
:10D65000FF1FE555F64F808191818C179D0791F74B
:10D66000CF3FD10509F060F480E090E01CC089E074
:10D6700090E09093B20C8093B10C8FEF9FEF13C0AA
:10D68000888199810E94696A009709F47C01CE0122
:10D690000E945A6EE12FFF27EE0FFF1FE555F64F50
:10D6A00010821182C701DF91CF911F91FF90EF90FF
:10D6B0000895CF92DF92EF92FF920F931F93CF9333
:10D6C000DF936C01CB010E94076C7C018FEFE816A1
:10D6D0008FEFF80699F103E08091B1099091B209BA
:10D6E000892B69F0073020F50F5FE02FFF27EE0F41
:10D6F000FF1FE555F64F80819181892B99F7C02F47
:10D70000DD278E010C0F1D1F0555164F87E090E099
:10D710000E94576EFC01D8018D939C93892B89F050
:10D72000C082D182E282F3821482158216820FC0F7
:10D7300087E190E09093B20C8093B10C80E090E090
:10D740000CC08CE090E09093B20C8093B10CCC0FA5
:10D75000DD1FC555D64F88819981DF91CF911F91EB
:10D760000F91FF90EF90DF90CF900895FC0140E083
:10D7700050E0BA01808191810E94E171009711F01F
:10D780008FEF9FEF0895CF93DF93CDB7DEB7249748
:10D790000FB6F894DEBF0FBECDBFDC0112968D919F
:10D7A0009C9113970097B1F41B962D913C911C9777
:10D7B00021153105A9F0AE014F5F5F4F6AE070E0BF
:10D7C000CD01F9010995892B59F469817A818B8101
:10D7D0009C8114C0FC0121A132A12115310559F40D
:10D7E00089E090E09093B20C8093B10C6FEF7FEFE3
:10D7F0008FEF9FEF03C0CD01F901099524960FB675
:10D80000F894DEBF0FBECDBFDF91CF910895FC012C
:10D8100040E050E48081282F332727FD30952237C0
:10D82000310579F02337310524F42136310539F0FB
:10D830001EC027373105D9F441E050E402C048E06A
:10D8400050E4319680818823F9F08081282F332796
:10D8500027FD30952B32310521F02236310521F09C
:10D8600006C04E7F42600CC05F7B506809C086E1F5
:10D8700090E09093B20C8093B10C8FEF9FEF0895DE
:10D8800031968081882309F7CA010895CF92DF92EB
:10D89000EF92FF920F931F93CF93DF936C01CB0115
:10D8A0000E94076C7C018F5F9F4FD1F123E0809134
:10D8B000B1099091B209892B69F0273058F52F5F93
:10D8C000E22FFF27EE0FFF1FE555F64F8081918174
:10D8D000892B99F7C22FDD27CC0FDD1FC555D64FF9
:10D8E00087E090E00E94576E8C01888399830097AF
:10D8F00021F1B701C6010E94926AF80180839183E9
:10D900008F5F9F4F81F4888199810E945A6E18829F
:10D91000198206C087E190E09093B20C8093B10C1D
:10D9200080E090E00AC0E881F981E282F38214820B
:10D93000E881F98115821682CF01DF91CF911F9185
:10D940000F91FF90EF90DF90CF9008958F929F926C
:10D95000BF92CF92DF92EF92FF920F931F93CF93DC
:10D96000DF934C01CB01EA010E94076C6C018F5FD1
:10D970009F4F09F459C0BB248091AB099091AC0929
:10D980008C179D0781F0B39487E08B1508F446C08F
:10D99000EB2DFF27EE0FFF1FE555F64F808191819C
:10D9A0008C179D0781F7E1E0C130DE0728F0888100
:10D9B00099810E94696A0FC00B2D1127000F111F5A
:10D9C0000555164F87E090E00E94576EF80180835E
:10D9D00091830097B1F1EB2CFF24E701CE0DDF1D01
:10D9E000C555D64F08811981B601C4010E94926ABB
:10D9F000F801808391838F5F9F4FC9F4888199815B
:10DA00000E945A6E22E02B1530F00894E11CF11CA4
:10DA1000E882F98209C01882198206C089E090E084
:10DA20009093B20C8093B10C80E090E00AC0E88142
:10DA3000F981C282D3821482E881F981158216822B
:10DA4000CF01DF91CF911F910F91FF90EF90DF9069
:10DA5000CF90BF909F908F900895CF92DF92EF92DA
:10DA6000FF920F931F93CF93DF937C01EB016A0129
:10DA70008C01219762307105ACF0C6010E940B72D7
:10DA80002FEF8F3F920729F4F801108280E090E099
:10DA90000CC0F80181938F010A9721F0CE012197E4
:10DAA00002975CF7F8011082C701DF91CF911F91B7
:10DAB0000F91FF90EF90DF90CF900895CF93DF9379
:10DAC000CDB7DEB72D813E818F819885AE01475F4E
:10DAD0005F4FBC01C9010E941F6EDF91CF91089575
:10DAE000DC01CB01FD0101900020E9F73197EA1B31
:10DAF000FB0BAF01BD01FC01808191810E94E171AE
:10DB00000895EF92FF920F931F938C017B010E9467
:10DB10000373AC01B801F701808191810E94F67115
:10DB20001F910F91FF90EF900895CF93DF93EB013A
:10DB3000F9016230710540F0469F9001479F300D1A
:10DB4000569F300D1124A901BC01808191810E9452
:10DB5000E171BC01181619061CF060E070E006C007
:10DB6000C230D10518F0BE010E946873CB01DF916D
:10DB7000CF910895CF93DF93CDB7DEB7E5E0F0E026
:10DB8000EC0FFD1F81919191AF01BC018091AD0916
:10DB90009091AE090E94156EDF91CF910895CF93B9
:10DBA000DF93CDB7DEB7E5E0F0E0EC0FFD1F81912C
:10DBB0009191AF01BC018091AD099091AE090E9495
:10DBC0001F6EDF91CF9108956091AD097091AE09FC
:10DBD0000E94377208956091AD097091AE090E945C
:10DBE000706D2FEF8F3F920751F06091AD097091EA
:10DBF000AE098AE090E00E94377280E090E00895DC
:10DC00006091AD097091AE090E94816D2FEF8F3F39
:10DC1000920751F06091AD097091AE098AE090E0F1
:10DC20000E94377280E090E00895FC019A01AB01F8
:10DC30006081718181EE91E70E948B6E0895AF92B1
:10DC4000BF92CF92DF92EF92FF920F931F93CF93E9
:10DC5000DF935C018B016A01CB010E940373EC012D
:10DC60002196CE010E9433517C01009719F48FEF69
:10DC70009FEF12C0AE01B8010E94A7729601A701E2
:10DC8000F5016081718181EE91E70E948B6E8C01BC
:10DC9000C7010E94BF51C801DF91CF911F910F9121
:10DCA000FF90EF90DF90CF90BF90AF9008950E94CB
:10DCB0003351089521E08130920710F00E94BF5146
:10DCC0000895CF92DF92EF92FF920F931F93CF931D
:10DCD000DF936C017B018A01E9012131310554F0A8
:10DCE00040E150E0B801C701F60109956097C131E4
:10DCF000D105B4F71C161D062CF4AE01B801C701FE
:10DD0000F6010995DF91CF911F910F91FF90EF9050
:10DD1000DF90CF9008952F923F924F925F926F9233
:10DD20007F928F929F92AF92BF92CF92DF92EF92AB
:10DD3000FF920F931F93CF93DF93CDB7DEB76B970F
:10DD40000FB6F894DEBF0FBECDBF8A8B9B8B6C8B5A
:10DD50007D8B3A0149011E8A1F8A6301F3015080BD
:10DD6000552069F0F5E25F1651F00894611C711CB2
:10DD7000F3015080552019F0F5E25F16B1F78301E9
:10DD80000C191D0971F0A801B6018C899D892A8999
:10DD90003B89F90109954E895F89400F511F4E8BD0
:10DDA0005F8B552009F4F2C20894611C711C442455
:10DDB000498A188E198E80E090E08A8F9B8F8FEFB2
:10DDC000282E382EF30151903F01F0E25F1621F426
:10DDD00089898823B9F703C02BE2521611F4598AB6
:10DDE000F1CF3DE2531619F444E0442AEBCF53E25D
:10DDF000551619F481E0482AE5CF90E3591619F435
:10DE0000E0E14E2ADFCFFCE65F1619F428E0422A53
:10DE1000D9CF3AE25316A1F4F40142E050E0840E67
:10DE2000951E0190F081E02DE88FF98FF7FFCACFA2
:10DE300054E0452AF095E195FF4FE88FF98FC2CF66
:10DE40008EE2581689F5F30180818A3259F40894DC
:10DE5000611C711CF40122E030E0820E931E2080D0
:10DE600031801FC02224332480538A30D0F4C10172
:10DE700003E0880F991F0A95E1F7820D931D280E84
:10DE8000391EF30181913F01992787FD9095280E56
:10DE9000391E20ED3FEF220E331E808180538A30E1
:10DEA00030F337FE8FCF8BCF852D8153252D332730
:10DEB000893060F520533040288F398FF30120815D
:10DEC000822F80538A3008F07DCF888D998D13E0A2
:10DED000880F991F1A95E1F7488D598D840F951F6A
:10DEE000480F591F822F992787FD9095480F591F7A
:10DEF00040535040488F598F0894611C711CF301A6
:10DF00002081822F80538A3000F35CCF2836310580
:10DF100004F5253631050CF0A8C12035310509F48A
:10DF200044C0213531054CF42534310509F49DC137
:10DF30002734310509F499C19CC12336310549F1D3
:10DF4000243631050CF079C02835310509F42CC18F
:10DF500090C12037310509F427C1213731054CF430
:10DF60002936310509F469C02F36310509F4D8C0C6
:10DF700080C12537310509F45FC02637310524F407
:10DF80002337310571F175C12837310509F40CC10A
:10DF900070C16E010894C11CD11CF40122E030E074
:10DFA000820E931E808189836CC1F40142E050E0AF
:10DFB000840E951EC080D180C114D10419F4B3E73A
:10DFC0005B2E16C0C6010E9403738C010F5F1F4FAA
:10DFD000C8010E94576E5C01B6010E94FC72650187
:10DFE00007C0F40182E090E0880E991EC080D180C5
:10DFF000C114D10421F4ABEDCA2EA9E0DA2E37FC0E
:10E0000011C0A10160E070E0C6010E948372009718
:10E0100039F08C010C191D09201631060CF033C1A2
:10E02000810131C1F60101900020E9F78F01015013
:10E0300010400C191D0927C1198A43FE0AC0F401BA
:10E0400024E030E0820E931EE080F1800281138193
:10E0500016C0C401029635E7531641F4F4014C0191
:10E06000808191817C010027112709C0F4014C01B6
:10E07000808191817C010027F7FC0095102F45E7F6
:10E08000541661F017FF0AC010950095F094E094C3
:10E09000E11CF11C011D111D8DE2898B2A8E3B8E26
:10E0A00037FC02C05FEE4522F1E1CF2ED12CCC0E21
:10E0B000DD1EE114F1040105110529F48A8D9B8D03
:10E0C000892B09F4CCC09AE0E916F1040105110589
:10E0D00048F4E0E1CE2ED12CCC0EDD1E8E2D805DDD
:10E0E000888BBDC0C801B7012AE030E040E050E0B5
:10E0F0000E948F73DC01CB01805DF60182936F017A
:10E10000C801B7012AE030E040E050E00E948F7380
:10E1100079018A01211531054105510519F79FC083
:10E1200043FE0AC0F40124E030E0820E931EE0803A
:10E13000F180028113810AC0F40142E050E0840EB4
:10E14000951E808191817C0100271127198A2A8ED2
:10E150003B8E37FC02C05FEE452271E1C72ED12C09
:10E16000CC0EDD1EE114F1040105110529F48A8DA0
:10E170009B8D892B09F473C08E2D8770805DF6010D
:10E1800082936F0163E016950795F794E7946A957B
:10E19000D1F7E114F1040105110571F740FE5FC0EC
:10E1A000803309F45CC058C0F0E75F1679F4F401DD
:10E1B00022E030E0820E931E808191817C01002755
:10E1C000112731E0432A58E7552E16C043FE0AC0F6
:10E1D000F40144E050E0840E951EE080F18002815D
:10E1E00013810AC0F40182E090E0880E991E8081BC
:10E1F00091817C0100271127198A2A8E3B8E37FCDA
:10E2000002C09FEE4922E8E55E1629F442EEA42EF4
:10E2100049E0B42E04C033EFA32E39E0B32E21E140
:10E22000C22ED12CCC0EDD1EF701EF70F070EA0D7E
:10E23000FB1D8081F60182936F0194E0169507958E
:10E24000F794E7949A95D1F7E114F10401051105CB
:10E2500059F740FE04C0529280E382936F018E0111
:10E260000C191D090F5E1F4F0FC024E030E0820E15
:10E27000931E552009F48AC06E010894C11CD11C5C
:10E28000598201E010E0198A78014A8D5B8D0417EC
:10E2900015070CF47A018989882319F00894E11C88
:10E2A000F11C242C332484E1A82EB12CA220B3200D
:10E2B000A114B10469F4888D998D8E199F099C0170
:10E2C0004BEB59E06C897D898A899B890E94616E3C
:10E2D0008989882351F041E050E0BE016F5E7F4F95
:10E2E0008C899D89EA89FB890995F0E1AF16B10413
:10E2F00069F4888D998D8E199F099C014BEC59E02A
:10E300006C897D898A899B890E94616E2A8D3B8DEB
:10E31000201B310B2A8F3B8F4BEC59E06C897D8998
:10E320008A899B890E94616E0115110539F0A80147
:10E33000B6018C899D89EA89FB890995F0E55F160C
:10E3400019F4C6010E945A6E22FE0DC0888D998D67
:10E350008E199F099C014BEB59E06C897D898A8954
:10E360009B890E94616E288D398D2E153F053CF0EA
:10E370004E895F89420F531F4E8B5F8BEECC8E8987
:10E380009F898E0D9F1D8E8B9F8BE7CC8E899F89D9
:10E390006B960FB6F894DEBF0FBECDBFDF91CF9165
:10E3A0001F910F91FF90EF90DF90CF90BF90AF90B3
:10E3B0009F908F907F906F905F904F903F902F90A5
:10E3C0000895CF93DF93DC011296ED91FC911397A2
:10E3D000309729F41796ED91FC91189703C0018CA2
:10E3E000F28DE02D0995DF91CF910895CF93DF93C2
:10E3F000DC011296ED91FC911397309729F4199650
:10E40000ED91FC911A9703C0038CF48DE02D0995D2
:10E41000DF91CF910895CF93DF93CDB7DEB72197EA
:10E420000FB6F894DEBF0FBECDBFFC01848183FF21
:10E4300005C0877F84838581968110C041E050E0CC
:10E44000BE01640F751F808191810E94F36A01975C
:10E4500019F08FEF9FEF02C08981992721960FB69F
:10E46000F894DEBF0FBECDBFDF91CF9108950F931B
:10E470001F93CF93DF93CDB7DEB721970FB6F894F4
:10E48000DEBF0FBECDBF8C01FB01898341E050E0B0
:10E49000BE01640F751F808191810E94E171019717
:10E4A00011F00FEF1FEFC80121960FB6F894DEBFF1
:10E4B0000FBECDBFDF91CF911F910F910895E199CC
:10E4C000FECF9FBB8EBBE09A99278DB3089541156F
:10E4D000510569F0DC01E199FECF7FBB6EBBE09A8C
:10E4E0006F5F7F4F0DB20D9241505040B1F70895CC
:10E4F000E199FECF9FBB8EBB6DBB0FB6F894E29A3D
:10E50000E19A0FBE0895FC014150504038F001904F
:10E510000616D1F731978E2F9F2F089588279927B8
:10E520000895FB01DC0104C08D910190801921F454
:10E5300041505040C8F7881B990B0895FB01DC013E
:10E5400002C001900D9241505040D8F70895FB0150
:10E55000DC0102C005900D9241505040D8F708955B
:10E56000DC0101C06D9341505040E0F70895FB017C
:10E57000DC018D916191562F5062513624F05B374A
:10E5800014F460628062861B11F4662391F7990B84
:10E590000895FB01DC010D900020E9F7119701902F
:10E5A0000D920020E1F70895FC010190061629F074
:10E5B0000020D9F788279927089531978E2F9F2F0C
:10E5C0000895FB01DC018D910190801911F4002068
:10E5D000D1F7990B0895FB01DC018D91059080190D
:10E5E00011F40020D1F7990B0895FB01DC01019093
:10E5F0000D920020E1F70895FB01DC0105900D92DA
:10E600000020E1F70895FC0105900020E9F78095CE
:10E6100090958E0F9F1F0895FB01DC0141505040E3
:10E6200070F08D913191232F2062213624F02B3709
:10E6300014F430628062831B19F4332379F7881B4A
:10E64000990B0895FB01DC014150504048F00190C6
:10E650000D920020C9F701C01D9241505040E0F7D3
:10E660000895FC0181E090E00190061611F48E2FD0
:10E670009F2F0020C9F701970895629FD001739FD3
:10E68000F001829FE00DF11D649FE00DF11D929F4E
:10E69000F00D839FF00D749FF00D659FF00D99278D
:10E6A000729FB00DE11DF91F639FB00DE11DF91FB1
:10E6B000BD01CF0111240895991B79E004C0991F71
:10E6C000961708F0961B881F7A95C9F780950895CC
:10E6D000AA1BBB1B51E107C0AA1FBB1FA617B70788
:10E6E00010F0A61BB70B881F991F5A95A9F78095A4
:10E6F0009095BC01CD01089597FB092E07260AD0FD
:10E7000077FD04D0E5DF06D000201AF470956195FE
:10E710007F4F0895F6F7909581959F4F0895A1E258
:10E720001A2EAA1BBB1BFD010DC0AA1FBB1FEE1F8B
:10E73000FF1FA217B307E407F50720F0A21BB30BD6
:10E74000E40BF50B661F771F881F991F1A9469F752
:10E7500060957095809590959B01AC01BD01CF01AE
:02E7600008951A
:10E76200342E312E320000010006980000006D6147
:10E77200696E00504F52544220626974732030789F
:10E78200253032580A07005B253032582D253032A9
:10E79200585D00504F52544420626974732030789F
:10E7A200253032580A0700504F525445206269748E
:10E7B20073203078253032580A0700504F525446A1
:10E7C2002062697473203078253032580A07000AB3
:10E7D2000A426173654D6F6E2025730A4E75742F60
:10E7E2004F532025730A00436F6D70696C65642076
:10E7F200627920004156524743430020666F7220DF
:10E8020041546D656761003132380042617564724E
:10E812006174652073656C656374203D2025640A0C
:10E82200004E6F207573657220696E707574206476
:10E83200657465637465640045787465726E616CB5
:10E842002052414D20546573742E2E2E20002575C2
:10E852002062797465730A0042616E6B65642052AE
:10E86200414D20546573742E2E2E202020002575D4
:10E872002062616E6B732C2025752062797465733A
:10E882002065612E0A006E6F6E65005365726961C4
:10E892006C20464C4153482E2E2E20202020202032
:10E8A20000256C752062797465730A00446574658D
:10E8B2006374696E67204E49432E2E2E202020203D
:10E8C20020006E6F6E65070052544C38303139416A
:10E8D20053004C414E393143313131005465737428
:10E8E200696E67204E49432E2E2E202020202020A4
:10E8F2002000492F4F20506F727420546573742E7C
:10E902002E2E2020202020004F4B00426F6F746972
:10E912006E672E2E2E000A4D41432061646472659B
:10E92200737320282530325825303258253032581A
:10E93200253032582530325825303258293A2000B5
:10E94200426164204D4143206164647265737300C7
:10E95200486F7374206E616D6520282573293A20F3
:10E962000049502061646472657373004E657420BF
:10E972006D61736B0044656661756C7420726F75AE
:10E982007465005573696E672044484350206F7266
:10E9920020415250206D6574686F64202859293ACD
:10E9A20020000A0077007561727430006574686532
:10E9B200726E757400657468300069646C6500433A
:10E9C2006865636B206164647265737320616E6451
:10E9D2002064617461206275732E004E6F20524173
:10E9E2004D206174203078253034580A0053572D59
:10E9F20052657365742E2E2E004F4B006661696C52
:10EA02006564070048572D5265736574000D69648B
:10EA12003D30782530345800006661696C65642C9D
:10EA220020676F74203078253034582C2065787038
:10EA32006563746564203078373035300A0700002A
:10EA42000698000000496E697420636F6E74726FDD
:10EA52006C6C65722E2E2E00206465746563746979
:10EA62006E672E2E2E00454550524F4D20456D7536
:10EA72006C6174696F6E2E2E2E00646F6E6500528B
:10EA8200544C38303139415320006A756D706572CB
:10EA9200206D6F64653A20004155492000504E5068
:10EAA200200052544C383031392000556E6B6E6F55
:10EAB200776E20636869702000424E43072000464B
:10EAC20061696C6564072000495251257520004137
:10EAD20075746F200031304261736554200031300B
:10EAE2004261736535200031304261736532200026
:10EAF2000D256C75007265736574206661696C65BD
:10EB0200640049525120737475636B006C696E6BBB
:10EB1200206661696C6564006E6F2049525100493C
:10EB22005251206661696C656400416C6C6F6320B0
:10EB32006661696C6564006261642076616C20259F
:10EB420030345820617420253034580A00427566EA
:10EB5200206661696C6564004F4B000006980000F6
:10EB6200000A496E697420636F6E74726F6C6C6513
:10EB7200722E2E2E00416C6C6F6300456E717565AE
:10EB82007565000D256C750020416C6C6F63000D7E
:10EB92007265763D307825303258202020202020A2
:10EBA20020200000257320282573293A2000010720
:10EBB200170B0C19052F330309020E1D403B5F672B
:10EBC200778154524D003C464F4E5420434F4C4F98
:10EBD200523D234343303030303E52554E3C2F4657
:10EBE2004F4E543E003C464F4E5420434F4C4F52E2
:10EBF2003D233333393936363E5244593C2F464F42
:10EC02004E543E00534C5000620566058505A4052E
:10EC12004F6B00746578742F68746D6C00436F726B
:10EC220072004F4B004C495354454E0053594E53BA
:10EC3200454E540053594E524356440046494E578E
:10EC4200414954310046494E574149543200434CE0
:10EC52004F53455741495400434C4F53494E470087
:10EC62004C41535441434B0054494D45574149543B
:10EC720000434C4F534544003F554E4B3F003C2F01
:10EC820054443E3C2F54523E0D0A003E3C2F7464C5
:10EC92003E0D0A003C2F74723E0D0A00444452415C
:10ECA2000050494E4100504F525441004444524298
:10ECB2000050494E4200504F52544200504F52545D
:10ECC2004300444452440050494E4400504F525471
:10ECD2004400444452450050494E4500504F52545E
:10ECE200450050494E460065746830004D4143204E
:10ECF20020253032582D253032582D253032582DCE
:10ED0200253032582D253032582D253032580A49B7
:10ED1200502020202573000A4D61736B202573005B
:10ED22000A41646420676174657761792025730004
:10ED32000A47617465202573000A485454502073B1
:10ED420065727665722072756E6E696E672E2055D9
:10ED5200524C20687474703A2F2F25732F0A007456
:10ED62006872656164732E6367690074696D6572A8
:10ED72002E63676900736F636B6574732E636769D3
:10ED820000706F7274732E63676900722B620000E9
:10ED9200004B12020B49072F072818D205561237CB
:10EDA20007B519820133183F0700103235352E326C
:10EDB20035352E3235352E3000746370736D006137
:10EDC2007270657800638253636468637063002EB7
:10EDD20074787400746578742F706C61696E002E9B
:10EDE20068746D6C00746578742F68746D6C002E95
:10EDF20068746D002E67696600696D6167652F67CB
:10EE02006966002E6A706700696D6167652F6A70B6
:10EE12006567002E706466006170706C696361746E
:10EE2200696F6E2F706466002E6A73006170706C79
:10EE320069636174696F6E2F782D6A61766173639D
:10EE420072697074006F0774077F0785078F0785E3
:10EE52000794079907A307A807B307B807C807CC01
:10EE620007426164205265717565737400556E6165
:10EE72007574686F72697A6564004E6F7420466FAC
:10EE8200756E6400496E7465726E616C20457272B3
:10EE92006F72004E6F7420496D706C656D656E7493
:10EEA2006564004572726F72002E006367692D629D
:10EEB200696E2F0055524F4D3A002F00696E6465FE
:10EEC200782E68746D6C004F6B00417574686F72B8
:10EED200697A6174696F6E3A00436F6E74656E741D
:10EEE2002D4C656E6774683A00436F6E74656E747C
:10EEF2002D547970653A00436F6F6B69653A00551E
:10EF02007365722D4167656E743A00474554004837
:10EF120045414400504F535400485454502F302E12
:10EF220039002E0042617369632000000055524F80
:10EF32004D00000000000100000000000000000081
:10EF420000006F50A650A950AC500E5125518000C0
:10EF5200332E352E302E3000000075617274300071
:10EF62000000000000000000000000AC597C5900C5
:10EF720000BB59DB59FC590B5A0000727869350005
:10EF82000600000000000000000000000000000079
:10EF9200000000DC0500000000D265C15D0A6600C9
:10EFA20000657468300000000000030000002009C2
:10EFB200720AF95D0000000000000000000000007D
:10EFC2000000060000000000000000000000000039
:10EFD2000000000000DC0500000000D265E8630AC2
:10EFE2006600006574683000000000000300000045
:10EFF2006209940A09640000000000000000000099
:10F002000000000072786935000010010002000360
:10F01200000000000000000000000020202020204E
:10F02200202020202020202020202030303030308E
:10F032003030303030303030303030286E756C6CDB
:10F04200290030313233343536373839414243447E
:10F0520045460030313233343536373839616263F0
:04F06200646566007B
:00000001FF
